 SSPH

 Timestamp is 5b98875a (Wed Sep 12 12:26:18 2018)

 Preferred load address is 00400000

 Start         Length     Name                   Class
 0001:00000000 00028704H .text                   CODE
 0001:00028710 0000159aH .text$x                 CODE
 0002:00000000 00000298H .idata$5                DATA
 0002:00000298 000085cfH .rdata                  DATA
 0002:00008868 000016b0H .xdata$x                DATA
 0002:00009f18 000000a0H .idata$2                DATA
 0002:00009fb8 00000014H .idata$3                DATA
 0002:00009fcc 00000298H .idata$4                DATA
 0002:0000a264 00000b92H .idata$6                DATA
 0002:0000adf6 00000000H .edata                  DATA
 0003:00000000 00000004H .CRT$XCA                DATA
 0003:00000004 00000024H .CRT$XCU                DATA
 0003:00000028 00000004H .CRT$XCZ                DATA
 0003:0000002c 00000004H .CRT$XIA                DATA
 0003:00000030 0000000cH .CRT$XIC                DATA
 0003:0000003c 00000004H .CRT$XIY                DATA
 0003:00000040 00000004H .CRT$XIZ                DATA
 0003:00000044 00000004H .CRT$XLA                DATA
 0003:00000048 00000004H .CRT$XLZ                DATA
 0003:0000004c 00000004H .CRT$XPA                DATA
 0003:00000050 00000004H .CRT$XPX                DATA
 0003:00000054 00000004H .CRT$XPZ                DATA
 0003:00000058 00000004H .CRT$XTA                DATA
 0003:0000005c 00000004H .CRT$XTB                DATA
 0003:00000060 00000004H .CRT$XTZ                DATA
 0003:00000070 0000330cH .data                   DATA
 0003:00003380 00003408H .bss                    DATA
 0004:00000000 00000004H .tls                    DATA
 0004:00000008 00001cd8H .tls$                   DATA
 0004:00001ce0 00000004H .tls$ZZZ                DATA
 0005:00000000 00000130H .rsrc$01                DATA
 0005:00000130 00001300H .rsrc$02                DATA

  Address         Publics by Value              Rva+Base     Lib:Object

 0001:00000000       ??1JLockable@@UAE@XZ       00401000 f i j_criticalsection.obj
 0001:00000010       ?SharedLock@JLockable@@UAE_NJ@Z 00401010 f i j_criticalsection.obj
 0001:00000020       ?SharedUnlock@JLockable@@UAEXXZ 00401020 f i j_criticalsection.obj
 0001:00000030       ??_GJLockable@@UAEPAXI@Z   00401030 f i j_criticalsection.obj
 0001:00000030       ??_EJLockable@@UAEPAXI@Z   00401030 f i j_criticalsection.obj
 0001:00000060       ??0JDynLoadSystem@@QAE@PBD@Z 00401060 f i j_criticalsection.obj
 0001:00000150       ??1JDynLoadStub@@UAE@XZ    00401150 f i j_criticalsection.obj
 0001:00000160       ?SetModuleName@JDynLoadStub@@UAEXPBD@Z 00401160 f i j_criticalsection.obj
 0001:00000160       ?Load@JDynLoadStub@@UAEXPBD@Z 00401160 f i j_criticalsection.obj
 0001:00000170       ?GetProc@JDynLoadStub@@UAEPAXPBD@Z 00401170 f i j_criticalsection.obj
 0001:00000180       ??_EJDynLoadStub@@UAEPAXI@Z 00401180 f i j_criticalsection.obj
 0001:00000180       ??_GJDynLoadStub@@UAEPAXI@Z 00401180 f i j_criticalsection.obj
 0001:000001b0       ??1JDynLoad@@UAE@XZ        004011b0 f i j_criticalsection.obj
 0001:00000210       ?Load@JDynLoad@@UAEXPBD@Z  00401210 f i j_criticalsection.obj
 0001:00000240       ??_EJDynLoad@@UAEPAXI@Z    00401240 f i j_criticalsection.obj
 0001:00000240       ??_GJDynLoad@@UAEPAXI@Z    00401240 f i j_criticalsection.obj
 0001:00000270       ??_EJDynLoadSystem@@UAEPAXI@Z 00401270 f i j_criticalsection.obj
 0001:00000270       ??_GJDynLoadSystem@@UAEPAXI@Z 00401270 f i j_criticalsection.obj
 0001:000002a0       ??1JDynLoadSystem@@UAE@XZ  004012a0 f i j_criticalsection.obj
 0001:00000300       ?SetNum@?$JArray@D@@QAEXK@Z 00401300 f i j_criticalsection.obj
 0001:00000350       ?InternalLoad@JDynLoad@@AAE_NXZ 00401350 f   j_dynload.obj
 0001:00000420       ?InternalUnload@JDynLoad@@AAEXXZ 00401420 f   j_dynload.obj
 0001:00000440       ?GetProc@JDynLoad@@UAEPAXPBD@Z 00401440 f   j_dynload.obj
 0001:00000470       ?SetModuleName@JDynLoad@@UAEXPBD@Z 00401470 f   j_dynload.obj
 0001:00000490       ?SetModuleName@JDynLoadSystem@@UAEXPBD@Z 00401490 f   j_dynload.obj
 0001:000004b0       ?Create@JMutex@@QAEHPBDH@Z 004014b0 f   j_mutex.obj
 0001:000004e0       ?Release@JMutex@@QAEXXZ    004014e0 f   j_mutex.obj
 0001:00000500       ?Lock@JMutex@@UAE_NJ@Z     00401500 f   j_mutex.obj
 0001:00000540       ?Unlock@JMutex@@UAEXXZ     00401540 f   j_mutex.obj
 0001:00000550       ??0JTokenStream@@QAE@XZ    00401550 f   j_stoken.obj
 0001:00000580       ??1JTokenStream@@QAE@XZ    00401580 f   j_stoken.obj
 0001:00000590       ?ReadEOL@JTokenStream@@IAEIAAPAD@Z 00401590 f   j_stoken.obj
 0001:00000640       ?SetSeparator@JTokenStream@@QAEXD@Z 00401640 f   j_stoken.obj
 0001:00000660       ?Open@JTokenStream@@QAEHPBD@Z 00401660 f   j_stoken.obj
 0001:00000700       ?Init@JTokenStream@@IAEXPAX@Z 00401700 f   j_stoken.obj
 0001:000007c0       ?Close@JTokenStream@@QAEXXZ 004017c0 f   j_stoken.obj
 0001:000007f0       ?ReadToken@JTokenStream@@IAEPADH@Z 004017f0 f   j_stoken.obj
 0001:00000830       ?NextToken@JTokenStream@@IAEHH@Z 00401830 f   j_stoken.obj
 0001:00000930       ?IsNextLineExist@JTokenStream@@QAE_NXZ 00401930 f   j_stoken.obj
 0001:00000950       ?NextLineIfNotLineEnd@JTokenStream@@QAEHXZ 00401950 f   j_stoken.obj
 0001:00000970       ?ProcessReturnPointer@JTokenStream@@IAEPADPAD@Z 00401970 f   j_stoken.obj
 0001:000009c0       ??0JString@@QAE@XZ         004019c0 f i j_str.obj
 0001:00000a90       ??1JWString@@QAE@XZ        00401a90 f   j_str.obj
 0001:00000a90       ??1JString@@QAE@XZ         00401a90 f   j_str.obj
 0001:00000ac0       ??4JString@@QAEAAV0@PBD@Z  00401ac0 f   j_str.obj
 0001:00000ba0       ??4JString@@QAEAAV0@ABV0@@Z 00401ba0 f   j_str.obj
 0001:00000ce0       ?Cat@JString@@QAEXPBDK@Z   00401ce0 f   j_str.obj
 0001:00000d90       ?Remove@JString@@QAE_NPBD@Z 00401d90 f   j_str.obj
 0001:00000e90       ?RemoveLast@JString@@QAEXJ@Z 00401e90 f   j_str.obj
 0001:00000f70       ?Replace@JString@@QAEHPBD0@Z 00401f70 f   j_str.obj
 0001:00001180       ?Find@JString@@QBEJPBDJ@Z  00402180 f   j_str.obj
 0001:000011b0       ?ConvEUCKRtoISOKR@JString@@QAEHXZ 004021b0 f   j_str.obj
 0001:000014a0       ?ConvHZtoGB2312@JString@@QAEHXZ 004024a0 f   j_str.obj
 0001:00001550       ?ConvGB2312toHZ@JString@@QAEHXZ 00402550 f   j_str.obj
 0001:000017f0       ?ConvEUCtoSJIS@JString@@QAEHXZ 004027f0 f   j_str.obj
 0001:00001930       ?ConvSJIStoEUC@JString@@QAEHXZ 00402930 f   j_str.obj
 0001:00001c20       ?ConvISOtoWindows@JString@@AAEHXZ 00402c20 f   j_str.obj
 0001:00001d80       ?ConvSJIStoJIS@JString@@QAEHXZ 00402d80 f   j_str.obj
 0001:00002120       ??0JString@@QAE@ABVJWString@@@Z 00403120 f   j_str.obj
 0001:00002170       ??4JString@@QAEAAV0@ABVJWString@@@Z 00403170 f   j_str.obj
 0001:00002190       ??4JString@@QAEAAV0@PBG@Z  00403190 f   j_str.obj
 0001:000021b0       ??YJString@@QAEAAV0@PBG@Z  004031b0 f   j_str.obj
 0001:00002240       ?ToMbs@JString@@QAEKABVJWString@@H@Z 00403240 f   j_str.obj
 0001:00002260       ?ToMbs@JString@@QAEKPBGPBD@Z 00403260 f   j_str.obj
 0001:00002390       ?ToMbs@JString@@QAEKPBGH@Z 00403390 f   j_str.obj
 0001:000025a0       ?ToMbsFunc@JString@@QAEKPBGH@Z 004035a0 f   j_str.obj
 0001:00002730       ?ConvUnicodeToUTF8@JString@@QAEKPBG@Z 00403730 f   j_str.obj
 0001:000029d0       ?Add@JString@@QAEXD@Z      004039d0 f i j_str.obj
 0001:00002b20       ?Last@?$JArray@D@@QAEAADXZ 00403b20 f i j_str.obj
 0001:00002b40       ?Release@?$JArray@G@@QAEXXZ 00403b40 f i j_str.obj
 0001:00002b40       ?Release@?$JArray@PAX@@QAEXXZ 00403b40 f i j_str.obj
 0001:00002b40       ??1SPUtils@@QAE@XZ         00403b40 f i j_str.obj
 0001:00002b40       ??1?$JPtrArray@PAG@@QAE@XZ 00403b40 f i j_str.obj
 0001:00002b40       ??1?$JPtrArray@PAE@@QAE@XZ 00403b40 f i j_str.obj
 0001:00002b40       ?Release@?$JArray@D@@QAEXXZ 00403b40 f i j_str.obj
 0001:00002b40       ??1?$JArray@G@@QAE@XZ      00403b40 f i j_str.obj
 0001:00002b40       ??1?$JPtrArray@PAVSPURLTranslateData@@@@QAE@XZ 00403b40 f i j_str.obj
 0001:00002b40       ??1?$JPtrArray@PAVJWString@@@@QAE@XZ 00403b40 f i j_str.obj
 0001:00002b40       ??1?$JArray@D@@QAE@XZ      00403b40 f i j_str.obj
 0001:00002b40       ??1?$JPtrArray@PAD@@QAE@XZ 00403b40 f i j_str.obj
 0001:00002b40       ??1?$JArray@PAX@@QAE@XZ    00403b40 f i j_str.obj
 0001:00002b40       ?Release@?$JArray@K@@QAEXXZ 00403b40 f i j_str.obj
 0001:00002b40       ??1?$JArray@K@@QAE@XZ      00403b40 f i j_str.obj
 0001:00002b70       ?Size@?$JArray@D@@QBEKXZ   00403b70 f i j_str.obj
 0001:00002b90       ?Alloc@?$JArray@D@@QAE_NK@Z 00403b90 f i j_str.obj
 0001:00002c70       ?SetNumNoPurge@?$JArray@D@@QAEXK_N@Z 00403c70 f i j_str.obj
 0001:00002cd0       ?SwapBuffer@?$JArray@D@@QAEXAAV1@@Z 00403cd0 f i j_str.obj
 0001:00002e80       ?Realloc@?$JArray@D@@QAE_NK@Z 00403e80 f i j_str.obj
 0001:00002f40       ?Add@?$JArray@D@@QAEAADXZ  00403f40 f i j_str.obj
 0001:000030c0       ??0JWString@@QAE@XZ        004040c0 f i j_wstr.obj
 0001:000031a0       ??4JWString@@QAEAAV0@PBG@Z 004041a0 f   j_wstr.obj
 0001:00003280       ??4JWString@@QAEAAV0@ABV0@@Z 00404280 f   j_wstr.obj
 0001:000033d0       ?Cat@JWString@@QAEXPBGK@Z  004043d0 f   j_wstr.obj
 0001:00003490       ?RemoveLast@JWString@@QAEXJ@Z 00404490 f   j_wstr.obj
 0001:00003580       ?Remove@JWString@@QAE_NJJ@Z 00404580 f   j_wstr.obj
 0001:00003620       ?Find@JWString@@QBEJPBGJ@Z 00404620 f   j_wstr.obj
 0001:00003650       ?FindList@JWString@@QBEJPBGJK@Z 00404650 f   j_wstr.obj
 0001:000036c0       ?ReverseFindList@JWString@@QBEJPBGJK@Z 004046c0 f   j_wstr.obj
 0001:00003730       ?ExtractRight@JWString@@QBE?AV1@K@Z 00404730 f   j_wstr.obj
 0001:000037a0       ?ExtractLeft@JWString@@QBE?AV1@K@Z 004047a0 f   j_wstr.obj
 0001:000038e0       ??YJWString@@QAEAAV0@PBD@Z 004048e0 f   j_wstr.obj
 0001:00003950       ?ConvUTF8ToUnicode@JWString@@AAEKPBD@Z 00404950 f   j_wstr.obj
 0001:00003c20       ?ConvMSUnicode@JWString@@QAEXXZ 00404c20 f   j_wstr.obj
 0001:00003c90       ?GetDefaultCodePage@JWString@@SIHXZ 00404c90 f   j_wstr.obj
 0001:00003cb0       ?GetCodePage@JWString@@SIHPBD@Z 00404cb0 f   j_wstr.obj
 0001:00003db0       ?GetCodePageText@JWString@@SIPBDH@Z 00404db0 f   j_wstr.obj
 0001:00003de0       ?ToUnicode@JWString@@QAEKPBD0@Z 00404de0 f   j_wstr.obj
 0001:00003f20       ?ToUnicode@JWString@@QAEKPBDH@Z 00404f20 f   j_wstr.obj
 0001:000041b0       ?ToUnicodeFunc@JWString@@AAEKPBDH@Z 004051b0 f   j_wstr.obj
 0001:000042e0       ??0?$JArray@D@@QAE@K@Z     004052e0 f i j_wstr.obj
 0001:00004370       ?Size@?$JArray@G@@QBEKXZ   00405370 f i j_wstr.obj
 0001:00004390       ?SetNum@?$JArray@G@@QAEXK@Z 00405390 f i j_wstr.obj
 0001:000043e0       ?SetNumNoPurge@?$JArray@G@@QAEXK_N@Z 004053e0 f i j_wstr.obj
 0001:00004440       ?Realloc@?$JArray@G@@QAE_NK@Z 00405440 f i j_wstr.obj
 0001:00004510       ?Add@?$JArray@G@@QAEAAGXZ  00405510 f i j_wstr.obj
 0001:00004600       ?JGXMakeSystemPath@@YAPBDPBD@Z 00405600 f   jgxbase.obj
 0001:00004700       ?atol_impl@@YIJPBD@Z       00405700 f   libc_custom.obj
 0001:00004750       ?wtol_impl@@YIJPBG@Z       00405750 f   libc_custom.obj
 0001:000047c0       ?stricmp_custom@@YIHPBD0@Z 004057c0 f   libc_custom.obj
 0001:00004830       ?wcsicmp_custom@@YIHPBG0@Z 00405830 f   libc_custom.obj
 0001:000048d0       ?strnicmp_custom@@YIHPBD0I@Z 004058d0 f   libc_custom.obj
 0001:00004990       ?stricmp_opt@@YIHPBD0@Z    00405990 f   libc_custom.obj
 0001:00004a00       ?wcsicmp_opt@@YIHPBG0@Z    00405a00 f   libc_custom.obj
 0001:00004a80       ?strnicmp_opt@@YIHPBD0I@Z  00405a80 f   libc_custom.obj
 0001:00004b10       ?strstri_custom@@YIPADPBD0@Z 00405b10 f   libc_custom.obj
 0001:00004be0       ?strstri_opt@@YIPADPBD0@Z  00405be0 f   libc_custom.obj
 0001:00004ca0       ?strlcat@@YAIPADPBDI@Z     00405ca0 f   libc_custom.obj
 0001:00004d30       ?strlcpy@@YAIPADPBDI@Z     00405d30 f   libc_custom.obj
 0001:00004d90       _sp_resetstkoflw           00405d90 f   resetstk.obj
 0001:00004ef0       ??0SPAdjustPrivADVAPI32@@QAE@XZ 00405ef0 f   sp_adjustpriv.obj
 0001:00004fe0       ??1SPAdjustPrivADVAPI32@@QAE@XZ 00405fe0 f   sp_adjustpriv.obj
 0001:00005040       ?OpenProcessToken@SPAdjustPrivADVAPI32@@QAEHPAXKPAPAX@Z 00406040 f   sp_adjustpriv.obj
 0001:00005070       ?LookupPrivilegeValueA@SPAdjustPrivADVAPI32@@QAEHPAD0PAU_LUID@@@Z 00406070 f   sp_adjustpriv.obj
 0001:000050a0       ?AdjustTokenPrivileges@SPAdjustPrivADVAPI32@@QAEHPAXHPAU_TOKEN_PRIVILEGES@@K1PAK@Z 004060a0 f   sp_adjustpriv.obj
 0001:000050d0       ?GetTokenInformation@SPAdjustPrivADVAPI32@@QAEHPAXW4INFO_TOKEN_INFORMATION_CLASS@@0KPAK@Z 004060d0 f   sp_adjustpriv.obj
 0001:00005100       ??0SPAdjustPriv@@QAE@PADH@Z 00406100 f   sp_adjustpriv.obj
 0001:000051f0       ??1SPAdjustPriv@@QAE@XZ    004061f0 f   sp_adjustpriv.obj
 0001:00005350       ??0SPNTPrivSystem@@QAE@XZ  00406350 f   sp_adjustpriv.obj
 0001:000053c0       ??1SPNTPrivSystem@@QAE@XZ  004063c0 f   sp_adjustpriv.obj
 0001:000053e0       ?GetSPNTPrivSystem@@YAAAVSPNTPrivSystem@@XZ 004063e0 f   sp_adjustpriv.obj
 0001:00005430       ?IsNT@SPNTPrivSystem@@AAE_NXZ 00406430 f   sp_adjustpriv.obj
 0001:00005440       ?SetPriv@SPNTPrivSystem@@QAE_NPADH@Z 00406440 f   sp_adjustpriv.obj
 0001:00005500       ?IsUAC@SPNTPrivSystem@@QAE_NXZ 00406500 f   sp_adjustpriv.obj
 0001:000055c0       ?IsElevated@SPNTPrivSystem@@QAE_NXZ 004065c0 f   sp_adjustpriv.obj
 0001:00005640       __purecall                 00406640 f   sp_debugger.obj
 0001:00005650       ?GetEip@@YAKXZ             00406650 f   sp_debugger.obj
 0001:00005660       ?trace_and_exit@@YAXXZ     00406660 f   sp_debugger.obj
 0001:00005700       ?sig_trace_and_exit@@YAXH@Z 00406700 f   sp_debugger.obj
 0001:00005770       ?SPSEDefaultFilter@@YGJPAU_EXCEPTION_POINTERS@@@Z 00406770 f   sp_debugger.obj
 0001:00006780       ?SPGetExceptionReasonTextA@@YAPADK@Z 00407780 f   sp_debugger.obj
 0001:00006b40       ??1SPVersionInfo@@QAE@XZ   00407b40 f i sp_debugger.obj
 0001:00006e50       ?SPCalcCodeStartPos@@YAPAXPAXAAHPAPAXPAK@Z 00407e50 f   sp_debugger.obj
 0001:00007330       ?Release@SPEventObject@@QAEXXZ 00408330 f   sp_eventobj.obj
 0001:00007350       ?Create@SPEventObject@@QAE_N_N0@Z 00408350 f   sp_eventobj.obj
 0001:000073c0       ?Activate@SPEventObject@@QAEXXZ 004083c0 f   sp_eventobj.obj
 0001:000073d0       ?DeActivate@SPEventObject@@QAEXXZ 004083d0 f   sp_eventobj.obj
 0001:00007420       ??0SPFindFile@@QAE@XZ      00408420 f   sp_findfile.obj
 0001:00007530       ?Close@SPFindFile@@QAEXXZ  00408530 f   sp_findfile.obj
 0001:00007560       ?First@SPFindFile@@QAE_NPBD@Z 00408560 f   sp_findfile.obj
 0001:000077b0       ?Next@SPFindFile@@QAE_NXZ  004087b0 f   sp_findfile.obj
 0001:00007870       ??0SPKeiArchiver@@QAE@XZ   00408870 f   sp_kei.obj
 0001:00007880       ?LoadVarTxt@SPProp@@QAEXXZ 00408880 f   sp_kei.obj
 0001:00007880       ??1SPKeiArchiver@@QAE@XZ   00408880 f   sp_kei.obj
 0001:00007880       ??1SPSystemInfo@@QAE@XZ    00408880 f   sp_kei.obj
 0001:00007890       ?Extract@SPKeiArchiver@@QAEHPAD00H@Z 00408890 f   sp_kei.obj
 0001:00007900       ?SPM_Dummy_load@@YAHPAXJ@Z 00408900 f   sp_module.obj
 0001:00007920       ?SPM_Dummy_unload@@YAHXZ   00408920 f   sp_module.obj
 0001:00007930       ?SPM_Dummy_request@@YAPAXPAXPAJ@Z 00408930 f   sp_module.obj
 0001:00007950       ??0SPModule@@QAE@XZ        00408950 f   sp_module.obj
 0001:00007c20       ??0JWString@@QAE@PBG@Z     00408c20 f i sp_module.obj
 0001:00007c70       ??1SPVarSystemNode@@UAE@XZ 00408c70 f i sp_module.obj
 0001:00007c80       ??_GSPVarSystemNode@@UAEPAXI@Z 00408c80 f i sp_module.obj
 0001:00007c80       ??_ESPVarSystemNode@@UAEPAXI@Z 00408c80 f i sp_module.obj
 0001:00007cb0       ??1SPProp@@UAE@XZ          00408cb0 f i sp_module.obj
 0001:00007d80       ??_ESPProp@@UAEPAXI@Z      00408d80 f i sp_module.obj
 0001:00007d80       ??_GSPProp@@UAEPAXI@Z      00408d80 f i sp_module.obj
 0001:00007db0       ??0SPParamManager@@QAE@XZ  00408db0 f i sp_module.obj
 0001:00007ef0       ??1SPStaticStringArrayW@@QAE@XZ 00408ef0 f i sp_module.obj
 0001:00007f80       ??1SPStaticStringArrayA@@QAE@XZ 00408f80 f i sp_module.obj
 0001:00008010       ??1SPParamManager@@QAE@XZ  00409010 f i sp_module.obj
 0001:00008150       ??1JMutex@@UAE@XZ          00409150 f i sp_module.obj
 0001:000081a0       ??_GJMutex@@UAEPAXI@Z      004091a0 f i sp_module.obj
 0001:000081a0       ??_EJMutex@@UAEPAXI@Z      004091a0 f i sp_module.obj
 0001:000081d0       ?Lock@SPModule@@UAE_NJ@Z   004091d0 f i sp_module.obj
 0001:000081f0       ?Unlock@SPModule@@UAEXXZ   004091f0 f i sp_module.obj
 0001:00008200       ??_GSPModule@@UAEPAXI@Z    00409200 f i sp_module.obj
 0001:00008200       ??_ESPModule@@UAEPAXI@Z    00409200 f i sp_module.obj
 0001:00008230       ??1SPModule@@UAE@XZ        00409230 f   sp_module.obj
 0001:00008470       ?Release@SPModule@@UAEXXZ  00409470 f   sp_module.obj
 0001:00008480       ?LoadLib@SPModule@@QAE_NPBD@Z 00409480 f   sp_module.obj
 0001:000089f0       ?UnloadLib@SPModule@@QAE_NXZ 004099f0 f   sp_module.obj
 0001:00008b60       ?CheckReentrant@SPModule@@AAE_NPBG@Z 00409b60 f   sp_module.obj
 0001:00008b90       ?ExecLoadSEHReal@SPModule@@AAEHP6AHPAXJ@Z0J@Z 00409b90 f   sp_module.obj
 0001:00008cd0       ?ExecLoadSEH@SPModule@@QAEHP6AHPAXJ@Z0J@Z 00409cd0 f   sp_module.obj
 0001:00008e90       ?ExecUnloadSEHReal@SPModule@@AAEHP6AHXZ@Z 00409e90 f   sp_module.obj
 0001:00008fc0       ?ExecUnloadSEH@SPModule@@QAEHP6AHXZ@Z 00409fc0 f   sp_module.obj
 0001:00009130       ?ExecRequestSEHReal@SPModule@@AAEPAXP6APAXPAXPAJ@Z01@Z 0040a130 f   sp_module.obj
 0001:00009260       ?ExecRequestSEH@SPModule@@QAEPAXP6APAXPAXPAJ@Z01@Z 0040a260 f   sp_module.obj
 0001:00009490       ?ExecGetSEH@SPModule@@QAEPAGP6APAXPAJ@Z@Z 0040a490 f   sp_module.obj
 0001:00009600       ?CallRequestAndLog@SPModule@@QAEPAXAAVJString@@AAJ@Z 0040a600 f   sp_module.obj
 0001:00009720       ??1JUnlock@@QAE@XZ         0040a720 f i sp_module.obj
 0001:00009730       ?WriteLog@SPModule@@QAEXPADPAXHK@Z 0040a730 f   sp_module.obj
 0001:00009740       ?CallGetVersionAndLoad@SPModule@@IAE?AVSPModuleGetVersionResult@@PAG@Z 0040a740 f   sp_module.obj
 0001:00009900       ?GetGenericProcAddress@SPModule@@IAEXXZ 0040a900 f   sp_module.obj
 0001:000099a0       ?SetPath@SPModule@@UAEXPAD@Z 0040a9a0 f   sp_module.obj
 0001:00009a10       ?ToString@SPModule@@QAEPAGPAXJ@Z 0040aa10 f   sp_module.obj
 0001:00009ae0       ?ToHandleASub@SPModule@@IAEPAXPBDAAJ@Z 0040aae0 f   sp_module.obj
 0001:00009b20       ?ToHandleA@SPModule@@QAEPAXAAVJString@@AAJ@Z 0040ab20 f   sp_module.obj
 0001:00009b40       ?GetLoadPath@SPModule@@QAEPAXAAJ@Z 0040ab40 f   sp_module.obj
 0001:00009b60       ?GMFree@SPModule@@SAXPAX@Z 0040ab60 f   sp_module.obj
 0001:00009bc0       ?GMSize@SPModule@@SAJPAXJ@Z 0040abc0 f   sp_module.obj
 0001:00009c40       ?GetProcAddressModule@SPModule@@QAEPAXPAD@Z 0040ac40 f   sp_module.obj
 0001:00009c80       ?ParseCharset@SPModule@@QAEXXZ 0040ac80 f   sp_module.obj
 0001:00009d20       ?MakeLastReference@SPModule@@IAEPAGPAPAGK0K@Z 0040ad20 f   sp_module.obj
 0001:00009ec0       ?SendRecvPipeSSPEXT@SPModule@@AAE_NPBD0AAVJString@@@Z 0040aec0 f   sp_module.obj
 0001:0000a220       ?SendRecvPipeSHIOLINK@SPModule@@AAE_NPBD0AAVJString@@@Z 0040b220 f   sp_module.obj
 0001:0000a600       ?SendRecvPipe@SPModule@@IAE_NPBD0AAVJString@@@Z 0040b600 f   sp_module.obj
 0001:0000a640       ?Last@?$JArray@G@@QAEAAGXZ 0040b640 f i sp_module.obj
 0001:0000a660       ??0?$JPtrArray@PAG@@QAE@J@Z 0040b660 f i sp_module.obj
 0001:0000a6c0       ??0?$JPtrArray@PAD@@QAE@J@Z 0040b6c0 f i sp_module.obj
 0001:0000a720       ?SetNumNoPurge@?$JArray@PAX@@QAEXK_N@Z 0040b720 f i sp_module.obj
 0001:0000a780       ?Realloc@?$JArray@PAX@@QAE_NK@Z 0040b780 f i sp_module.obj
 0001:0000a780       ?Realloc@?$JArray@K@@QAE_NK@Z 0040b780 f i sp_module.obj
 0001:0000a860       ??_ESPModule@@WCGI@AEPAXI@Z 0040b860 f i sp_module.obj
 0001:0000a870       ?Release@SPParamManager@@QAEXXZ 0040b870 f   sp_param.obj
 0001:0000a8a0       ?SetResponseGMEM@SPParamManager@@QAE_NPAXK@Z 0040b8a0 f   sp_param.obj
 0001:0000a910       ?ParseValue@SPParamManager@@AAE_NPAD_N@Z 0040b910 f   sp_param.obj
 0001:0000abe0       ?Find@SPParamManager@@QAEJPBD_N@Z 0040bbe0 f   sp_param.obj
 0001:0000ac60       ?GetValue@SPParamManager@@QAEPAGPBD_N@Z 0040bc60 f   sp_param.obj
 0001:0000aca0       ?GetValueA@SPParamManager@@QAEPADPBDH_N@Z 0040bca0 f   sp_param.obj
 0001:0000ad50       ?VarGet@SPProp@@UAE_NPAVSPGhost@@PAGAAVJWString@@PAVSPVarSystemNode@@@Z 0040bd50 f   sp_prop.obj
 0001:0000b130       ?ReadDescript@SPProp@@UAEHXZ 0040c130 f   sp_prop.obj
 0001:0000b150       ?ParseSingleEntry@SPProp@@UAE_NPADHAAVJTokenStream@@@Z 0040c150 f   sp_prop.obj
 0001:0000b450       ?Serialize@SPProp@@UAEXAAVJWString@@@Z 0040c450 f   sp_prop.obj
 0001:0000b6c0       ?GetThumbnail@SPProp@@UAE_NAAVJString@@@Z 0040c6c0 f   sp_prop.obj
 0001:0000b700       ?GetNowLoading@SPProp@@UAE_NAAVJString@@@Z 0040c700 f   sp_prop.obj
 0001:0000b740       ?GetNowLoadingReal@SPProp@@IAE_NAAVJString@@0@Z 0040c740 f   sp_prop.obj
 0001:0000b740       ?GetThumbnailReal@SPProp@@IAE_NAAVJString@@0@Z 0040c740 f   sp_prop.obj
 0001:0000b750       ?GetUpdateTime@SPProp@@QAEKXZ 0040c750 f   sp_prop.obj
 0001:0000ba00       ?GetUpdateResult@SPProp@@QAEPBGXZ 0040ca00 f   sp_prop.obj
 0001:0000ba10       ?LoadDeferredInfo@SPProp@@UAE_NXZ 0040ca10 f   sp_prop.obj
 0001:0000ba40       ?InvalidateCacheData@SPProp@@UAEXXZ 0040ca40 f   sp_prop.obj
 0001:0000bb60       ??0SPSetCurrentDir@@QAE@PBD@Z 0040cb60 f   sp_setcurrentdir.obj
 0001:0000bb90       ??1SPSetCurrentDir@@QAE@XZ 0040cb90 f   sp_setcurrentdir.obj
 0001:0000bba0       ??0SPShiori@@QAE@XZ        0040cba0 f   sp_shiori.obj
 0001:0000bdc0       ?GetModuleDesc@SPShiori@@UAEPBGXZ 0040cdc0 f i sp_shiori.obj
 0001:0000bdd0       ?GetLogFileName@SPShiori@@UAEPBDXZ 0040cdd0 f i sp_shiori.obj
 0001:0000bde0       ??_ESPShiori@@UAEPAXI@Z    0040cde0 f i sp_shiori.obj
 0001:0000bde0       ??_GSPShiori@@UAEPAXI@Z    0040cde0 f i sp_shiori.obj
 0001:0000be10       ??1SPShiori@@UAE@XZ        0040ce10 f   sp_shiori.obj
 0001:0000bf60       ?MakeShiori30Request@SPShiori@@AAEXAAVJString@@AAVSPShioriEvent@@PBG@Z 0040cf60 f   sp_shiori.obj
 0001:0000c250       ?Load@SPShiori@@QAEHPBD@Z  0040d250 f   sp_shiori.obj
 0001:0000cbb0       ?Unload@SPShiori@@QAEXXZ   0040dbb0 f   sp_shiori.obj
 0001:0000cd70       ?Clear@SPModuleEvent@@QAEXXZ 0040dd70 f i sp_shiori.obj
 0001:0000cd90       ??1SPModuleEvent@@UAE@XZ   0040dd90 f i sp_shiori.obj
 0001:0000cd90       ??1SPShioriEvent@@UAE@XZ   0040dd90 f i sp_shiori.obj
 0001:0000cda0       ??_GSPModuleEvent@@UAEPAXI@Z 0040dda0 f i sp_shiori.obj
 0001:0000cda0       ??_ESPModuleEvent@@UAEPAXI@Z 0040dda0 f i sp_shiori.obj
 0001:0000cdd0       ??_ESPShioriEvent@@UAEPAXI@Z 0040ddd0 f i sp_shiori.obj
 0001:0000cdd0       ??_GSPShioriEvent@@UAEPAXI@Z 0040ddd0 f i sp_shiori.obj
 0001:0000ce00       ?SendEvent@SPShiori@@QAE?AVSPShioriEventResult@@AAVSPShioriEvent@@@Z 0040de00 f   sp_shiori.obj
 0001:0000d2b0       ??0SPModuleEvent@@QAE@ABV0@@Z 0040e2b0 f i sp_shiori.obj
 0001:0000d2f0       ?SendCommunicate@SPShiori@@QAEHXZ 0040e2f0 f   sp_shiori.obj
 0001:0000d300       ?Request@SPShiori@@AAEPAGAAVJString@@@Z 0040e300 f   sp_shiori.obj
 0001:0000d590       ?GetStringShiori@SPShiori@@QAEPAGPAG_N@Z 0040e590 f   sp_shiori.obj
 0001:0000d850       ?GetVersion@SPShiori@@QAEHXZ 0040e850 f   sp_shiori.obj
 0001:0000da70       ?ResetDataCache@SPShiori@@QAEXXZ 0040ea70 f   sp_shiori.obj
 0001:0000da90       ?ResetMenuAvailableTableChar@SPShiori@@AAEXXZ 0040ea90 f   sp_shiori.obj
 0001:0000db00       ?ParseGenericHeaders@SPShiori@@AAEXXZ 0040eb00 f   sp_shiori.obj
 0001:0000db50       ?ClearTeachArray@SPShiori@@QAEXXZ 0040eb50 f   sp_shiori.obj
 0001:0000dbd0       ?SetBaseWareID_Fake@SPShiori@@QAEXPBG@Z 0040ebd0 f   sp_shiori.obj
 0001:0000dbf0       ?GetCurrentDirectoryShiori@SPShiori@@QAEPADXZ 0040ebf0 f   sp_shiori.obj
 0001:0000dc10       ?GetBaseWareID@SPShiori@@AAEPAGXZ 0040ec10 f   sp_shiori.obj
 0001:0000dc40       ?SPShiori_SearchFileFromParentDir@@YA_NAAVJString@@PBD1@Z 0040ec40 f   sp_shiori.obj
 0001:0000de80       ?LoadModuleAndModifySpecificDLL@SPShiori@@AAEPADAAVJString@@0@Z 0040ee80 f   sp_shiori.obj
 0001:0000e9d0       ?HookAPICall@SPShiori@@AAEXXZ 0040f9d0 f   sp_shiori.obj
 0001:0000f510       ??0?$JArray@PAX@@QAE@K@Z   00410510 f i sp_shiori.obj
 0001:0000f5b0       ??0?$JArray@G@@QAE@K@Z     004105b0 f i sp_shiori.obj
 0001:0000f640       ??_ESPShiori@@WCGI@AEPAXI@Z 00410640 f i sp_shiori.obj
 0001:0000f650       ?Release@SPStaticStringArrayW@@QAEXXZ 00410650 f   sp_staticstringarray.obj
 0001:0000f6d0       ?AddW@SPStaticStringArrayW@@QAEJPBGJ@Z 004106d0 f   sp_staticstringarray.obj
 0001:0000f860       ?AddA@SPStaticStringArrayW@@QAEJPBDH@Z 00410860 f   sp_staticstringarray.obj
 0001:0000f910       ?Get@SPStaticStringArrayW@@QAEPAGK@Z 00410910 f   sp_staticstringarray.obj
 0001:0000f940       ?MakeTable@SPStaticStringArrayW@@ABEXXZ 00410940 f   sp_staticstringarray.obj
 0001:0000fa80       ?Release@SPStaticStringArrayA@@QAEXXZ 00410a80 f   sp_staticstringarray.obj
 0001:0000fb00       ?AddA@SPStaticStringArrayA@@QAEJPBDJ@Z 00410b00 f   sp_staticstringarray.obj
 0001:0000fc90       ?Get@SPStaticStringArrayA@@QAEPADK@Z 00410c90 f   sp_staticstringarray.obj
 0001:0000fcc0       ?GetNum@SPStaticStringArrayA@@QBEKXZ 00410cc0 f   sp_staticstringarray.obj
 0001:0000fcd0       ?MakeTable@SPStaticStringArrayA@@ABEXXZ 00410cd0 f   sp_staticstringarray.obj
 0001:0000fe10       ?SetNum@?$JArray@PAX@@QAEXK@Z 00410e10 f i sp_staticstringarray.obj
 0001:0000fe60       ?GetSPSystemInfo@@YAAAVSPSystemInfo@@XZ 00410e60 f   sp_sysinfo.obj
 0001:0000feb0       ??0SPSystemInfo@@QAE@XZ    00410eb0 f   sp_sysinfo.obj
 0001:00010c20       ?GetCPUClock@SPSystemInfo@@QAEKXZ 00411c20 f   sp_sysinfo.obj
 0001:00010d90       ?IsHT@SPSystemInfo@@QAEHXZ 00411d90 f   sp_sysinfo.obj
 0001:00010db0       ?GetMemoryStatus@SPSystemInfo@@QAEXAAUSPMemoryStatus@@@Z 00411db0 f   sp_sysinfo.obj
 0001:00010eb0       ?CreateVersionString@SPSystemInfo@@AAEXAAU_OSVERSIONINFOEXA@@@Z 00411eb0 f   sp_sysinfo.obj
 0001:00011ab0       ?GetSPURLTranslate@@YAAAVSPURLTranslate@@XZ 00412ab0 f   sp_urltranslate.obj
 0001:00011b00       ??0SPURLTranslate@@AAE@XZ  00412b00 f   sp_urltranslate.obj
 0001:00011b40       ??1SPURLTranslate@@QAE@XZ  00412b40 f   sp_urltranslate.obj
 0001:00011c00       ?Translate@SPURLTranslate@@QAE_NAAVJWString@@@Z 00412c00 f   sp_urltranslate.obj
 0001:00011d10       ?Translate@SPURLTranslate@@QAE_NAAVJString@@@Z 00412d10 f   sp_urltranslate.obj
 0001:00011d60       ?GetSPUtils@@YAAAVSPUtils@@XZ 00412d60 f   sp_utils.obj
 0001:00011db0       ??0SPUtils@@QAE@XZ         00412db0 f i sp_utils.obj
 0001:00011dc0       ?GetLocalObjectName@SPUtils@@QAEPBDPBD@Z 00412dc0 f   sp_utils.obj
 0001:00011e10       ?GetFileTimeAsSystemSeconds@SPUtils@@QAE?B_NPBDAAK11@Z 00412e10 f   sp_utils.obj
 0001:00011ea0       ?IsRelativePath@SPUtils@@QAE_NPBD@Z 00412ea0 f   sp_utils.obj
 0001:00011f10       ?MakeAbsolutePath@SPUtils@@QAE_NAAVJString@@PBD_N@Z 00412f10 f   sp_utils.obj
 0001:000123f0       ?SplitTokenW@SPUtils@@QAEKPAGPAPAGKPBG_N@Z 004133f0 f   sp_utils.obj
 0001:000124f0       ?CreateProcessWrapper@SPUtils@@QAEHPBD0K_N1@Z 004134f0 f   sp_utils.obj
 0001:000126f0       ?ConvertSystemSecondsToLocalSystemTime@SPUtils@@QAEXKAAU_SYSTEMTIME@@@Z 004136f0 f   sp_utils.obj
 0001:00012740       ?ConvertFileTimeToSystemSeconds@SPUtils@@QAEKAAU_FILETIME@@@Z 00413740 f   sp_utils.obj
 0001:00012780       ?SystemTimeToCommaSeparatedTime@SPUtils@@QAEPBDABU_SYSTEMTIME@@@Z 00413780 f   sp_utils.obj
 0001:000127e0       ?GUIDToStringA@SPUtils@@QAEPBDAAU_GUID@@@Z 004137e0 f   sp_utils.obj
 0001:00012850       ??1SPFindFile@@QAE@XZ      00413850 f i sp_utils.obj
 0001:000128a0       ?VarSet@SPProp@@UAE_NPAVSPGhost@@PAG1PAVSPVarSystemNode@@@Z 004138a0 f   sp_varsystemnode.obj
 0001:000128a0       ?VarSet@SPVarSystemNode@@UAE_NPAVSPGhost@@PAG1PAV1@@Z 004138a0 f   sp_varsystemnode.obj
 0001:000128a0       ?VarGet@SPVarSystemNode@@UAE_NPAVSPGhost@@PAGAAVJWString@@PAV1@@Z 004138a0 f   sp_varsystemnode.obj
 0001:000128b0       ?Release@SPVersionInfo@@QAEXXZ 004138b0 f   sp_versioninfo.obj
 0001:000128d0       ?Open@SPVersionInfo@@QAE_NPBD@Z 004138d0 f   sp_versioninfo.obj
 0001:00012970       ?FileInfo@SPVersionInfo@@QAEPAUtagVS_FIXEDFILEINFO@@XZ 00413970 f   sp_versioninfo.obj
 0001:000129b0       ?GetEntry@SPVersionInfo@@QAEPADPAD@Z 004139b0 f   sp_versioninfo.obj
 0001:00012ac0       ?CallWndRetProc@@YGJHIJ@Z  00413ac0 f   ssph.obj
 0001:00012b70       _WinMain@16                00413b70 f   ssph.obj
 0001:00012b90       ??0CSSPHApp@@QAE@XZ        00413b90 f   ssph.obj
 0001:00012c60       ??1CSSPHApp@@QAE@XZ        00413c60 f   ssph.obj
 0001:00012c90       ?Main@CSSPHApp@@QAEHPAUHINSTANCE__@@PADH@Z 00413c90 f   ssph.obj
 0001:00012f20       ?UpdateSelf@CSSPHApp@@AAEXXZ 00413f20 f   ssph.obj
 0001:000130b0       ?SetTime@CSSPHApp@@AAEXXZ  004140b0 f   ssph.obj
 0001:00013160       ?ShioriURL@CSSPHApp@@AAEXXZ 00414160 f   ssph.obj
 0001:000131a0       ?GetURL@CSSPHApp@@AAEXXZ   004141a0 f   ssph.obj
 0001:000132e0       ?GetURLMain@CSSPHApp@@AAEHAAV?$JArray@D@@PAD@Z 004142e0 f   ssph.obj
 0001:00013710       ?SSPH_ScanURL@@YAHPADAAVJString@@@Z 00414710 f   ssph_url.obj
 0001:00013e70       _call_zopen64              00414e70 f   ioapi.obj
 0001:00013eb0       _call_zseek64              00414eb0 f   ioapi.obj
 0001:00013f10       _call_ztell64              00414f10 f   ioapi.obj
 0001:00013fc0       _fill_fopen64_filefunc     00414fc0 f   ioapi.obj
 0001:000140c0       ?CanExtractExtension@@YAHPAD@Z 004150c0 f   kei.obj
 0001:00014110       ?JZIPExtract@@YAHPAD00H@Z  00415110 f   kei.obj
 0001:00014230       ?JZIPExtractReal@@YAHPAD00HI@Z 00415230 f   kei.obj
 0001:000146e0       ?Unpack@@YAHPAD00H@Z       004156e0 f   kei.obj
 0001:000147a0       ?ZipUnpack@@YAHPAD00HK@Z   004157a0 f   kei.obj
 0001:000148b0       ?ZipUnpackReal@@YAHPAD00HK@Z 004158b0 f   kei.obj
 0001:000149c0       ?LhaUnpackCallback@@YGHPAX@Z 004159c0 f   kei.obj
 0001:00014a20       ?LhaUnpack@@YAHPAD00H@Z    00415a20 f   kei.obj
 0001:00014b10       ?LhaInit@@YAHXZ            00415b10 f   kei.obj
 0001:00014bb0       ?CabExtractFindNextPathDelim@@YIPBDPBD@Z 00415bb0 f   kei.obj
 0001:00014bd0       ?CabExtractMakePath@@YIHPBD0@Z 00415bd0 f   kei.obj
 0001:00014cd0       ?CabExtractCallback@@YGIPAXIII@Z 00415cd0 f   kei.obj
 0001:00014df0       ?CabInfoCallback@@YGIPAXIII@Z 00415df0 f   kei.obj
 0001:00014e30       ?CabUnpack@@YAHPAD00H@Z    00415e30 f   kei.obj
 0001:00014eb0       ?JZIPIsSelfUnpack@@YAPBDPADPAK@Z 00415eb0 f   kei.obj
 0001:00015100       ?ExeUnpack@@YAHPAD00H@Z    00416100 f   kei.obj
 0001:00015390       ?id@?$ctype@G@std@@$E      00416390 f i kei.obj
 0001:00015fb0       _unzOpen                   00416fb0 f   unzip.obj
 0001:00015fd0       _unzClose                  00416fd0 f   unzip.obj
 0001:00016010       _unzGetGlobalInfo          00417010 f   unzip.obj
 0001:00016590       _unzGetCurrentFileInfo     00417590 f   unzip.obj
 0001:00016640       _unzGoToFirstFile          00417640 f   unzip.obj
 0001:000166b0       _unzGoToNextFile           004176b0 f   unzip.obj
 0001:00016780       _unzOpenCurrentFile3       00417780 f   unzip.obj
 0001:00016c20       _unzOpenCurrentFile        00417c20 f   unzip.obj
 0001:00016c40       _unzReadCurrentFile        00417c40 f   unzip.obj
 0001:00016f50       _unzCloseCurrentFile       00417f50 f   unzip.obj
 0001:00017000       _unzSetOffset64            00418000 f   unzip.obj
 0001:00017070       _unzSetOffset              00418070 f   unzip.obj
 0001:00017090       ??0CUnzipper@@QAE@PBD@Z    00418090 f   Unzipper.obj
 0001:000170d0       ??_ECUnzipper@@UAEPAXI@Z   004180d0 f i Unzipper.obj
 0001:000170d0       ??_GCUnzipper@@UAEPAXI@Z   004180d0 f i Unzipper.obj
 0001:00017100       ??1CUnzipper@@UAE@XZ       00418100 f   Unzipper.obj
 0001:00017130       ?CloseZip@CUnzipper@@QAE_NXZ 00418130 f   Unzipper.obj
 0001:00017160       ?OpenZip@CUnzipper@@QAE_NPBDK@Z 00418160 f   Unzipper.obj
 0001:00017230       ?SetOutputFolder@CUnzipper@@QAE_NPBD@Z 00418230 f   Unzipper.obj
 0001:00017270       ?GetFileCount@CUnzipper@@QAEHXZ 00418270 f   Unzipper.obj
 0001:000172a0       ?GotoFirstFile@CUnzipper@@QAE_NPBD@Z 004182a0 f   Unzipper.obj
 0001:00017370       ?GotoNextFile@CUnzipper@@QAE_NPBD@Z 00418370 f   Unzipper.obj
 0001:00017450       ?GetFileInfo@CUnzipper@@QAE_NAAUUZ_FileInfo@@@Z 00418450 f   Unzipper.obj
 0001:00017750       ?UnzipFile@CUnzipper@@QAE_NPBD_N@Z 00418750 f   Unzipper.obj
 0001:00017930       ?CreateFolder@CUnzipper@@KA_NPBD@Z 00418930 f   Unzipper.obj
 0001:000179c0       ?CreateFilePath@CUnzipper@@KA_NPBD@Z 004189c0 f   Unzipper.obj
 0001:00017a00       ?SetFileModTime@CUnzipper@@KA_NPBDK@Z 00418a00 f   Unzipper.obj
 0001:00017ab0       _Module32Next@8            00418ab0 f   kernel32:KERNEL32.dll
 0001:00017ab6       _Module32First@8           00418ab6 f   kernel32:KERNEL32.dll
 0001:00017abc       _CreateToolhelp32Snapshot@8 00418abc f   kernel32:KERNEL32.dll
 0001:00017ac2       _Process32Next@8           00418ac2 f   kernel32:KERNEL32.dll
 0001:00017ac8       _Process32First@8          00418ac8 f   kernel32:KERNEL32.dll
 0001:00017ace       _VerQueryValueA@16         00418ace f   Version:VERSION.dll
 0001:00017ad4       _GetFileVersionInfoA@16    00418ad4 f   Version:VERSION.dll
 0001:00017ada       _GetFileVersionInfoSizeA@8 00418ada f   Version:VERSION.dll
 0001:00017ae0       _inflateResetKeep          00418ae0 f   zlib:inflate.obj
 0001:00017bb0       _inflateReset              00418bb0 f   zlib:inflate.obj
 0001:00017bf0       _inflateReset2             00418bf0 f   zlib:inflate.obj
 0001:00017c90       _inflateInit2_             00418c90 f   zlib:inflate.obj
 0001:00017d60       _inflate                   00418d60 f   zlib:inflate.obj
 0001:00019670       _inflateEnd                0041a670 f   zlib:inflate.obj
 0001:000196c0       _crc32_z                   0041a6c0 f   zlib:crc32.obj
 0001:000196e0       _crc32                     0041a6e0 f   zlib:crc32.obj
 0001:0001aa70       _zcalloc                   0041ba70 f   zlib:zutil.obj
 0001:0001aa90       _zcfree                    0041ba90 f   zlib:zutil.obj
 0001:0001aab0       _inflate_fast              0041bab0 f   zlib:inffast.obj
 0001:0001af10       _inflate_table             0041bf10 f   zlib:inftrees.obj
 0001:0001b300       _adler32_z                 0041c300 f   zlib:adler32.obj
 0001:0001b580       _adler32                   0041c580 f   zlib:adler32.obj
 0001:0001b610       __tr_stored_block          0041c610 f   zlib:trees.obj
 0001:0001b720       __tr_flush_bits            0041c720 f   zlib:trees.obj
 0001:0001b740       __tr_flush_block           0041c740 f   zlib:trees.obj
 0001:0001ce90       ??3@YAXPAX@Z               0041de90 f   libcpmt:delop.obj
 0001:0001ce9b       ?_JumpToContinuation@@YGXPAXPAUEHRegistrationNode@@@Z 0041de9b f   LIBCMT:trnsctrl.obj
 0001:0001cecf       ?_CallMemberFunction0@@YGXPAX0@Z 0041decf f   LIBCMT:trnsctrl.obj
 0001:0001cecf       ?_CallMemberFunction1@@YGXPAX00@Z 0041decf f   LIBCMT:trnsctrl.obj
 0001:0001ced6       ?_CallMemberFunction2@@YGXPAX00H@Z 0041ded6 f   LIBCMT:trnsctrl.obj
 0001:0001cedd       ?_UnwindNestedFrames@@YGXPAUEHRegistrationNode@@PAUEHExceptionRecord@@@Z 0041dedd f   LIBCMT:trnsctrl.obj
 0001:0001cf2c       ___CxxFrameHandler         0041df2c f   LIBCMT:trnsctrl.obj
 0001:0001cf62       ?_CallCatchBlock2@@YAPAXPAUEHRegistrationNode@@PBU_s_FuncInfo@@PAXHK@Z 0041df62 f   LIBCMT:trnsctrl.obj
 0001:0001cfdb       ?_CallSETranslator@@YAHPAUEHExceptionRecord@@PAUEHRegistrationNode@@PAX2PBU_s_FuncInfo@@H1@Z 0041dfdb f   LIBCMT:trnsctrl.obj
 0001:0001d106       ?_GetRangeOfTrysToCheck@@YAPBU_s_TryBlockMapEntry@@PBU_s_FuncInfo@@HHPAI1@Z 0041e106 f   LIBCMT:trnsctrl.obj
 0001:0001d184       __global_unwind2           0041e184 f   LIBCMT:exsup.obj
 0001:0001d1c6       __local_unwind2            0041e1c6 f   LIBCMT:exsup.obj
 0001:0001d21e       __NLG_Return2              0041e21e f   LIBCMT:exsup.obj
 0001:0001d22e       __abnormal_termination     0041e22e f   LIBCMT:exsup.obj
 0001:0001d251       __NLG_Notify1              0041e251 f   LIBCMT:exsup.obj
 0001:0001d25a       __NLG_Notify               0041e25a f   LIBCMT:exsup.obj
 0001:0001d26d       __NLG_Dispatch             0041e26d f   LIBCMT:exsup.obj
 0001:0001d272       __onexit                   0041e272 f   LIBCMT:onexit.obj
 0001:0001d2f0       _atexit                    0041e2f0 f   LIBCMT:onexit.obj
 0001:0001d302       ___onexitinit              0041e302 f   LIBCMT:onexit.obj
 0001:0001d331       _malloc                    0041e331 f   LIBCMT:malloc.obj
 0001:0001d343       __nh_malloc                0041e343 f   LIBCMT:malloc.obj
 0001:0001d36f       __heap_alloc               0041e36f f   LIBCMT:malloc.obj
 0001:0001d46b       _free                      0041e46b f   LIBCMT:free.obj
 0001:0001d554       __fpmath                   0041e554 f   LIBCMT:fpinit.obj
 0001:0001d56b       __fpclear                  0041e56b f   LIBCMT:fpinit.obj
 0001:0001d56c       __cfltcvt_init             0041e56c f   LIBCMT:fpinit.obj
 0001:0001d5a4       ??2@YAPAXI@Z               0041e5a4 f   LIBCMT:new.obj
 0001:0001d5b4       __ftol                     0041e5b4 f   LIBCMT:ftol.obj
 0001:0001d5db       __mbsrchr                  0041e5db f   LIBCMT:mbsrchr.obj
 0001:0001d650       _strncmp                   0041e650 f   LIBCMT:strncmp.obj
 0001:0001d690       _memmove                   0041e690 f   LIBCMT:memmove.obj
 0001:0001d9c5       _realloc                   0041e9c5 f   LIBCMT:realloc.obj
 0001:0001dd00       _strstr                    0041ed00 f   LIBCMT:strstr.obj
 0001:0001dd80       _wcslen                    0041ed80 f   LIBCMT:wcslen.obj
 0001:0001dd9d       __setmbcp                  0041ed9d f   LIBCMT:mbctype.obj
 0001:0001e175       ___initmbctable            0041f175 f   LIBCMT:mbctype.obj
 0001:0001e191       _wcsncmp                   0041f191 f   LIBCMT:wcsncmp.obj
 0001:0001e1c9       _wcsstr                    0041f1c9 f   LIBCMT:wcsstr.obj
 0001:0001e20a       _isspace                   0041f20a f   LIBCMT:_ctype.obj
 0001:0001e232       _isalnum                   0041f232 f   LIBCMT:_ctype.obj
 0001:0001e260       _strtol                    0041f260 f   LIBCMT:strtol.obj
 0001:0001e47c       _strtoul                   0041f47c f   LIBCMT:strtol.obj
 0001:0001e493       _wcstol                    0041f493 f   LIBCMT:wcstol.obj
 0001:0001e651       _wcstoul                   0041f651 f   LIBCMT:wcstol.obj
 0001:0001e668       _sprintf                   0041f668 f   LIBCMT:sprintf.obj
 0001:0001e6ba       _swprintf                  0041f6ba f   LIBCMT:swprintf.obj
 0001:0001e729       _wcschr                    0041f729 f   LIBCMT:wcschr.obj
 0001:0001e760       __chkstk                   0041f760 f   LIBCMT:chkstk.obj
 0001:0001e760       __alloca_probe             0041f760 f   LIBCMT:chkstk.obj
 0001:0001e78f       _wcscmp                    0041f78f f   LIBCMT:wcscmp.obj
 0001:0001e7c4       _signal                    0041f7c4 f   LIBCMT:winsig.obj
 0001:0001e9a8       _raise                     0041f9a8 f   LIBCMT:winsig.obj
 0001:0001eb67       ?set_terminate@@YAP6AXXZP6AXXZ@Z 0041fb67 f   LIBCMT:user.obj
 0001:0001eb80       ?set_unexpected@@YAP6AXXZP6AXXZ@Z 0041fb80 f   LIBCMT:user.obj
 0001:0001eb99       _fclose                    0041fb99 f   LIBCMT:fclose.obj
 0001:0001ebca       __fclose_lk                0041fbca f   LIBCMT:fclose.obj
 0001:0001ec16       _fflush                    0041fc16 f   LIBCMT:fflush.obj
 0001:0001ec45       __fflush_lk                0041fc45 f   LIBCMT:fflush.obj
 0001:0001ec73       __flush                    0041fc73 f   LIBCMT:fflush.obj
 0001:0001eccf       __flushall                 0041fccf f   LIBCMT:fflush.obj
 0001:0001ed7c       __fsopen                   0041fd7c f   LIBCMT:fopen.obj
 0001:0001edad       _fopen                     0041fdad f   LIBCMT:fopen.obj
 0001:0001edc0       _strrchr                   0041fdc0 f   LIBCMT:strrchr.obj
 0001:0001edf0       __except_handler3          0041fdf0 f   LIBCMT:exsup3.obj
 0001:0001eead       __seh_longjmp_unwind@4     0041fead f   LIBCMT:exsup3.obj
 0001:0001eec8       _fprintf                   0041fec8 f   LIBCMT:fprintf.obj
 0001:0001ef04       _fputs                     0041ff04 f   LIBCMT:fputs.obj
 0001:0001ef60       __aullshr                  0041ff60 f   LIBCMT:ullshr.obj
 0001:0001ef80       __allmul                   0041ff80 f   LIBCMT:llmul.obj
 0001:0001efb4       _qsort                     0041ffb4 f   LIBCMT:qsort.obj
 0001:0001f182       ??_M@YGXPAXIHP6EX0@Z@Z     00420182 f   LIBCMT:ehvecdtr.obj
 0001:0001f202       ?__ArrayUnwind@@YGXPAXIHP6EX0@Z@Z 00420202 f   LIBCMT:ehvecdtr.obj
 0001:0001f276       ??_L@YGXPAXIHP6EX0@Z1@Z    00420276 f   LIBCMT:ehvecctr.obj
 0001:0001f310       _strchr                    00420310 f   LIBCMT:strchr.obj
 0001:0001f316       ___from_strstr_to_strchr   00420316 f   LIBCMT:strchr.obj
 0001:0001f3cc       _longjmp                   004203cc f   LIBCMT:longjmp.obj
 0001:0001f448       __setjmp3                  00420448 f   LIBCMT:setjmp3.obj
 0001:0001f4c3       _atof                      004204c3 f   LIBCMT:atof.obj
 0001:0001f51a       _calloc                    0042051a f   LIBCMT:calloc.obj
 0001:0001f657       __mbschr                   00420657 f   LIBCMT:mbschr.obj
 0001:0001f6ee       _strtok                    004206ee f   LIBCMT:strtok.obj
 0001:0001f7a0       __aulldiv                  004207a0 f   LIBCMT:ulldiv.obj
 0001:0001f810       __alldiv                   00420810 f   LIBCMT:lldiv.obj
 0001:0001f8c0       _strpbrk                   004208c0 f   LIBCMT:strpbrk.obj
 0001:0001f8fa       _wcspbrk                   004208fa f   LIBCMT:wcspbrk.obj
 0001:0001f938       _iswspace                  00420938 f   LIBCMT:_wctype.obj
 0001:0001f950       _strncat                   00420950 f   LIBCMT:strncat.obj
 0001:0001fa73       _fread                     00420a73 f   LIBCMT:fread.obj
 0001:0001faa2       __fread_lk                 00420aa2 f   LIBCMT:fread.obj
 0001:0001fb8a       _fwrite                    00420b8a f   LIBCMT:fwrite.obj
 0001:0001fbb9       __fwrite_lk                00420bb9 f   LIBCMT:fwrite.obj
 0001:0001fcc3       _ftell                     00420cc3 f   LIBCMT:ftell.obj
 0001:0001fce5       __ftell_lk                 00420ce5 f   LIBCMT:ftell.obj
 0001:0001fe46       _fseek                     00420e46 f   LIBCMT:fseek.obj
 0001:0001fe72       __fseek_lk                 00420e72 f   LIBCMT:fseek.obj
 0001:0001ff00       _strncpy                   00420f00 f   LIBCMT:strncpy.obj
 0001:00020000       __allshl                   00421000 f   LIBCMT:llshl.obj
 0001:0002001f       __makepath                 0042101f f   LIBCMT:makepath.obj
 0001:000200b0       __splitpath                004210b0 f   LIBCMT:splitpat.obj
 0001:000201f7       __strdup                   004211f7 f   LIBCMT:strdup.obj
 0001:00020230       __strnicmp                 00421230 f   LIBCMT:strnicmp.obj
 0001:00020331       _WinMainCRTStartup         00421331 f   LIBCMT:wincrt0.obj
 0001:00020439       __amsg_exit                00421439 f   LIBCMT:wincrt0.obj
 0001:00020490       __allshr                   00421490 f   LIBCMT:llshr.obj
 0001:000204c0       __allrem                   004214c0 f   LIBCMT:llrem.obj
 0001:00020572       ___InternalCxxFrameHandler 00421572 f   LIBCMT:frame.obj
 0001:000208c7       ___FrameUnwindToState      004218c7 f   LIBCMT:frame.obj
 0001:00020ce9       ?_DestructExceptionObject@@YAXPAUEHExceptionRecord@@E@Z 00421ce9 f   LIBCMT:frame.obj
 0001:00020d80       __CallSettingFrame@12      00421d80 f   LIBCMT:lowhelpr.obj
 0001:00020da7       __NLG_Return               00421da7 f   LIBCMT:lowhelpr.obj
 0001:00020dcc       __mtinit                   00421dcc f   LIBCMT:tidtable.obj
 0001:00020e20       __initptd                  00421e20 f   LIBCMT:tidtable.obj
 0001:00020e33       __getptd                   00421e33 f   LIBCMT:tidtable.obj
 0001:00020e9a       ?terminate@@YAXXZ          00421e9a f   LIBCMT:hooks.obj
 0001:00020efb       ?_inconsistency@@YAXXZ     00421efb f   LIBCMT:hooks.obj
 0001:00020f51       __cinit                    00421f51 f   LIBCMT:crt0dat.obj
 0001:00020f7e       _exit                      00421f7e f   LIBCMT:crt0dat.obj
 0001:00020f8f       __exit                     00421f8f f   LIBCMT:crt0dat.obj
 0001:00021045       __lockexit                 00422045 f   LIBCMT:crt0dat.obj
 0001:0002104e       __unlockexit               0042204e f   LIBCMT:crt0dat.obj
 0001:00021071       __msize                    00422071 f   LIBCMT:msize.obj
 0001:0002115f       __callnewh                 0042215f f   LIBCMT:handler.obj
 0001:0002117a       __GetLinkerVersion         0042217a f   LIBCMT:heapinit.obj
 0001:000211a7       ___heap_select             004221a7 f   LIBCMT:heapinit.obj
 0001:000212ef       __heap_init                004222ef f   LIBCMT:heapinit.obj
 0001:0002134c       ___sbh_heap_init           0042234c f   LIBCMT:sbheap.obj
 0001:00021394       ___sbh_find_block          00422394 f   LIBCMT:sbheap.obj
 0001:000213bf       ___sbh_free_block          004223bf f   LIBCMT:sbheap.obj
 0001:000216e8       ___sbh_alloc_block         004226e8 f   LIBCMT:sbheap.obj
 0001:000219f1       ___sbh_alloc_new_region    004229f1 f   LIBCMT:sbheap.obj
 0001:00021aa2       ___sbh_alloc_new_group     00422aa2 f   LIBCMT:sbheap.obj
 0001:00021b9d       ___sbh_resize_block        00422b9d f   LIBCMT:sbheap.obj
 0001:00021e93       ___old_sbh_new_region      00422e93 f   LIBCMT:sbheap.obj
 0001:00021fd7       ___old_sbh_release_region  00422fd7 f   LIBCMT:sbheap.obj
 0001:0002202d       ___old_sbh_decommit_pages  0042302d f   LIBCMT:sbheap.obj
 0001:000220ef       ___old_sbh_find_block      004230ef f   LIBCMT:sbheap.obj
 0001:00022146       ___old_sbh_free_block      00423146 f   LIBCMT:sbheap.obj
 0001:0002218b       ___old_sbh_alloc_block     0042318b f   LIBCMT:sbheap.obj
 0001:00022393       ___old_sbh_alloc_block_from_page 00423393 f   LIBCMT:sbheap.obj
 0001:000224b7       ___old_sbh_resize_block    004234b7 f   LIBCMT:sbheap.obj
 0001:00022560       __mtinitlocks              00423560 f   LIBCMT:mlock.obj
 0001:00022589       __lock                     00423589 f   LIBCMT:mlock.obj
 0001:000225ea       __unlock                   004235ea f   LIBCMT:mlock.obj
 0001:000225ff       __setdefaultprecision      004235ff f   LIBCMT:fp8.obj
 0001:00022611       __ms_p5_test_fdiv          00423611 f   LIBCMT:testfdiv.obj
 0001:0002264f       __ms_p5_mp_test_fdiv       0042364f f   LIBCMT:testfdiv.obj
 0001:00022678       __forcdecpt                00423678 f   LIBCMT:cvt.obj
 0001:000226d2       __cropzeros                004236d2 f   LIBCMT:cvt.obj
 0001:00022720       __positive                 00423720 f   LIBCMT:cvt.obj
 0001:00022738       __fassign                  00423738 f   LIBCMT:cvt.obj
 0001:00022776       __cftoe                    00423776 f   LIBCMT:cvt.obj
 0001:00022899       __cftof                    00423899 f   LIBCMT:cvt.obj
 0001:00022995       __cftog                    00423995 f   LIBCMT:cvt.obj
 0001:00022a28       __cfltcvt                  00423a28 f   LIBCMT:cvt.obj
 0001:00022aa0       _memcpy                    00423aa0 f   LIBCMT:memcpy.obj
 0001:00022de0       _strcmp                    00423de0 f   LIBCMT:strcmp.obj
 0001:00022e64       ___crtLCMapStringA         00423e64 f   LIBCMT:a_map.obj
 0001:000230b3       __dosmaperr                004240b3 f   LIBCMT:dosmap.obj
 0001:00023126       __errno                    00424126 f   LIBCMT:dosmap.obj
 0001:0002312f       ___doserrno                0042412f f   LIBCMT:dosmap.obj
 0001:00023138       __XcptFilter               00424138 f   LIBCMT:winxfltr.obj
 0001:000232b0       ___crtGetStringTypeA       004242b0 f   LIBCMT:a_str.obj
 0001:00023400       _strcspn                   00424400 f   LIBCMT:strcspn.obj
 0001:00023440       _strlen                    00424440 f   LIBCMT:strlen.obj
 0001:000234c0       _strcpy                    004244c0 f   LIBCMT:strcat.obj
 0001:000234d0       _strcat                    004244d0 f   LIBCMT:strcat.obj
 0001:000235b0       _memset                    004245b0 f   LIBCMT:memset.obj
 0001:00023608       __isctype                  00424608 f   LIBCMT:isctype.obj
 0001:0002367d       _toupper                   0042467d f   LIBCMT:toupper.obj
 0001:000236ec       __toupper_lk               004246ec f   LIBCMT:toupper.obj
 0001:000237b8       _towupper                  004247b8 f   LIBCMT:towupper.obj
 0001:0002382c       __towupper_lk              0042482c f   LIBCMT:towupper.obj
 0001:000238a3       _iswctype                  004248a3 f   LIBCMT:iswctype.obj
 0001:000238f5       __flsbuf                   004248f5 f   LIBCMT:_flsbuf.obj
 0001:00023a0d       __output                   00424a0d f   LIBCMT:output.obj
 0001:00024264       __woutput                  00425264 f   LIBCMT:woutput.obj
 0001:00024a93       ___initstdio               00425a93 f   LIBCMT:_file.obj
 0001:00024b3b       ___endstdio                00425b3b f   LIBCMT:_file.obj
 0001:00024b4f       __lock_file                00425b4f f   LIBCMT:_file.obj
 0001:00024b7e       __lock_file2               00425b7e f   LIBCMT:_file.obj
 0001:00024ba1       __unlock_file              00425ba1 f   LIBCMT:_file.obj
 0001:00024bd0       __unlock_file2             00425bd0 f   LIBCMT:_file.obj
 0001:00024bf3       __close                    00425bf3 f   LIBCMT:close.obj
 0001:00024c50       __close_lk                 00425c50 f   LIBCMT:close.obj
 0001:00024cd3       __freebuf                  00425cd3 f   LIBCMT:_freebuf.obj
 0001:00024cfe       __commit                   00425cfe f   LIBCMT:commit.obj
 0001:00024d91       __write                    00425d91 f   LIBCMT:write.obj
 0001:00024df6       __write_lk                 00425df6 f   LIBCMT:write.obj
 0001:00024f81       __openfile                 00425f81 f   LIBCMT:_open.obj
 0001:000250f1       __getstream                004260f1 f   LIBCMT:stream.obj
 0001:000251b9       __stbuf                    004261b9 f   LIBCMT:_sftbuf.obj
 0001:00025246       __ftbuf                    00426246 f   LIBCMT:_sftbuf.obj
 0001:00025270       __rt_probe_read4@4         00426270 f   LIBCMT:sehsupp.obj
 0001:000252d5       __fltin2                   004262d5 f   LIBCMT:cfin.obj
 0001:00025354       __filbuf                   00426354 f   LIBCMT:_filbuf.obj
 0001:00025430       __read                     00426430 f   LIBCMT:read.obj
 0001:00025495       __read_lk                  00426495 f   LIBCMT:read.obj
 0001:0002566e       __ioinit                   0042666e f   LIBCMT:ioinit.obj
 0001:0002582a       __lseek                    0042682a f   LIBCMT:lseek.obj
 0001:0002588f       __lseek_lk                 0042688f f   LIBCMT:lseek.obj
 0001:00025902       __mbsdec                   00426902 f   LIBCMT:mbsdec.obj
 0001:0002596f       __mbsnbcpy                 0042696f f   LIBCMT:mbsnbcpy.obj
 0001:00025a09       _tolower                   00426a09 f   LIBCMT:tolower.obj
 0001:00025a78       __tolower_lk               00426a78 f   LIBCMT:tolower.obj
 0001:00025b43       __wincmdln                 00426b43 f   LIBCMT:wincmdln.obj
 0001:00025b9b       __setenvp                  00426b9b f   LIBCMT:stdenvp.obj
 0001:00025c54       __setargv                  00426c54 f   LIBCMT:stdargv.obj
 0001:00025ea1       ___crtGetEnvironmentStringsA 00426ea1 f   LIBCMT:a_env.obj
 0001:00025fd3       __FF_MSGBANNER             00426fd3 f   LIBCMT:crt0msg.obj
 0001:0002600c       __NMSG_WRITE               0042700c f   LIBCMT:crt0msg.obj
 0001:0002615f       ?__CxxUnhandledExceptionFilter@@YGJPAU_EXCEPTION_POINTERS@@@Z 0042715f f   LIBCMT:unhandld.obj
 0001:000261a5       ?__CxxSetUnhandledExceptionFilter@@YAXXZ 004271a5 f   LIBCMT:unhandld.obj
 0001:000261b6       ?__CxxRestoreUnhandledExceptionFilter@@YAXXZ 004271b6 f   LIBCMT:unhandld.obj
 0001:000261c3       ?_ValidateRead@@YAHPBXI@Z  004271c3 f   LIBCMT:validate.obj
 0001:000261df       ?_ValidateWrite@@YAHPAXI@Z 004271df f   LIBCMT:validate.obj
 0001:000261fb       ?_ValidateExecute@@YAHP6GHXZ@Z 004271fb f   LIBCMT:validate.obj
 0001:00026213       _abort                     00427213 f   LIBCMT:abort.obj
 0001:0002622a       __control87                0042722a f   LIBCMT:ieee87.obj
 0001:0002625f       __controlfp                0042725f f   LIBCMT:ieee87.obj
 0001:00026390       __ZeroTail                 00427390 f   LIBCMT:intrncvt.obj
 0001:000263d9       __IncMan                   004273d9 f   LIBCMT:intrncvt.obj
 0001:0002642f       __RoundMan                 0042742f f   LIBCMT:intrncvt.obj
 0001:000264bb       __CopyMan                  004274bb f   LIBCMT:intrncvt.obj
 0001:000264d6       __FillZeroMan              004274d6 f   LIBCMT:intrncvt.obj
 0001:000264e2       __IsZeroMan                004274e2 f   LIBCMT:intrncvt.obj
 0001:000264fd       __ShrMan                   004274fd f   LIBCMT:intrncvt.obj
 0001:0002658a       __ld12cvt                  0042758a f   LIBCMT:intrncvt.obj
 0001:000266f6       __ld12tod                  004276f6 f   LIBCMT:intrncvt.obj
 0001:0002670c       __ld12tof                  0042770c f   LIBCMT:intrncvt.obj
 0001:00026722       __atodbl                   00427722 f   LIBCMT:intrncvt.obj
 0001:0002674f       __atoflt                   0042774f f   LIBCMT:intrncvt.obj
 0001:0002677c       __fptostr                  0042777c f   LIBCMT:_fptostr.obj
 0001:000267f3       __fltout2                  004277f3 f   LIBCMT:cfout.obj
 0001:0002684f       ___dtold                   0042784f f   LIBCMT:cfout.obj
 0001:00026905       __fptrap                   00427905 f   LIBCMT:crt0fp.obj
 0001:0002690e       ___crtGetStringTypeW       0042790e f   LIBCMT:w_str.obj
 0001:00026ae0       __strcmpi                  00427ae0 f   LIBCMT:stricmp.obj
 0001:00026ae0       __stricmp                  00427ae0 f   LIBCMT:stricmp.obj
 0001:00026bb0       ___crtLCMapStringW         00427bb0 f   LIBCMT:w_map.obj
 0001:00026de9       __getbuf                   00427de9 f   LIBCMT:_getbuf.obj
 0001:00026e2d       __isatty                   00427e2d f   LIBCMT:isatty.obj
 0001:00026e56       _wctomb                    00427e56 f   LIBCMT:wctomb.obj
 0001:00026eaf       __wctomb_lk                00427eaf f   LIBCMT:wctomb.obj
 0001:00026f20       __aullrem                  00427f20 f   LIBCMT:ullrem.obj
 0001:00026f95       _mbtowc                    00427f95 f   LIBCMT:mbtowc.obj
 0001:00026ff2       __mbtowc_lk                00427ff2 f   LIBCMT:mbtowc.obj
 0001:000270bb       __putwc_lk                 004280bb f   LIBCMT:fputwc.obj
 0001:000271b4       __fcloseall                004281b4 f   LIBCMT:closeall.obj
 0001:00027235       __alloc_osfhnd             00428235 f   LIBCMT:osfinfo.obj
 0001:00027358       __set_osfhnd               00428358 f   LIBCMT:osfinfo.obj
 0001:000273d4       __free_osfhnd              004283d4 f   LIBCMT:osfinfo.obj
 0001:00027453       __get_osfhandle            00428453 f   LIBCMT:osfinfo.obj
 0001:00027495       __lock_fhandle             00428495 f   LIBCMT:osfinfo.obj
 0001:000274f4       __unlock_fhandle           004284f4 f   LIBCMT:osfinfo.obj
 0001:00027516       __sopen                    00428516 f   LIBCMT:open.obj
 0001:000277e5       ___strgtold12              004287e5 f   LIBCMT:strgtold.obj
 0001:00027cb6       __ismbblead                00428cb6 f   LIBCMT:ismbbyte.obj
 0001:00027cf8       ___crtMessageBoxA          00428cf8 f   LIBCMT:crtmbox.obj
 0001:00027d81       ___addl                    00428d81 f   LIBCMT:mantold.obj
 0001:00027da2       ___add_12                  00428da2 f   LIBCMT:mantold.obj
 0001:00027e00       ___shl_12                  00428e00 f   LIBCMT:mantold.obj
 0001:00027e2e       ___shr_12                  00428e2e f   LIBCMT:mantold.obj
 0001:00027e5b       ___mtold12                 00428e5b f   LIBCMT:mantold.obj
 0001:00027f22       _$I10_OUTPUT               00428f22 f   LIBCMT:x10fout.obj
 0001:000281b5       __flswbuf                  004291b5 f   LIBCMT:_flswbuf.obj
 0001:000282dc       __chsize_lk                004292dc f   LIBCMT:chsize.obj
 0001:00028401       ___ld12mul                 00429401 f   LIBCMT:tenpow.obj
 0001:00028621       ___multtenpow12            00429621 f   LIBCMT:tenpow.obj
 0001:0002869d       __setmode_lk               0042969d f   LIBCMT:setmode.obj
 0001:000286fe       _RtlUnwind@16              004296fe f   kernel32:KERNEL32.dll
 0002:00000000       __imp__RegOpenKeyExA@20    0042b000     advapi32:ADVAPI32.dll
 0002:00000004       __imp__RegCloseKey@4       0042b004     advapi32:ADVAPI32.dll
 0002:00000008       __imp__RegQueryValueExA@24 0042b008     advapi32:ADVAPI32.dll
 0002:0000000c       \177ADVAPI32_NULL_THUNK_DATA 0042b00c     advapi32:ADVAPI32.dll
 0002:00000010       __imp__GetCurrentThread@0  0042b010     kernel32:KERNEL32.dll
 0002:00000014       __imp__SetEvent@4          0042b014     kernel32:KERNEL32.dll
 0002:00000018       __imp__GetOEMCP@0          0042b018     kernel32:KERNEL32.dll
 0002:0000001c       __imp__GetACP@0            0042b01c     kernel32:KERNEL32.dll
 0002:00000020       __imp__AreFileApisANSI@0   0042b020     kernel32:KERNEL32.dll
 0002:00000024       __imp__MultiByteToWideChar@24 0042b024     kernel32:KERNEL32.dll
 0002:00000028       __imp__GetSystemDirectoryA@8 0042b028     kernel32:KERNEL32.dll
 0002:0000002c       __imp__VirtualProtect@16   0042b02c     kernel32:KERNEL32.dll
 0002:00000030       __imp__VirtualAlloc@16     0042b030     kernel32:KERNEL32.dll
 0002:00000034       __imp__GetVersionExA@4     0042b034     kernel32:KERNEL32.dll
 0002:00000038       __imp__GetSystemInfo@4     0042b038     kernel32:KERNEL32.dll
 0002:0000003c       __imp__VirtualQuery@12     0042b03c     kernel32:KERNEL32.dll
 0002:00000040       __imp__GetCurrentProcess@0 0042b040     kernel32:KERNEL32.dll
 0002:00000044       __imp__ExitProcess@4       0042b044     kernel32:KERNEL32.dll
 0002:00000048       __imp__GetModuleFileNameA@12 0042b048     kernel32:KERNEL32.dll
 0002:0000004c       __imp__IsBadReadPtr@8      0042b04c     kernel32:KERNEL32.dll
 0002:00000050       __imp__FreeEnvironmentStringsA@4 0042b050     kernel32:KERNEL32.dll
 0002:00000054       __imp__GetEnvironmentStrings@0 0042b054     kernel32:KERNEL32.dll
 0002:00000058       __imp__GetDriveTypeA@4     0042b058     kernel32:KERNEL32.dll
 0002:0000005c       __imp__GetVolumeInformationA@32 0042b05c     kernel32:KERNEL32.dll
 0002:00000060       __imp__GetLogicalDrives@0  0042b060     kernel32:KERNEL32.dll
 0002:00000064       __imp__GetLocalTime@4      0042b064     kernel32:KERNEL32.dll
 0002:00000068       __imp__GetDiskFreeSpaceA@20 0042b068     kernel32:KERNEL32.dll
 0002:0000006c       __imp__Module32Next@8      0042b06c     kernel32:KERNEL32.dll
 0002:00000070       __imp__Module32First@8     0042b070     kernel32:KERNEL32.dll
 0002:00000074       __imp__CreateToolhelp32Snapshot@8 0042b074     kernel32:KERNEL32.dll
 0002:00000078       __imp__GetCurrentProcessId@0 0042b078     kernel32:KERNEL32.dll
 0002:0000007c       __imp__GetLastError@0      0042b07c     kernel32:KERNEL32.dll
 0002:00000080       __imp__Process32Next@8     0042b080     kernel32:KERNEL32.dll
 0002:00000084       __imp__Process32First@8    0042b084     kernel32:KERNEL32.dll
 0002:00000088       __imp__ResetEvent@4        0042b088     kernel32:KERNEL32.dll
 0002:0000008c       __imp__FindClose@4         0042b08c     kernel32:KERNEL32.dll
 0002:00000090       __imp__FindFirstFileA@8    0042b090     kernel32:KERNEL32.dll
 0002:00000094       __imp__FindNextFileA@8     0042b094     kernel32:KERNEL32.dll
 0002:00000098       __imp__GetFileAttributesA@4 0042b098     kernel32:KERNEL32.dll
 0002:0000009c       __imp__GlobalFree@4        0042b09c     kernel32:KERNEL32.dll
 0002:000000a0       __imp__CreateProcessA@40   0042b0a0     kernel32:KERNEL32.dll
 0002:000000a4       __imp__DuplicateHandle@28  0042b0a4     kernel32:KERNEL32.dll
 0002:000000a8       __imp__CreatePipe@16       0042b0a8     kernel32:KERNEL32.dll
 0002:000000ac       __imp__LoadLibraryExA@12   0042b0ac     kernel32:KERNEL32.dll
 0002:000000b0       __imp__TerminateProcess@8  0042b0b0     kernel32:KERNEL32.dll
 0002:000000b4       __imp__InterlockedDecrement@4 0042b0b4     kernel32:KERNEL32.dll
 0002:000000b8       __imp__InterlockedIncrement@4 0042b0b8     kernel32:KERNEL32.dll
 0002:000000bc       __imp__GlobalAlloc@8       0042b0bc     kernel32:KERNEL32.dll
 0002:000000c0       __imp__GlobalSize@4        0042b0c0     kernel32:KERNEL32.dll
 0002:000000c4       __imp__SetFileTime@16      0042b0c4     kernel32:KERNEL32.dll
 0002:000000c8       __imp__GetFileTime@16      0042b0c8     kernel32:KERNEL32.dll
 0002:000000cc       __imp__CreateDirectoryA@8  0042b0cc     kernel32:KERNEL32.dll
 0002:000000d0       __imp__SetCurrentDirectoryA@4 0042b0d0     kernel32:KERNEL32.dll
 0002:000000d4       __imp__GetCurrentDirectoryA@8 0042b0d4     kernel32:KERNEL32.dll
 0002:000000d8       __imp__DeleteFileA@4       0042b0d8     kernel32:KERNEL32.dll
 0002:000000dc       __imp__LockResource@4      0042b0dc     kernel32:KERNEL32.dll
 0002:000000e0       __imp__SizeofResource@8    0042b0e0     kernel32:KERNEL32.dll
 0002:000000e4       __imp__LoadResource@8      0042b0e4     kernel32:KERNEL32.dll
 0002:000000e8       __imp__FindResourceA@12    0042b0e8     kernel32:KERNEL32.dll
 0002:000000ec       __imp__GetWindowsDirectoryA@8 0042b0ec     kernel32:KERNEL32.dll
 0002:000000f0       __imp__LoadLibraryW@4      0042b0f0     kernel32:KERNEL32.dll
 0002:000000f4       __imp__GetModuleHandleW@4  0042b0f4     kernel32:KERNEL32.dll
 0002:000000f8       __imp__LoadLibraryExW@12   0042b0f8     kernel32:KERNEL32.dll
 0002:000000fc       __imp__VirtualProtectEx@20 0042b0fc     kernel32:KERNEL32.dll
 0002:00000100       __imp__QueryPerformanceCounter@4 0042b100     kernel32:KERNEL32.dll
 0002:00000104       __imp__SetThreadPriority@8 0042b104     kernel32:KERNEL32.dll
 0002:00000108       __imp__GetThreadPriority@4 0042b108     kernel32:KERNEL32.dll
 0002:0000010c       __imp__GlobalMemoryStatus@4 0042b10c     kernel32:KERNEL32.dll
 0002:00000110       __imp__CopyFileA@12        0042b110     kernel32:KERNEL32.dll
 0002:00000114       __imp__GetEnvironmentVariableA@12 0042b114     kernel32:KERNEL32.dll
 0002:00000118       __imp__WaitForMultipleObjects@16 0042b118     kernel32:KERNEL32.dll
 0002:0000011c       __imp__GetPriorityClass@4  0042b11c     kernel32:KERNEL32.dll
 0002:00000120       __imp__GetCurrentThreadId@0 0042b120     kernel32:KERNEL32.dll
 0002:00000124       __imp__FileTimeToSystemTime@8 0042b124     kernel32:KERNEL32.dll
 0002:00000128       __imp__FileTimeToLocalFileTime@8 0042b128     kernel32:KERNEL32.dll
 0002:0000012c       __imp__lstrcpyA@8          0042b12c     kernel32:KERNEL32.dll
 0002:00000130       __imp__SetUnhandledExceptionFilter@4 0042b130     kernel32:KERNEL32.dll
 0002:00000134       __imp__SetErrorMode@4      0042b134     kernel32:KERNEL32.dll
 0002:00000138       __imp__OpenProcess@12      0042b138     kernel32:KERNEL32.dll
 0002:0000013c       __imp__SetSystemTime@4     0042b13c     kernel32:KERNEL32.dll
 0002:00000140       __imp__OpenFileMappingA@12 0042b140     kernel32:KERNEL32.dll
 0002:00000144       __imp__GetTempPathA@8      0042b144     kernel32:KERNEL32.dll
 0002:00000148       __imp__GetTempFileNameA@16 0042b148     kernel32:KERNEL32.dll
 0002:0000014c       __imp__GetFullPathNameA@16 0042b14c     kernel32:KERNEL32.dll
 0002:00000150       __imp__lstrlenA@4          0042b150     kernel32:KERNEL32.dll
 0002:00000154       __imp__lstrcmpiA@8         0042b154     kernel32:KERNEL32.dll
 0002:00000158       __imp__LocalFileTimeToFileTime@8 0042b158     kernel32:KERNEL32.dll
 0002:0000015c       __imp__DosDateTimeToFileTime@12 0042b15c     kernel32:KERNEL32.dll
 0002:00000160       __imp__SetEndOfFile@4      0042b160     kernel32:KERNEL32.dll
 0002:00000164       __imp__SetStdHandle@8      0042b164     kernel32:KERNEL32.dll
 0002:00000168       __imp__IsBadCodePtr@4      0042b168     kernel32:KERNEL32.dll
 0002:0000016c       __imp__GetEnvironmentStringsW@0 0042b16c     kernel32:KERNEL32.dll
 0002:00000170       __imp__FreeEnvironmentStringsW@4 0042b170     kernel32:KERNEL32.dll
 0002:00000174       __imp__GetFileType@4       0042b174     kernel32:KERNEL32.dll
 0002:00000178       __imp__GetStdHandle@4      0042b178     kernel32:KERNEL32.dll
 0002:0000017c       __imp__SetHandleCount@4    0042b17c     kernel32:KERNEL32.dll
 0002:00000180       __imp__GetStringTypeW@16   0042b180     kernel32:KERNEL32.dll
 0002:00000184       __imp__GetStringTypeA@20   0042b184     kernel32:KERNEL32.dll
 0002:00000188       __imp__UnhandledExceptionFilter@4 0042b188     kernel32:KERNEL32.dll
 0002:0000018c       __imp__LCMapStringW@24     0042b18c     kernel32:KERNEL32.dll
 0002:00000190       __imp__LCMapStringA@24     0042b190     kernel32:KERNEL32.dll
 0002:00000194       __imp__IsBadWritePtr@8     0042b194     kernel32:KERNEL32.dll
 0002:00000198       __imp__VirtualFree@12      0042b198     kernel32:KERNEL32.dll
 0002:0000019c       __imp__HeapCreate@12       0042b19c     kernel32:KERNEL32.dll
 0002:000001a0       __imp__HeapDestroy@4       0042b1a0     kernel32:KERNEL32.dll
 0002:000001a4       __imp__HeapSize@12         0042b1a4     kernel32:KERNEL32.dll
 0002:000001a8       __imp__SetLastError@4      0042b1a8     kernel32:KERNEL32.dll
 0002:000001ac       __imp__TlsAlloc@0          0042b1ac     kernel32:KERNEL32.dll
 0002:000001b0       __imp__GetVersion@0        0042b1b0     kernel32:KERNEL32.dll
 0002:000001b4       __imp__CreateEventA@16     0042b1b4     kernel32:KERNEL32.dll
 0002:000001b8       __imp__Sleep@4             0042b1b8     kernel32:KERNEL32.dll
 0002:000001bc       __imp__SetFilePointer@16   0042b1bc     kernel32:KERNEL32.dll
 0002:000001c0       __imp__WriteFile@20        0042b1c0     kernel32:KERNEL32.dll
 0002:000001c4       __imp__FlushFileBuffers@4  0042b1c4     kernel32:KERNEL32.dll
 0002:000001c8       __imp__WideCharToMultiByte@32 0042b1c8     kernel32:KERNEL32.dll
 0002:000001cc       __imp__ReleaseMutex@4      0042b1cc     kernel32:KERNEL32.dll
 0002:000001d0       __imp__WaitForSingleObject@8 0042b1d0     kernel32:KERNEL32.dll
 0002:000001d4       __imp__CreateMutexA@12     0042b1d4     kernel32:KERNEL32.dll
 0002:000001d8       __imp__UnmapViewOfFile@4   0042b1d8     kernel32:KERNEL32.dll
 0002:000001dc       __imp__CreateFileA@28      0042b1dc     kernel32:KERNEL32.dll
 0002:000001e0       __imp__GetFileSize@8       0042b1e0     kernel32:KERNEL32.dll
 0002:000001e4       __imp__CloseHandle@4       0042b1e4     kernel32:KERNEL32.dll
 0002:000001e8       __imp__MapViewOfFile@20    0042b1e8     kernel32:KERNEL32.dll
 0002:000001ec       __imp__GetProcAddress@8    0042b1ec     kernel32:KERNEL32.dll
 0002:000001f0       __imp__ReadFile@20         0042b1f0     kernel32:KERNEL32.dll
 0002:000001f4       __imp__FreeLibrary@4       0042b1f4     kernel32:KERNEL32.dll
 0002:000001f8       __imp__LoadLibraryA@4      0042b1f8     kernel32:KERNEL32.dll
 0002:000001fc       __imp__GetModuleHandleA@4  0042b1fc     kernel32:KERNEL32.dll
 0002:00000200       __imp__LeaveCriticalSection@4 0042b200     kernel32:KERNEL32.dll
 0002:00000204       __imp__EnterCriticalSection@4 0042b204     kernel32:KERNEL32.dll
 0002:00000208       __imp__DeleteCriticalSection@4 0042b208     kernel32:KERNEL32.dll
 0002:0000020c       __imp__QueryPerformanceFrequency@4 0042b20c     kernel32:KERNEL32.dll
 0002:00000210       __imp__InitializeCriticalSection@4 0042b210     kernel32:KERNEL32.dll
 0002:00000214       __imp__GetCommandLineA@0   0042b214     kernel32:KERNEL32.dll
 0002:00000218       __imp__GetStartupInfoA@4   0042b218     kernel32:KERNEL32.dll
 0002:0000021c       __imp__SetConsoleCtrlHandler@8 0042b21c     kernel32:KERNEL32.dll
 0002:00000220       __imp__GetCPInfo@8         0042b220     kernel32:KERNEL32.dll
 0002:00000224       __imp__TlsGetValue@4       0042b224     kernel32:KERNEL32.dll
 0002:00000228       __imp__TlsSetValue@8       0042b228     kernel32:KERNEL32.dll
 0002:0000022c       __imp__HeapReAlloc@16      0042b22c     kernel32:KERNEL32.dll
 0002:00000230       __imp__HeapFree@12         0042b230     kernel32:KERNEL32.dll
 0002:00000234       __imp__HeapAlloc@12        0042b234     kernel32:KERNEL32.dll
 0002:00000238       __imp__RtlUnwind@16        0042b238     kernel32:KERNEL32.dll
 0002:0000023c       \177KERNEL32_NULL_THUNK_DATA 0042b23c     kernel32:KERNEL32.dll
 0002:00000240       __imp__SetupIterateCabinetA@16 0042b240     setupapi:SETUPAPI.dll
 0002:00000244       \177SETUPAPI_NULL_THUNK_DATA 0042b244     setupapi:SETUPAPI.dll
 0002:00000248       __imp__ShellExecuteA@24    0042b248     shell32:SHELL32.dll
 0002:0000024c       \177SHELL32_NULL_THUNK_DATA 0042b24c     shell32:SHELL32.dll
 0002:00000250       __imp__MessageBoxW@16      0042b250     user32:USER32.dll
 0002:00000254       __imp__SystemParametersInfoA@16 0042b254     user32:USER32.dll
 0002:00000258       __imp__GetSystemMetrics@4  0042b258     user32:USER32.dll
 0002:0000025c       __imp__MessageBoxA@16      0042b25c     user32:USER32.dll
 0002:00000260       __imp__SetWindowsHookExA@16 0042b260     user32:USER32.dll
 0002:00000264       __imp__UnhookWindowsHookEx@4 0042b264     user32:USER32.dll
 0002:00000268       __imp__GetClassNameA@12    0042b268     user32:USER32.dll
 0002:0000026c       __imp__PostMessageA@16     0042b26c     user32:USER32.dll
 0002:00000270       __imp__CallNextHookEx@16   0042b270     user32:USER32.dll
 0002:00000274       \177USER32_NULL_THUNK_DATA 0042b274     user32:USER32.dll
 0002:00000278       __imp__GetFileVersionInfoSizeA@8 0042b278     Version:VERSION.dll
 0002:0000027c       __imp__VerQueryValueA@16   0042b27c     Version:VERSION.dll
 0002:00000280       __imp__GetFileVersionInfoA@16 0042b280     Version:VERSION.dll
 0002:00000284       \177VERSION_NULL_THUNK_DATA 0042b284     Version:VERSION.dll
 0002:00000288       __imp__timeGetTime@0       0042b288     winmm:WINMM.dll
 0002:0000028c       \177WINMM_NULL_THUNK_DATA  0042b28c     winmm:WINMM.dll
 0002:00000290       __imp__CoCreateGuid@4      0042b290     ole32:ole32.dll
 0002:00000294       \177ole32_NULL_THUNK_DATA  0042b294     ole32:ole32.dll
 0002:00000298       ??_7JLockable@@6B@         0042b298     j_criticalsection.obj
 0002:000002ac       ??_C@_08GONM@kernel32?$AA@ 0042b2ac     j_criticalsection.obj
 0002:000002b8       ??_7JDynLoadSystem@@6B@    0042b2b8     j_criticalsection.obj
 0002:000002c8       ??_7JDynLoadStub@@6B@      0042b2c8     j_criticalsection.obj
 0002:000002d8       ??_7JDynLoad@@6B@          0042b2d8     j_criticalsection.obj
 0002:000002e8       __real@8@00000000000000000000 0042b2e8     j_dib.obj
 0002:000002f0       ??_C@_04EJNG@?4dll?$AA@    0042b2f0     j_dynload.obj
 0002:000002f8       ??_C@_02FCOO@?1?1?$AA@     0042b2f8     j_stoken.obj
 0002:000002fc       ??_C@_03DHKI@?o?$LL?$LP?$AA@ 0042b2fc     j_stoken.obj
 0002:00000300       ??_C@_00A@?$AA@            0042b300     j_stoken.obj
 0002:00000304       ??_C@_04DGBN@?$BL$?$CJC?$AA@ 0042b304     j_str.obj
 0002:0000030c       ??_C@_02NNNG@?$HO?$HN?$AA@ 0042b30c     j_str.obj
 0002:00000310       ??_C@_02CCKE@?$HO?$HL?$AA@ 0042b310     j_str.obj
 0002:00000314       ??_C@_02CCGP@?$HO?$HO?$AA@ 0042b314     j_str.obj
 0002:00000318       ??_C@_03NHAM@?$BL?$CIB?$AA@ 0042b318     j_str.obj
 0002:0000031c       ??_C@_03HMAN@?$BL?$CII?$AA@ 0042b31c     j_str.obj
 0002:00000320       ??_C@_03DIPC@?$BL$B?$AA@   0042b320     j_str.obj
 0002:00000338       ??_C@_07EJCK@combase?$AA@  0042b338     j_wintrd.obj
 0002:00000340       ??_C@_05NKLI@ole32?$AA@    0042b340     j_wintrd.obj
 0002:00000468       ??_C@_0BL@HLLE@Raw?5Convert?$CIchar?9?$DOwchar_t?$CJ?$AA@ 0042b468     j_wstr.obj
 0002:00000484       ??_C@_03OFLH@RAW?$AA@      0042b484     j_wstr.obj
 0002:00000488       ??_C@_0P@HGIB@Unicode?$CIUTF?98?$CJ?$AA@ 0042b488     j_wstr.obj
 0002:00000498       ??_C@_05FFKO@UTF?98?$AA@   0042b498     j_wstr.obj
 0002:000004a0       ??_C@_0BC@BOOJ@Ukrainian?$CIKOI8?9U?$CJ?$AA@ 0042b4a0     j_wstr.obj
 0002:000004b4       ??_C@_06JLFM@KOI8?9U?$AA@  0042b4b4     j_wstr.obj
 0002:000004bc       ??_C@_0BA@LBFH@Russian?$CIKOI8?9R?$CJ?$AA@ 0042b4bc     j_wstr.obj
 0002:000004cc       ??_C@_06MOLJ@KOI8?9R?$AA@  0042b4cc     j_wstr.obj
 0002:000004d4       ??_C@_0BB@FMMC@Cyrillic?$CICP1251?$CJ?$AA@ 0042b4d4     j_wstr.obj
 0002:000004e8       ??_C@_08CNCJ@x?9cp1251?$AA@ 0042b4e8     j_wstr.obj
 0002:000004f4       ??_C@_0N@JCHI@windows?91251?$AA@ 0042b4f4     j_wstr.obj
 0002:00000504       ??_C@_0BA@IMEL@Cyrillic?$CICP866?$CJ?$AA@ 0042b504     j_wstr.obj
 0002:00000514       ??_C@_07EJJF@x?9cp866?$AA@ 0042b514     j_wstr.obj
 0002:0000051c       ??_C@_05HJJL@cp866?$AA@    0042b51c     j_wstr.obj
 0002:00000524       ??_C@_0M@IHLF@Korean?$CIISO?$CJ?$AA@ 0042b524     j_wstr.obj
 0002:00000530       ??_C@_0M@KMHM@ISO?92022?9KR?$AA@ 0042b530     j_wstr.obj
 0002:0000053c       ??_C@_0M@DLOE@Korean?$CIEUC?$CJ?$AA@ 0042b53c     j_wstr.obj
 0002:00000548       ??_C@_03PLAE@UHC?$AA@      0042b548     j_wstr.obj
 0002:0000054c       ??_C@_06OFH@EUC?9KR?$AA@   0042b54c     j_wstr.obj
 0002:00000554       ??_C@_0O@PEDG@Japanese?$CIJIS?$CJ?$AA@ 0042b554     j_wstr.obj
 0002:00000564       ??_C@_0M@OPPI@ISO?92022?9JP?$AA@ 0042b564     j_wstr.obj
 0002:00000570       ??_C@_0O@LHDE@Japanese?$CIEUC?$CJ?$AA@ 0042b570     j_wstr.obj
 0002:00000580       ??_C@_08LHDB@X?9EUC?9JP?$AA@ 0042b580     j_wstr.obj
 0002:0000058c       ??_C@_06ENND@EUC?9JP?$AA@  0042b58c     j_wstr.obj
 0002:00000594       ??_C@_0BD@FHAA@Japanese?$CIShiftJIS?$CJ?$AA@ 0042b594     j_wstr.obj
 0002:000005a8       ??_C@_06JPAI@X?9SJIS?$AA@  0042b5a8     j_wstr.obj
 0002:000005b0       ??_C@_09MHON@Shift?9JIS?$AA@ 0042b5b0     j_wstr.obj
 0002:000005bc       ??_C@_0BM@HHJI@Chinese?9GB18030?$CIWinXP?5Only?$CJ?$AA@ 0042b5bc     j_wstr.obj
 0002:000005d8       ??_C@_07EAML@GB18030?$AA@  0042b5d8     j_wstr.obj
 0002:000005e0       ??_C@_0BH@FNHG@Chinese?9Simplified?$CIHZ?$CJ?$AA@ 0042b5e0     j_wstr.obj
 0002:000005f8       ??_C@_09ECO@HZ?9GB2312?$AA@ 0042b5f8     j_wstr.obj
 0002:00000604       ??_C@_0BI@HAMB@Chinese?9Simplified?$CIGBK?$CJ?$AA@ 0042b604     j_wstr.obj
 0002:0000061c       ??_C@_03LCPK@GBK?$AA@      0042b61c     j_wstr.obj
 0002:00000620       ??_C@_06OONL@GB2312?$AA@   0042b620     j_wstr.obj
 0002:00000628       ??_C@_0BK@JOLN@Chinese?9Traditional?$CIBig5?$CJ?$AA@ 0042b628     j_wstr.obj
 0002:00000644       ??_C@_04POAE@Big5?$AA@     0042b644     j_wstr.obj
 0002:0000064c       ??_C@_0L@KGGH@ISO?98859?91?$AA@ 0042b64c     j_wstr.obj
 0002:00000658       ??_C@_05OGAG@ASCII?$AA@    0042b658     j_wstr.obj
 0002:00000660       ??_C@_0BA@DKCI@Default?5Charset?$AA@ 0042b660     j_wstr.obj
 0002:00000670       ??_C@_08DGLP@OSNative?$AA@ 0042b670     j_wstr.obj
 0002:0000067c       ??_C@_04EJDC@?4drv?$AA@    0042b67c     jgxbase.obj
 0002:00000684       ??_C@_04PIHF@?4ocx?$AA@    0042b684     jgxbase.obj
 0002:0000068c       ??_C@_01PCFE@?2?$AA@       0042b68c     jgxbase.obj
 0002:00000690       ?convTable@@3QBEB          0042b690     libc_custom.obj
 0002:00000870       ??_C@_02MHMJ@?$CFu?$AA@    0042b870     libc_custom.obj
 0002:00000874       ??_C@_15NIED@?$AA?$CF?$AAu?$AA?$AA@ 0042b874     libc_custom.obj
 0002:0000087c       ??_C@_0BE@EPFF@GetTokenInformation?$AA@ 0042b87c     sp_adjustpriv.obj
 0002:00000890       ??_C@_0BG@GACJ@AdjustTokenPrivileges?$AA@ 0042b890     sp_adjustpriv.obj
 0002:000008a8       ??_C@_0BG@EFIJ@LookupPrivilegeValueA?$AA@ 0042b8a8     sp_adjustpriv.obj
 0002:000008c0       ??_C@_0BB@NPFI@OpenProcessToken?$AA@ 0042b8c0     sp_adjustpriv.obj
 0002:000008d4       ??_C@_08FJEH@advapi32?$AA@ 0042b8d4     sp_adjustpriv.obj
 0002:00000ec8       ??_C@_19BNP@?$AAz?$AAw?$AAn?$AAj?$AA?$AA@ 0042bec8     sp_char.obj
 0002:00000ed4       ??_C@_17CLLG@?$AAz?$AAw?$AAj?$AA?$AA@ 0042bed4     sp_char.obj
 0002:00000edc       ??_C@_19JABF@?$AAz?$AAe?$AAt?$AAa?$AA?$AA@ 0042bedc     sp_char.obj
 0002:00000ee8       ??_C@_19BGDE@?$AAy?$AAu?$AAm?$AAl?$AA?$AA@ 0042bee8     sp_char.obj
 0002:00000ef4       ??_C@_17FCEN@?$AAy?$AAe?$AAn?$AA?$AA@ 0042bef4     sp_char.obj
 0002:00000efc       ??_C@_1O@GHAC@?$AAy?$AAa?$AAc?$AAu?$AAt?$AAe?$AA?$AA@ 0042befc     sp_char.obj
 0002:00000f0c       ??_C@_15LFN@?$AAx?$AAi?$AA?$AA@ 0042bf0c     sp_char.obj
 0002:00000f14       ??_C@_1O@CFEM@?$AAw?$AAe?$AAi?$AAe?$AAr?$AAp?$AA?$AA@ 0042bf14     sp_char.obj
 0002:00000f24       ??_C@_19NFF@?$AAu?$AAu?$AAm?$AAl?$AA?$AA@ 0042bf24     sp_char.obj
 0002:00000f30       ??_C@_1BA@HOPE@?$AAu?$AAp?$AAs?$AAi?$AAl?$AAo?$AAn?$AA?$AA@ 0042bf30     sp_char.obj
 0002:00000f40       ??_C@_1M@PDML@?$AAu?$AAp?$AAs?$AAi?$AAh?$AA?$AA@ 0042bf40     sp_char.obj
 0002:00000f4c       ??_C@_17DJLB@?$AAu?$AAm?$AAl?$AA?$AA@ 0042bf4c     sp_char.obj
 0002:00000f54       ??_C@_1O@CDHG@?$AAu?$AAg?$AAr?$AAa?$AAv?$AAe?$AA?$AA@ 0042bf54     sp_char.obj
 0002:00000f64       ??_C@_1M@NEND@?$AAu?$AAc?$AAi?$AAr?$AAc?$AA?$AA@ 0042bf64     sp_char.obj
 0002:00000f70       ??_C@_19GAHE@?$AAu?$AAa?$AAr?$AAr?$AA?$AA@ 0042bf70     sp_char.obj
 0002:00000f7c       ??_C@_1O@KJNK@?$AAu?$AAa?$AAc?$AAu?$AAt?$AAe?$AA?$AA@ 0042bf7c     sp_char.obj
 0002:00000f8c       ??_C@_19LCMA@?$AAu?$AAA?$AAr?$AAr?$AA?$AA@ 0042bf8c     sp_char.obj
 0002:00000f98       ??_C@_1M@ICMG@?$AAt?$AAr?$AAa?$AAd?$AAe?$AA?$AA@ 0042bf98     sp_char.obj
 0002:00000fa4       ??_C@_1M@FBBO@?$AAt?$AAi?$AAm?$AAe?$AAs?$AA?$AA@ 0042bfa4     sp_char.obj
 0002:00000fb0       ??_C@_1M@BCLD@?$AAt?$AAi?$AAl?$AAd?$AAe?$AA?$AA@ 0042bfb0     sp_char.obj
 0002:00000fbc       ??_C@_1M@HEB@?$AAt?$AAh?$AAo?$AAr?$AAn?$AA?$AA@ 0042bfbc     sp_char.obj
 0002:00000fc8       ??_C@_1O@GFAC@?$AAt?$AAh?$AAi?$AAn?$AAs?$AAp?$AA?$AA@ 0042bfc8     sp_char.obj
 0002:00000fd8       ??_C@_1BC@HCEF@?$AAt?$AAh?$AAe?$AAt?$AAa?$AAs?$AAy?$AAm?$AA?$AA@ 0042bfd8     sp_char.obj
 0002:00000fec       ??_C@_1M@MAMM@?$AAt?$AAh?$AAe?$AAt?$AAa?$AA?$AA@ 0042bfec     sp_char.obj
 0002:00000ff8       ??_C@_1O@FGLI@?$AAt?$AAh?$AAe?$AAr?$AAe?$AA4?$AA?$AA@ 0042bff8     sp_char.obj
 0002:00001008       ??_C@_17HFFC@?$AAt?$AAa?$AAu?$AA?$AA@ 0042c008     sp_char.obj
 0002:00001010       ??_C@_1M@GAPB@?$AAs?$AAz?$AAl?$AAi?$AAg?$AA?$AA@ 0042c010     sp_char.obj
 0002:0000101c       ??_C@_19GBIJ@?$AAs?$AAu?$AAp?$AAe?$AA?$AA@ 0042c01c     sp_char.obj
 0002:00001028       ??_C@_19CJDO@?$AAs?$AAu?$AAp?$AA3?$AA?$AA@ 0042c028     sp_char.obj
 0002:00001034       ??_C@_19HLCI@?$AAs?$AAu?$AAp?$AA2?$AA?$AA@ 0042c034     sp_char.obj
 0002:00001040       ??_C@_19INBD@?$AAs?$AAu?$AAp?$AA1?$AA?$AA@ 0042c040     sp_char.obj
 0002:0000104c       ??_C@_17CEDG@?$AAs?$AAu?$AAp?$AA?$AA@ 0042c04c     sp_char.obj
 0002:00001054       ??_C@_17IPKF@?$AAs?$AAu?$AAm?$AA?$AA@ 0042c054     sp_char.obj
 0002:0000105c       ??_C@_19CDJG@?$AAs?$AAu?$AAb?$AAe?$AA?$AA@ 0042c05c     sp_char.obj
 0002:00001068       ??_C@_17KBHB@?$AAs?$AAu?$AAb?$AA?$AA@ 0042c068     sp_char.obj
 0002:00001070       ??_C@_1O@CAPH@?$AAs?$AAp?$AAa?$AAd?$AAe?$AAs?$AA?$AA@ 0042c070     sp_char.obj
 0002:00001080       ??_C@_17MEP@?$AAs?$AAi?$AAm?$AA?$AA@ 0042c080     sp_char.obj
 0002:00001088       ??_C@_1O@FKMB@?$AAs?$AAi?$AAg?$AAm?$AAa?$AAf?$AA?$AA@ 0042c088     sp_char.obj
 0002:00001098       ??_C@_1M@GJFK@?$AAs?$AAi?$AAg?$AAm?$AAa?$AA?$AA@ 0042c098     sp_char.obj
 0002:000010a4       ??_C@_17MFFK@?$AAs?$AAh?$AAy?$AA?$AA@ 0042c0a4     sp_char.obj
 0002:000010ac       ??_C@_19BJJF@?$AAs?$AAe?$AAc?$AAt?$AA?$AA@ 0042c0ac     sp_char.obj
 0002:000010b8       ??_C@_19LGLP@?$AAs?$AAd?$AAo?$AAt?$AA?$AA@ 0042c0b8     sp_char.obj
 0002:000010c4       ??_C@_1O@FDEP@?$AAs?$AAc?$AAa?$AAr?$AAo?$AAn?$AA?$AA@ 0042c0c4     sp_char.obj
 0002:000010d4       ??_C@_1M@EMFJ@?$AAs?$AAb?$AAq?$AAu?$AAo?$AA?$AA@ 0042c0d4     sp_char.obj
 0002:000010e0       ??_C@_1M@EABM@?$AAr?$AAs?$AAq?$AAu?$AAo?$AA?$AA@ 0042c0e0     sp_char.obj
 0002:000010ec       ??_C@_1O@MIED@?$AAr?$AAs?$AAa?$AAq?$AAu?$AAo?$AA?$AA@ 0042c0ec     sp_char.obj
 0002:000010fc       ??_C@_17CGK@?$AAr?$AAl?$AAm?$AA?$AA@ 0042c0fc     sp_char.obj
 0002:00001104       ??_C@_17CGNC@?$AAr?$AAh?$AAo?$AA?$AA@ 0042c104     sp_char.obj
 0002:0000110c       ??_C@_1O@GLAK@?$AAr?$AAf?$AAl?$AAo?$AAo?$AAr?$AA?$AA@ 0042c10c     sp_char.obj
 0002:0000111c       ??_C@_17JHPN@?$AAr?$AAe?$AAg?$AA?$AA@ 0042c11c     sp_char.obj
 0002:00001124       ??_C@_19CKEI@?$AAr?$AAe?$AAa?$AAl?$AA?$AA@ 0042c124     sp_char.obj
 0002:00001130       ??_C@_1M@CLGG@?$AAr?$AAd?$AAq?$AAu?$AAo?$AA?$AA@ 0042c130     sp_char.obj
 0002:0000113c       ??_C@_1M@ECED@?$AAr?$AAc?$AAe?$AAi?$AAl?$AA?$AA@ 0042c13c     sp_char.obj
 0002:00001148       ??_C@_19CPIM@?$AAr?$AAa?$AAr?$AAr?$AA?$AA@ 0042c148     sp_char.obj
 0002:00001154       ??_C@_1M@OAAO@?$AAr?$AAa?$AAq?$AAu?$AAo?$AA?$AA@ 0042c154     sp_char.obj
 0002:00001160       ??_C@_19JHEA@?$AAr?$AAa?$AAn?$AAg?$AA?$AA@ 0042c160     sp_char.obj
 0002:0000116c       ??_C@_1M@MGJC@?$AAr?$AAa?$AAd?$AAi?$AAc?$AA?$AA@ 0042c16c     sp_char.obj
 0002:00001178       ??_C@_19PNDI@?$AAr?$AAA?$AAr?$AAr?$AA?$AA@ 0042c178     sp_char.obj
 0002:00001184       ??_C@_19PFOA@?$AAq?$AAu?$AAo?$AAt?$AA?$AA@ 0042c184     sp_char.obj
 0002:00001190       ??_C@_17HEJO@?$AAp?$AAs?$AAi?$AA?$AA@ 0042c190     sp_char.obj
 0002:00001198       ??_C@_19LGBK@?$AAp?$AAr?$AAo?$AAp?$AA?$AA@ 0042c198     sp_char.obj
 0002:000011a4       ??_C@_19NPCK@?$AAp?$AAr?$AAo?$AAd?$AA?$AA@ 0042c1a4     sp_char.obj
 0002:000011b0       ??_C@_1M@PNFL@?$AAp?$AAr?$AAi?$AAm?$AAe?$AA?$AA@ 0042c1b0     sp_char.obj
 0002:000011bc       ??_C@_1M@JFCI@?$AAp?$AAo?$AAu?$AAn?$AAd?$AA?$AA@ 0042c1bc     sp_char.obj
 0002:000011c8       ??_C@_1O@CCFF@?$AAp?$AAl?$AAu?$AAs?$AAm?$AAn?$AA?$AA@ 0042c1c8     sp_char.obj
 0002:000011d8       ??_C@_17DIBF@?$AAp?$AAi?$AAv?$AA?$AA@ 0042c1d8     sp_char.obj
 0002:000011e0       ??_C@_15KHH@?$AAp?$AAi?$AA?$AA@ 0042c1e0     sp_char.obj
 0002:000011e8       ??_C@_17JHIO@?$AAp?$AAh?$AAi?$AA?$AA@ 0042c1e8     sp_char.obj
 0002:000011f0       ??_C@_19LFGH@?$AAp?$AAe?$AAr?$AAp?$AA?$AA@ 0042c1f0     sp_char.obj
 0002:000011fc       ??_C@_1O@INGO@?$AAp?$AAe?$AAr?$AAm?$AAi?$AAl?$AA?$AA@ 0042c1fc     sp_char.obj
 0002:0000120c       ??_C@_19EHGL@?$AAp?$AAa?$AAr?$AAt?$AA?$AA@ 0042c20c     sp_char.obj
 0002:00001218       ??_C@_19HMEN@?$AAp?$AAa?$AAr?$AAa?$AA?$AA@ 0042c218     sp_char.obj
 0002:00001224       ??_C@_19LPAG@?$AAo?$AAu?$AAm?$AAl?$AA?$AA@ 0042c224     sp_char.obj
 0002:00001230       ??_C@_1O@BKLH@?$AAo?$AAt?$AAi?$AAm?$AAe?$AAs?$AA?$AA@ 0042c230     sp_char.obj
 0002:00001240       ??_C@_1O@FJBK@?$AAo?$AAt?$AAi?$AAl?$AAd?$AAe?$AA?$AA@ 0042c240     sp_char.obj
 0002:00001250       ??_C@_1O@POF@?$AAo?$AAs?$AAl?$AAa?$AAs?$AAh?$AA?$AA@ 0042c250     sp_char.obj
 0002:00001260       ??_C@_19IFPH@?$AAo?$AAr?$AAd?$AAm?$AA?$AA@ 0042c260     sp_char.obj
 0002:0000126c       ??_C@_19ODHJ@?$AAo?$AAr?$AAd?$AAf?$AA?$AA@ 0042c26c     sp_char.obj
 0002:00001278       ??_C@_15COBG@?$AAo?$AAr?$AA?$AA@ 0042c278     sp_char.obj
 0002:00001280       ??_C@_1M@EKEH@?$AAo?$AAp?$AAl?$AAu?$AAs?$AA?$AA@ 0042c280     sp_char.obj
 0002:0000128c       ??_C@_1BA@IIBO@?$AAo?$AAm?$AAi?$AAc?$AAr?$AAo?$AAn?$AA?$AA@ 0042c28c     sp_char.obj
 0002:0000129c       ??_C@_1M@CKIM@?$AAo?$AAm?$AAe?$AAg?$AAa?$AA?$AA@ 0042c29c     sp_char.obj
 0002:000012a8       ??_C@_1M@MPGK@?$AAo?$AAl?$AAi?$AAn?$AAe?$AA?$AA@ 0042c2a8     sp_char.obj
 0002:000012b4       ??_C@_1O@BMBM@?$AAo?$AAg?$AAr?$AAa?$AAv?$AAe?$AA?$AA@ 0042c2b4     sp_char.obj
 0002:000012c4       ??_C@_1M@EPHH@?$AAo?$AAe?$AAl?$AAi?$AAg?$AA?$AA@ 0042c2c4     sp_char.obj
 0002:000012d0       ??_C@_1M@PNEO@?$AAo?$AAc?$AAi?$AAr?$AAc?$AA?$AA@ 0042c2d0     sp_char.obj
 0002:000012dc       ??_C@_1O@JGLA@?$AAo?$AAa?$AAc?$AAu?$AAt?$AAe?$AA?$AA@ 0042c2dc     sp_char.obj
 0002:000012ec       ??_C@_15DAFC@?$AAn?$AAu?$AA?$AA@ 0042c2ec     sp_char.obj
 0002:000012f4       ??_C@_1O@IHH@?$AAn?$AAt?$AAi?$AAl?$AAd?$AAe?$AA?$AA@ 0042c2f4     sp_char.obj
 0002:00001304       ??_C@_19OFIO@?$AAn?$AAs?$AAu?$AAb?$AA?$AA@ 0042c304     sp_char.obj
 0002:00001310       ??_C@_1M@GMHN@?$AAn?$AAo?$AAt?$AAi?$AAn?$AA?$AA@ 0042c310     sp_char.obj
 0002:0000131c       ??_C@_17CGGN@?$AAn?$AAo?$AAt?$AA?$AA@ 0042c31c     sp_char.obj
 0002:00001324       ??_C@_15MJNH@?$AAn?$AAi?$AA?$AA@ 0042c324     sp_char.obj
 0002:0000132c       ??_C@_15BBDI@?$AAn?$AAe?$AA?$AA@ 0042c32c     sp_char.obj
 0002:00001334       ??_C@_1M@OKDP@?$AAn?$AAd?$AAa?$AAs?$AAh?$AA?$AA@ 0042c334     sp_char.obj
 0002:00001340       ??_C@_19GHNJ@?$AAn?$AAb?$AAs?$AAp?$AA?$AA@ 0042c340     sp_char.obj
 0002:0000134c       ??_C@_1M@PDMP@?$AAn?$AAa?$AAb?$AAl?$AAa?$AA?$AA@ 0042c34c     sp_char.obj
 0002:00001358       ??_C@_15NADN@?$AAm?$AAu?$AA?$AA@ 0042c358     sp_char.obj
 0002:00001360       ??_C@_1M@DGPI@?$AAm?$AAi?$AAn?$AAu?$AAs?$AA?$AA@ 0042c360     sp_char.obj
 0002:0000136c       ??_C@_1O@HIEO@?$AAm?$AAi?$AAd?$AAd?$AAo?$AAt?$AA?$AA@ 0042c36c     sp_char.obj
 0002:0000137c       ??_C@_1M@EPOJ@?$AAm?$AAi?$AAc?$AAr?$AAo?$AA?$AA@ 0042c37c     sp_char.obj
 0002:00001388       ??_C@_1M@NFKP@?$AAm?$AAd?$AAa?$AAs?$AAh?$AA?$AA@ 0042c388     sp_char.obj
 0002:00001394       ??_C@_19PEMH@?$AAm?$AAa?$AAc?$AAr?$AA?$AA@ 0042c394     sp_char.obj
 0002:000013a0       ??_C@_15CCAO@?$AAl?$AAt?$AA?$AA@ 0042c3a0     sp_char.obj
 0002:000013a8       ??_C@_1M@MDLO@?$AAl?$AAs?$AAq?$AAu?$AAo?$AA?$AA@ 0042c3a8     sp_char.obj
 0002:000013b4       ??_C@_1O@LCJO@?$AAl?$AAs?$AAa?$AAq?$AAu?$AAo?$AA?$AA@ 0042c3b4     sp_char.obj
 0002:000013c4       ??_C@_17LLEA@?$AAl?$AAr?$AAm?$AA?$AA@ 0042c3c4     sp_char.obj
 0002:000013cc       ??_C@_17HIE@?$AAl?$AAo?$AAz?$AA?$AA@ 0042c3cc     sp_char.obj
 0002:000013d4       ??_C@_1O@CDHA@?$AAl?$AAo?$AAw?$AAa?$AAs?$AAt?$AA?$AA@ 0042c3d4     sp_char.obj
 0002:000013e4       ??_C@_1O@BBNH@?$AAl?$AAf?$AAl?$AAo?$AAo?$AAr?$AA?$AA@ 0042c3e4     sp_char.obj
 0002:000013f4       ??_C@_15FBHC@?$AAl?$AAe?$AA?$AA@ 0042c3f4     sp_char.obj
 0002:000013fc       ??_C@_1M@KIME@?$AAl?$AAd?$AAq?$AAu?$AAo?$AA?$AA@ 0042c3fc     sp_char.obj
 0002:00001408       ??_C@_1M@MBOB@?$AAl?$AAc?$AAe?$AAi?$AAl?$AA?$AA@ 0042c408     sp_char.obj
 0002:00001414       ??_C@_19JEPP@?$AAl?$AAa?$AAr?$AAr?$AA?$AA@ 0042c414     sp_char.obj
 0002:00001420       ??_C@_1M@GDKM@?$AAl?$AAa?$AAq?$AAu?$AAo?$AA?$AA@ 0042c420     sp_char.obj
 0002:0000142c       ??_C@_19CMDD@?$AAl?$AAa?$AAn?$AAg?$AA?$AA@ 0042c42c     sp_char.obj
 0002:00001438       ??_C@_1O@JAEK@?$AAl?$AAa?$AAm?$AAb?$AAd?$AAa?$AA?$AA@ 0042c438     sp_char.obj
 0002:00001448       ??_C@_19EGEL@?$AAl?$AAA?$AAr?$AAr?$AA?$AA@ 0042c448     sp_char.obj
 0002:00001454       ??_C@_1M@IEOE@?$AAk?$AAa?$AAp?$AAp?$AAa?$AA?$AA@ 0042c454     sp_char.obj
 0002:00001460       ??_C@_19DCLG@?$AAi?$AAu?$AAm?$AAl?$AA?$AA@ 0042c460     sp_char.obj
 0002:0000146c       ??_C@_19PBHD@?$AAi?$AAs?$AAi?$AAn?$AA?$AA@ 0042c46c     sp_char.obj
 0002:00001478       ??_C@_1O@IKMO@?$AAi?$AAq?$AAu?$AAe?$AAs?$AAt?$AA?$AA@ 0042c478     sp_char.obj
 0002:00001488       ??_C@_19NLMJ@?$AAi?$AAo?$AAt?$AAa?$AA?$AA@ 0042c488     sp_char.obj
 0002:00001494       ??_C@_17EPKA@?$AAi?$AAn?$AAt?$AA?$AA@ 0042c494     sp_char.obj
 0002:0000149c       ??_C@_1M@IPOL@?$AAi?$AAn?$AAf?$AAi?$AAn?$AA?$AA@ 0042c49c     sp_char.obj
 0002:000014a8       ??_C@_1M@KHKA@?$AAi?$AAm?$AAa?$AAg?$AAe?$AA?$AA@ 0042c4a8     sp_char.obj
 0002:000014b4       ??_C@_1O@PLHA@?$AAi?$AAg?$AAr?$AAa?$AAv?$AAe?$AA?$AA@ 0042c4b4     sp_char.obj
 0002:000014c4       ??_C@_1M@EELF@?$AAi?$AAe?$AAx?$AAc?$AAl?$AA?$AA@ 0042c4c4     sp_char.obj
 0002:000014d0       ??_C@_1M@ICGO@?$AAi?$AAc?$AAi?$AAr?$AAc?$AA?$AA@ 0042c4d0     sp_char.obj
 0002:000014dc       ??_C@_1O@HBNM@?$AAi?$AAa?$AAc?$AAu?$AAt?$AAe?$AA?$AA@ 0042c4dc     sp_char.obj
 0002:000014ec       ??_C@_1O@HMLM@?$AAh?$AAe?$AAl?$AAl?$AAi?$AAp?$AA?$AA@ 0042c4ec     sp_char.obj
 0002:000014fc       ??_C@_1O@KOL@?$AAh?$AAe?$AAa?$AAr?$AAt?$AAs?$AA?$AA@ 0042c4fc     sp_char.obj
 0002:0000150c       ??_C@_19JNNP@?$AAh?$AAa?$AAr?$AAr?$AA?$AA@ 0042c50c     sp_char.obj
 0002:00001518       ??_C@_19EPGL@?$AAh?$AAA?$AAr?$AAr?$AA?$AA@ 0042c518     sp_char.obj
 0002:00001524       ??_C@_15MDEL@?$AAg?$AAt?$AA?$AA@ 0042c524     sp_char.obj
 0002:0000152c       ??_C@_15LADH@?$AAg?$AAe?$AA?$AA@ 0042c52c     sp_char.obj
 0002:00001534       ??_C@_1M@FAFO@?$AAg?$AAa?$AAm?$AAm?$AAa?$AA?$AA@ 0042c534     sp_char.obj
 0002:00001540       ??_C@_1M@FPCJ@?$AAf?$AAr?$AAa?$AAs?$AAl?$AA?$AA@ 0042c540     sp_char.obj
 0002:0000154c       ??_C@_1O@MOBB@?$AAf?$AAr?$AAa?$AAc?$AA3?$AA4?$AA?$AA@ 0042c54c     sp_char.obj
 0002:0000155c       ??_C@_1O@IOFL@?$AAf?$AAr?$AAa?$AAc?$AA1?$AA4?$AA?$AA@ 0042c55c     sp_char.obj
 0002:0000156c       ??_C@_1O@GCCM@?$AAf?$AAr?$AAa?$AAc?$AA1?$AA2?$AA?$AA@ 0042c56c     sp_char.obj
 0002:0000157c       ??_C@_1O@BDPG@?$AAf?$AAo?$AAr?$AAa?$AAl?$AAl?$AA?$AA@ 0042c57c     sp_char.obj
 0002:0000158c       ??_C@_19PFJE@?$AAf?$AAn?$AAo?$AAf?$AA?$AA@ 0042c58c     sp_char.obj
 0002:00001598       ??_C@_1M@DDBK@?$AAe?$AAx?$AAi?$AAs?$AAt?$AA?$AA@ 0042c598     sp_char.obj
 0002:000015a4       ??_C@_19LMGJ@?$AAe?$AAu?$AAr?$AAo?$AA?$AA@ 0042c5a4     sp_char.obj
 0002:000015b0       ??_C@_19CJNH@?$AAe?$AAu?$AAm?$AAl?$AA?$AA@ 0042c5b0     sp_char.obj
 0002:000015bc       ??_C@_17DLOL@?$AAe?$AAt?$AAh?$AA?$AA@ 0042c5bc     sp_char.obj
 0002:000015c4       ??_C@_17PJEI@?$AAe?$AAt?$AAa?$AA?$AA@ 0042c5c4     sp_char.obj
 0002:000015cc       ??_C@_1M@CDKK@?$AAe?$AAq?$AAu?$AAi?$AAv?$AA?$AA@ 0042c5cc     sp_char.obj
 0002:000015d8       ??_C@_1BA@FEPB@?$AAe?$AAp?$AAs?$AAi?$AAl?$AAo?$AAn?$AA?$AA@ 0042c5d8     sp_char.obj
 0002:000015e8       ??_C@_19PNLL@?$AAe?$AAn?$AAs?$AAp?$AA?$AA@ 0042c5e8     sp_char.obj
 0002:000015f4       ??_C@_19IOAF@?$AAe?$AAm?$AAs?$AAp?$AA?$AA@ 0042c5f4     sp_char.obj
 0002:00001600       ??_C@_1M@IFJB@?$AAe?$AAm?$AAp?$AAt?$AAy?$AA?$AA@ 0042c600     sp_char.obj
 0002:0000160c       ??_C@_1O@DFKI@?$AAe?$AAg?$AAr?$AAa?$AAv?$AAe?$AA?$AA@ 0042c60c     sp_char.obj
 0002:0000161c       ??_C@_1M@HMCP@?$AAe?$AAc?$AAi?$AAr?$AAc?$AA?$AA@ 0042c61c     sp_char.obj
 0002:00001628       ??_C@_1O@LPAE@?$AAe?$AAa?$AAc?$AAu?$AAt?$AAe?$AA?$AA@ 0042c628     sp_char.obj
 0002:00001638       ??_C@_1O@HAAJ@?$AAd?$AAi?$AAv?$AAi?$AAd?$AAe?$AA?$AA@ 0042c638     sp_char.obj
 0002:00001648       ??_C@_1M@DGDD@?$AAd?$AAi?$AAa?$AAm?$AAs?$AA?$AA@ 0042c648     sp_char.obj
 0002:00001654       ??_C@_1M@OLCB@?$AAd?$AAe?$AAl?$AAt?$AAa?$AA?$AA@ 0042c654     sp_char.obj
 0002:00001660       ??_C@_17JJNK@?$AAd?$AAe?$AAg?$AA?$AA@ 0042c660     sp_char.obj
 0002:00001668       ??_C@_19IGLO@?$AAd?$AAa?$AAr?$AAr?$AA?$AA@ 0042c668     sp_char.obj
 0002:00001674       ??_C@_1O@GOED@?$AAd?$AAa?$AAg?$AAg?$AAe?$AAr?$AA?$AA@ 0042c674     sp_char.obj
 0002:00001684       ??_C@_19FEAK@?$AAd?$AAA?$AAr?$AAr?$AA?$AA@ 0042c684     sp_char.obj
 0002:00001690       ??_C@_1O@LBHH@?$AAc?$AAu?$AAr?$AAr?$AAe?$AAn?$AA?$AA@ 0042c690     sp_char.obj
 0002:000016a0       ??_C@_17MNGM@?$AAc?$AAu?$AAp?$AA?$AA@ 0042c6a0     sp_char.obj
 0002:000016a8       ??_C@_1M@OCBE@?$AAc?$AAr?$AAa?$AAr?$AAr?$AA?$AA@ 0042c6a8     sp_char.obj
 0002:000016b4       ??_C@_19HMFC@?$AAc?$AAo?$AAp?$AAy?$AA?$AA@ 0042c6b4     sp_char.obj
 0002:000016c0       ??_C@_19OCFK@?$AAc?$AAo?$AAn?$AAg?$AA?$AA@ 0042c6c0     sp_char.obj
 0002:000016cc       ??_C@_1M@FKCI@?$AAc?$AAl?$AAu?$AAb?$AAs?$AA?$AA@ 0042c6cc     sp_char.obj
 0002:000016d8       ??_C@_19MOJH@?$AAc?$AAi?$AAr?$AAc?$AA?$AA@ 0042c6d8     sp_char.obj
 0002:000016e4       ??_C@_17NGK@?$AAc?$AAh?$AAi?$AA?$AA@ 0042c6e4     sp_char.obj
 0002:000016ec       ??_C@_19BMIN@?$AAc?$AAe?$AAn?$AAt?$AA?$AA@ 0042c6ec     sp_char.obj
 0002:000016f8       ??_C@_1M@KDBF@?$AAc?$AAe?$AAd?$AAi?$AAl?$AA?$AA@ 0042c6f8     sp_char.obj
 0002:00001704       ??_C@_1O@CGGE@?$AAc?$AAc?$AAe?$AAd?$AAi?$AAl?$AA?$AA@ 0042c704     sp_char.obj
 0002:00001714       ??_C@_17EPKM@?$AAc?$AAa?$AAp?$AA?$AA@ 0042c714     sp_char.obj
 0002:0000171c       ??_C@_19MGAK@?$AAb?$AAu?$AAl?$AAl?$AA?$AA@ 0042c71c     sp_char.obj
 0002:00001728       ??_C@_1O@OMNP@?$AAb?$AAr?$AAv?$AAb?$AAa?$AAr?$AA?$AA@ 0042c728     sp_char.obj
 0002:00001738       ??_C@_19KGNG@?$AAb?$AAe?$AAt?$AAa?$AA?$AA@ 0042c738     sp_char.obj
 0002:00001744       ??_C@_1M@IDJK@?$AAb?$AAd?$AAq?$AAu?$AAo?$AA?$AA@ 0042c744     sp_char.obj
 0002:00001750       ??_C@_19CAPH@?$AAa?$AAu?$AAm?$AAl?$AA?$AA@ 0042c750     sp_char.obj
 0002:0000175c       ??_C@_1O@DFBJ@?$AAa?$AAt?$AAi?$AAl?$AAd?$AAe?$AA?$AA@ 0042c75c     sp_char.obj
 0002:0000176c       ??_C@_1M@KPBM@?$AAa?$AAs?$AAy?$AAm?$AAp?$AA?$AA@ 0042c76c     sp_char.obj
 0002:00001778       ??_C@_1M@PLGK@?$AAa?$AAr?$AAi?$AAn?$AAg?$AA?$AA@ 0042c778     sp_char.obj
 0002:00001784       ??_C@_17OMFM@?$AAa?$AAn?$AAg?$AA?$AA@ 0042c784     sp_char.obj
 0002:0000178c       ??_C@_17BKGH@?$AAa?$AAn?$AAd?$AA?$AA@ 0042c78c     sp_char.obj
 0002:00001794       ??_C@_17JDDI@?$AAa?$AAm?$AAp?$AA?$AA@ 0042c794     sp_char.obj
 0002:0000179c       ??_C@_1M@NPND@?$AAa?$AAl?$AAp?$AAh?$AAa?$AA?$AA@ 0042c79c     sp_char.obj
 0002:000017a8       ??_C@_1BA@GMLN@?$AAa?$AAl?$AAe?$AAf?$AAs?$AAy?$AAm?$AA?$AA@ 0042c7a8     sp_char.obj
 0002:000017b8       ??_C@_1O@HABP@?$AAa?$AAg?$AAr?$AAa?$AAv?$AAe?$AA?$AA@ 0042c7b8     sp_char.obj
 0002:000017c8       ??_C@_1M@GECJ@?$AAa?$AAe?$AAl?$AAi?$AAg?$AA?$AA@ 0042c7c8     sp_char.obj
 0002:000017d4       ??_C@_1M@NNBJ@?$AAa?$AAc?$AAu?$AAt?$AAe?$AA?$AA@ 0042c7d4     sp_char.obj
 0002:000017e0       ??_C@_1M@NGBA@?$AAa?$AAc?$AAi?$AAr?$AAc?$AA?$AA@ 0042c7e0     sp_char.obj
 0002:000017ec       ??_C@_1O@PKLD@?$AAa?$AAa?$AAc?$AAu?$AAt?$AAe?$AA?$AA@ 0042c7ec     sp_char.obj
 0002:000017fc       ??_C@_19NJBA@?$AAZ?$AAe?$AAt?$AAa?$AA?$AA@ 0042c7fc     sp_char.obj
 0002:00001808       ??_C@_19FPDB@?$AAY?$AAu?$AAm?$AAl?$AA?$AA@ 0042c808     sp_char.obj
 0002:00001814       ??_C@_1O@EKLP@?$AAY?$AAa?$AAc?$AAu?$AAt?$AAe?$AA?$AA@ 0042c814     sp_char.obj
 0002:00001824       ??_C@_15PPH@?$AAX?$AAi?$AA?$AA@ 0042c824     sp_char.obj
 0002:0000182c       ??_C@_19EEFA@?$AAU?$AAu?$AAm?$AAl?$AA?$AA@ 0042c82c     sp_char.obj
 0002:00001838       ??_C@_1BA@CKPO@?$AAU?$AAp?$AAs?$AAi?$AAl?$AAo?$AAn?$AA?$AA@ 0042c838     sp_char.obj
 0002:00001848       ??_C@_1O@OML@?$AAU?$AAg?$AAr?$AAa?$AAv?$AAe?$AA?$AA@ 0042c848     sp_char.obj
 0002:00001858       ??_C@_1M@IFCL@?$AAU?$AAc?$AAi?$AAr?$AAc?$AA?$AA@ 0042c858     sp_char.obj
 0002:00001864       ??_C@_1O@IEGH@?$AAU?$AAa?$AAc?$AAu?$AAt?$AAe?$AA?$AA@ 0042c864     sp_char.obj
 0002:00001874       ??_C@_1M@JBDE@?$AAT?$AAh?$AAe?$AAt?$AAa?$AA?$AA@ 0042c874     sp_char.obj
 0002:00001880       ??_C@_17KHOG@?$AAT?$AAa?$AAu?$AA?$AA@ 0042c880     sp_char.obj
 0002:00001888       ??_C@_1M@ILHH@?$AAT?$AAH?$AAO?$AAR?$AAN?$AA?$AA@ 0042c888     sp_char.obj
 0002:00001894       ??_C@_1M@DIKC@?$AAS?$AAi?$AAg?$AAm?$AAa?$AA?$AA@ 0042c894     sp_char.obj
 0002:000018a0       ??_C@_1O@HOPC@?$AAS?$AAc?$AAa?$AAr?$AAo?$AAn?$AA?$AA@ 0042c8a0     sp_char.obj
 0002:000018b0       ??_C@_17PEGG@?$AAR?$AAh?$AAo?$AA?$AA@ 0042c8b0     sp_char.obj
 0002:000018b8       ??_C@_17KGCK@?$AAP?$AAs?$AAi?$AA?$AA@ 0042c8b8     sp_char.obj
 0002:000018c0       ??_C@_1M@KMKD@?$AAP?$AAr?$AAi?$AAm?$AAe?$AA?$AA@ 0042c8c0     sp_char.obj
 0002:000018cc       ??_C@_15ONN@?$AAP?$AAi?$AA?$AA@ 0042c8cc     sp_char.obj
 0002:000018d4       ??_C@_17EFDK@?$AAP?$AAh?$AAi?$AA?$AA@ 0042c8d4     sp_char.obj
 0002:000018dc       ??_C@_19PGAD@?$AAO?$AAu?$AAm?$AAl?$AA?$AA@ 0042c8dc     sp_char.obj
 0002:000018e8       ??_C@_1O@HEKH@?$AAO?$AAt?$AAi?$AAl?$AAd?$AAe?$AA?$AA@ 0042c8e8     sp_char.obj
 0002:000018f8       ??_C@_1O@CCFI@?$AAO?$AAs?$AAl?$AAa?$AAs?$AAh?$AA?$AA@ 0042c8f8     sp_char.obj
 0002:00001908       ??_C@_1BA@NMBE@?$AAO?$AAm?$AAi?$AAc?$AAr?$AAo?$AAn?$AA?$AA@ 0042c908     sp_char.obj
 0002:00001918       ??_C@_1M@HLHE@?$AAO?$AAm?$AAe?$AAg?$AAa?$AA?$AA@ 0042c918     sp_char.obj
 0002:00001924       ??_C@_1O@DBKB@?$AAO?$AAg?$AAr?$AAa?$AAv?$AAe?$AA?$AA@ 0042c924     sp_char.obj
 0002:00001934       ??_C@_1M@KMLG@?$AAO?$AAc?$AAi?$AAr?$AAc?$AA?$AA@ 0042c934     sp_char.obj
 0002:00001940       ??_C@_1O@LLAN@?$AAO?$AAa?$AAc?$AAu?$AAt?$AAe?$AA?$AA@ 0042c940     sp_char.obj
 0002:00001950       ??_C@_1M@FHIK@?$AAO?$AAE?$AAl?$AAi?$AAg?$AA?$AA@ 0042c950     sp_char.obj
 0002:0000195c       ??_C@_15DEPI@?$AAN?$AAu?$AA?$AA@ 0042c95c     sp_char.obj
 0002:00001964       ??_C@_1O@CFMK@?$AAN?$AAt?$AAi?$AAl?$AAd?$AAe?$AA?$AA@ 0042c964     sp_char.obj
 0002:00001974       ??_C@_15NEJH@?$AAM?$AAu?$AA?$AA@ 0042c974     sp_char.obj
 0002:0000197c       ??_C@_1O@LNPH@?$AAL?$AAa?$AAm?$AAb?$AAd?$AAa?$AA?$AA@ 0042c97c     sp_char.obj
 0002:0000198c       ??_C@_1M@NFBM@?$AAK?$AAa?$AAp?$AAp?$AAa?$AA?$AA@ 0042c98c     sp_char.obj
 0002:00001998       ??_C@_19HLLD@?$AAI?$AAu?$AAm?$AAl?$AA?$AA@ 0042c998     sp_char.obj
 0002:000019a4       ??_C@_19JCMM@?$AAI?$AAo?$AAt?$AAa?$AA?$AA@ 0042c9a4     sp_char.obj
 0002:000019b0       ??_C@_1O@NGMN@?$AAI?$AAg?$AAr?$AAa?$AAv?$AAe?$AA?$AA@ 0042c9b0     sp_char.obj
 0002:000019c0       ??_C@_1M@NDJG@?$AAI?$AAc?$AAi?$AAr?$AAc?$AA?$AA@ 0042c9c0     sp_char.obj
 0002:000019cc       ??_C@_1O@FMGB@?$AAI?$AAa?$AAc?$AAu?$AAt?$AAe?$AA?$AA@ 0042c9cc     sp_char.obj
 0002:000019dc       ??_C@_1M@BKG@?$AAG?$AAa?$AAm?$AAm?$AAa?$AA?$AA@ 0042c9dc     sp_char.obj
 0002:000019e8       ??_C@_19GANC@?$AAE?$AAu?$AAm?$AAl?$AA?$AA@ 0042c9e8     sp_char.obj
 0002:000019f4       ??_C@_17CLPM@?$AAE?$AAt?$AAa?$AA?$AA@ 0042c9f4     sp_char.obj
 0002:000019fc       ??_C@_1BA@PL@?$AAE?$AAp?$AAs?$AAi?$AAl?$AAo?$AAn?$AA?$AA@ 0042c9fc     sp_char.obj
 0002:00001a0c       ??_C@_1O@BIBF@?$AAE?$AAg?$AAr?$AAa?$AAv?$AAe?$AA?$AA@ 0042ca0c     sp_char.obj
 0002:00001a1c       ??_C@_1M@CNNH@?$AAE?$AAc?$AAi?$AAr?$AAc?$AA?$AA@ 0042ca1c     sp_char.obj
 0002:00001a28       ??_C@_1O@JCLJ@?$AAE?$AAa?$AAc?$AAu?$AAt?$AAe?$AA?$AA@ 0042ca28     sp_char.obj
 0002:00001a38       ??_C@_17KPCA@?$AAE?$AAT?$AAH?$AA?$AA@ 0042ca38     sp_char.obj
 0002:00001a40       ??_C@_1M@LKNJ@?$AAD?$AAe?$AAl?$AAt?$AAa?$AA?$AA@ 0042ca40     sp_char.obj
 0002:00001a4c       ??_C@_1O@EDPO@?$AAD?$AAa?$AAg?$AAg?$AAe?$AAr?$AA?$AA@ 0042ca4c     sp_char.obj
 0002:00001a5c       ??_C@_17NPNO@?$AAC?$AAh?$AAi?$AA?$AA@ 0042ca5c     sp_char.obj
 0002:00001a64       ??_C@_1O@LNJ@?$AAC?$AAc?$AAe?$AAd?$AAi?$AAl?$AA?$AA@ 0042ca64     sp_char.obj
 0002:00001a74       ??_C@_19OPND@?$AAB?$AAe?$AAt?$AAa?$AA?$AA@ 0042ca74     sp_char.obj
 0002:00001a80       ??_C@_19GJPC@?$AAA?$AAu?$AAm?$AAl?$AA?$AA@ 0042ca80     sp_char.obj
 0002:00001a8c       ??_C@_1O@BIKE@?$AAA?$AAt?$AAi?$AAl?$AAd?$AAe?$AA?$AA@ 0042ca8c     sp_char.obj
 0002:00001a9c       ??_C@_1M@KKJC@?$AAA?$AAr?$AAi?$AAn?$AAg?$AA?$AA@ 0042ca9c     sp_char.obj
 0002:00001aa8       ??_C@_1M@IOCL@?$AAA?$AAl?$AAp?$AAh?$AAa?$AA?$AA@ 0042caa8     sp_char.obj
 0002:00001ab4       ??_C@_1O@FNKC@?$AAA?$AAg?$AAr?$AAa?$AAv?$AAe?$AA?$AA@ 0042cab4     sp_char.obj
 0002:00001ac4       ??_C@_1M@IHOI@?$AAA?$AAc?$AAi?$AAr?$AAc?$AA?$AA@ 0042cac4     sp_char.obj
 0002:00001ad0       ??_C@_1O@NHAO@?$AAA?$AAa?$AAc?$AAu?$AAt?$AAe?$AA?$AA@ 0042cad0     sp_char.obj
 0002:00001ae0       ??_C@_1M@HMNE@?$AAA?$AAE?$AAl?$AAi?$AAg?$AA?$AA@ 0042cae0     sp_char.obj
 0002:00001af0       ?sp_debugger_version@@3QBDB 0042caf0     sp_debugger.obj
 0002:00001f64       ??_C@_1CI@BDFN@?$AAP?$AAU?$AAR?$AAE?$AA_?$AAV?$AAI?$AAR?$AAT?$AA_?$AAF?$AAU?$AAN?$AAC?$AA_?$AAC?$AAA?$AAL?$AAL?$AA?$AA@ 0042cf64     sp_debugger.obj
 0002:00001f8c       ??_C@_1CC@NIIL@?$AAS?$AAY?$AAS?$AAT?$AAE?$AAM?$AA_?$AAE?$AAX?$AAC?$AAE?$AAP?$AAT?$AAI?$AAO?$AAN?$AA?$AA@ 0042cf8c     sp_debugger.obj
 0002:00001fb0       ??_C@_1DA@DMD@?$AAM?$AAI?$AAC?$AAR?$AAO?$AAS?$AAO?$AAF?$AAT?$AA_?$AAC?$AA?$CL?$AA?$CL?$AA_?$AAE?$AAX?$AAC?$AAE?$AAP?$AAT@ 0042cfb0     sp_debugger.obj
 0002:00001fe0       ??_C@_1BO@FNOD@?$AAI?$AAN?$AAV?$AAA?$AAL?$AAI?$AAD?$AA_?$AAT?$AAH?$AAR?$AAE?$AAA?$AAD?$AA?$AA@ 0042cfe0     sp_debugger.obj
 0002:00002000       ??_C@_1DG@LCLP@?$AAI?$AAN?$AAV?$AAA?$AAL?$AAI?$AAD?$AA_?$AAC?$AAR?$AAU?$AAN?$AAT?$AAI?$AAM?$AAE?$AA_?$AAP?$AAA?$AAR@ 0042d000     sp_debugger.obj
 0002:00002038       ??_C@_1CK@IAGC@?$AAS?$AAT?$AAA?$AAC?$AAK?$AA_?$AAB?$AAU?$AAF?$AAF?$AAE?$AAR?$AA_?$AAO?$AAV?$AAE?$AAR?$AAR?$AAU?$AAN@ 0042d038     sp_debugger.obj
 0002:00002064       ??_C@_1CI@DGNG@?$AAR?$AAE?$AAG?$AA_?$AAN?$AAA?$AAT?$AA_?$AAC?$AAO?$AAN?$AAS?$AAU?$AAM?$AAP?$AAT?$AAI?$AAO?$AAN?$AA?$AA@ 0042d064     sp_debugger.obj
 0002:0000208c       ??_C@_1CK@DDIL@?$AAF?$AAL?$AAO?$AAA?$AAT?$AA_?$AAM?$AAU?$AAL?$AAT?$AAI?$AAP?$AAL?$AAE?$AA_?$AAT?$AAR?$AAA?$AAP?$AAS@ 0042d08c     sp_debugger.obj
 0002:000020b8       ??_C@_1CM@OJC@?$AAF?$AAL?$AAO?$AAA?$AAT?$AA_?$AAM?$AAU?$AAL?$AAT?$AAI?$AAP?$AAL?$AAE?$AA_?$AAF?$AAA?$AAU?$AAL?$AAT@ 0042d0b8     sp_debugger.obj
 0002:000020e4       ??_C@_1CA@NHOD@?$AAD?$AAL?$AAL?$AA_?$AAI?$AAN?$AAI?$AAT?$AA_?$AAF?$AAA?$AAI?$AAL?$AAE?$AAD?$AA?$AA@ 0042d0e4     sp_debugger.obj
 0002:00002104       ??_C@_1BO@NOOO@?$AAC?$AAO?$AAN?$AAT?$AAR?$AAO?$AAL?$AA_?$AAC?$AA_?$AAE?$AAX?$AAI?$AAT?$AA?$AA@ 0042d104     sp_debugger.obj
 0002:00002124       ??_C@_1BO@IPPP@?$AAS?$AAT?$AAA?$AAC?$AAK?$AA_?$AAO?$AAV?$AAE?$AAR?$AAF?$AAL?$AAO?$AAW?$AA?$AA@ 0042d124     sp_debugger.obj
 0002:00002144       ??_C@_1CO@IDDA@?$AAP?$AAR?$AAI?$AAV?$AAI?$AAL?$AAE?$AAG?$AAE?$AAD?$AA_?$AAI?$AAN?$AAS?$AAT?$AAR?$AAU?$AAC?$AAT?$AAI@ 0042d144     sp_debugger.obj
 0002:00002174       ??_C@_1CC@MMPM@?$AAI?$AAN?$AAT?$AAE?$AAG?$AAE?$AAR?$AA_?$AAO?$AAV?$AAE?$AAR?$AAF?$AAL?$AAO?$AAW?$AA?$AA@ 0042d174     sp_debugger.obj
 0002:00002198       ??_C@_1CO@KLJC@?$AAI?$AAN?$AAT?$AAE?$AAG?$AAE?$AAR?$AA_?$AAD?$AAI?$AAV?$AAI?$AAD?$AAE?$AA_?$AAB?$AAY?$AA_?$AAZ?$AAE@ 0042d198     sp_debugger.obj
 0002:000021c8       ??_C@_1CA@PDPE@?$AAF?$AAL?$AAO?$AAA?$AAT?$AA_?$AAU?$AAN?$AAD?$AAE?$AAR?$AAF?$AAL?$AAO?$AAW?$AA?$AA@ 0042d1c8     sp_debugger.obj
 0002:000021e8       ??_C@_1CE@DOEH@?$AAF?$AAL?$AAO?$AAA?$AAT?$AA_?$AAS?$AAT?$AAA?$AAC?$AAK?$AA_?$AAC?$AAH?$AAE?$AAC?$AAK?$AA?$AA@ 0042d1e8     sp_debugger.obj
 0002:0000220c       ??_C@_1BO@GFAD@?$AAF?$AAL?$AAO?$AAA?$AAT?$AA_?$AAO?$AAV?$AAE?$AAR?$AAF?$AAL?$AAO?$AAW?$AA?$AA@ 0042d20c     sp_debugger.obj
 0002:0000222c       ??_C@_1DA@BGKB@?$AAF?$AAL?$AAO?$AAA?$AAT?$AA_?$AAI?$AAN?$AAV?$AAA?$AAL?$AAI?$AAD?$AA_?$AAO?$AAP?$AAE?$AAR?$AAA?$AAT@ 0042d22c     sp_debugger.obj
 0002:0000225c       ??_C@_1CK@KHDK@?$AAF?$AAL?$AAO?$AAA?$AAT?$AA_?$AAI?$AAN?$AAE?$AAX?$AAA?$AAC?$AAT?$AA_?$AAR?$AAE?$AAS?$AAU?$AAL?$AAT@ 0042d25c     sp_debugger.obj
 0002:00002288       ??_C@_1CK@JKEP@?$AAF?$AAL?$AAO?$AAA?$AAT?$AA_?$AAD?$AAI?$AAV?$AAI?$AAD?$AAE?$AA_?$AAB?$AAY?$AA_?$AAZ?$AAE?$AAR?$AAO@ 0042d288     sp_debugger.obj
 0002:000022b4       ??_C@_1CO@KIKN@?$AAF?$AAL?$AAO?$AAA?$AAT?$AA_?$AAD?$AAE?$AAN?$AAO?$AAR?$AAM?$AAA?$AAL?$AA_?$AAO?$AAP?$AAE?$AAR?$AAA@ 0042d2b4     sp_debugger.obj
 0002:000022e4       ??_C@_1CM@NHP@?$AAA?$AAR?$AAR?$AAA?$AAY?$AA_?$AAB?$AAO?$AAU?$AAN?$AAD?$AAS?$AA_?$AAE?$AAX?$AAC?$AAE?$AAE?$AAD?$AAE@ 0042d2e4     sp_debugger.obj
 0002:00002310       ??_C@_1CI@OPCO@?$AAI?$AAN?$AAV?$AAA?$AAL?$AAI?$AAD?$AA_?$AAD?$AAI?$AAS?$AAP?$AAO?$AAS?$AAI?$AAT?$AAI?$AAO?$AAN?$AA?$AA@ 0042d310     sp_debugger.obj
 0002:00002338       ??_C@_1DC@EENN@?$AAN?$AAO?$AAN?$AAC?$AAO?$AAN?$AAT?$AAI?$AAN?$AAU?$AAA?$AAB?$AAL?$AAE?$AA_?$AAE?$AAX?$AAC?$AAE?$AAP@ 0042d338     sp_debugger.obj
 0002:0000236c       ??_C@_1CI@KAPO@?$AAI?$AAL?$AAL?$AAE?$AAG?$AAA?$AAL?$AA_?$AAI?$AAN?$AAS?$AAT?$AAR?$AAU?$AAC?$AAT?$AAI?$AAO?$AAN?$AA?$AA@ 0042d36c     sp_debugger.obj
 0002:00002394       ??_C@_1BE@JHOP@?$AAN?$AAO?$AA_?$AAM?$AAE?$AAM?$AAO?$AAR?$AAY?$AA?$AA@ 0042d394     sp_debugger.obj
 0002:000023a8       ??_C@_1CE@HNPJ@?$AAI?$AAN?$AAV?$AAA?$AAL?$AAI?$AAD?$AA_?$AAP?$AAA?$AAR?$AAA?$AAM?$AAE?$AAT?$AAE?$AAR?$AA?$AA@ 0042d3a8     sp_debugger.obj
 0002:000023cc       ??_C@_1BO@FJOO@?$AAI?$AAN?$AAV?$AAA?$AAL?$AAI?$AAD?$AA_?$AAH?$AAA?$AAN?$AAD?$AAL?$AAE?$AA?$AA@ 0042d3cc     sp_debugger.obj
 0002:000023ec       ??_C@_1BM@ECHG@?$AAI?$AAN?$AA_?$AAP?$AAA?$AAG?$AAE?$AA_?$AAE?$AAR?$AAR?$AAO?$AAR?$AA?$AA@ 0042d3ec     sp_debugger.obj
 0002:00002408       ??_C@_1CC@LLKF@?$AAA?$AAC?$AAC?$AAE?$AAS?$AAS?$AA_?$AAV?$AAI?$AAO?$AAL?$AAA?$AAT?$AAI?$AAO?$AAN?$AA?$AA@ 0042d408     sp_debugger.obj
 0002:0000242c       ??_C@_0BE@HOPG@PURE_VIRT_FUNC_CALL?$AA@ 0042d42c     sp_debugger.obj
 0002:00002440       ??_C@_0BB@CMAD@SYSTEM_EXCEPTION?$AA@ 0042d440     sp_debugger.obj
 0002:00002454       ??_C@_0BI@BODF@MICROSOFT_C?$CL?$CL_EXCEPTION?$AA@ 0042d454     sp_debugger.obj
 0002:0000246c       ??_C@_0P@CCJA@INVALID_THREAD?$AA@ 0042d46c     sp_debugger.obj
 0002:0000247c       ??_C@_0BL@IDND@INVALID_CRUNTIME_PARAMETER?$AA@ 0042d47c     sp_debugger.obj
 0002:00002498       ??_C@_0BF@BAKG@STACK_BUFFER_OVERRUN?$AA@ 0042d498     sp_debugger.obj
 0002:000024b0       ??_C@_0BE@DHJH@REG_NAT_CONSUMPTION?$AA@ 0042d4b0     sp_debugger.obj
 0002:000024c4       ??_C@_0BF@FOFC@FLOAT_MULTIPLE_TRAPS?$AA@ 0042d4c4     sp_debugger.obj
 0002:000024dc       ??_C@_0BG@JEJG@FLOAT_MULTIPLE_FAULTS?$AA@ 0042d4dc     sp_debugger.obj
 0002:000024f4       ??_C@_0BA@JAGE@DLL_INIT_FAILED?$AA@ 0042d4f4     sp_debugger.obj
 0002:00002504       ??_C@_0P@MOPO@CONTROL_C_EXIT?$AA@ 0042d504     sp_debugger.obj
 0002:00002514       ??_C@_0P@IPJK@STACK_OVERFLOW?$AA@ 0042d514     sp_debugger.obj
 0002:00002524       ??_C@_0BH@NGJG@PRIVILEGED_INSTRUCTION?$AA@ 0042d524     sp_debugger.obj
 0002:0000253c       ??_C@_0BB@NKJM@INTEGER_OVERFLOW?$AA@ 0042d53c     sp_debugger.obj
 0002:00002550       ??_C@_0BH@JADO@INTEGER_DIVIDE_BY_ZERO?$AA@ 0042d550     sp_debugger.obj
 0002:00002568       ??_C@_0BA@DEJD@FLOAT_UNDERFLOW?$AA@ 0042d568     sp_debugger.obj
 0002:00002578       ??_C@_0BC@IJFD@FLOAT_STACK_CHECK?$AA@ 0042d578     sp_debugger.obj
 0002:0000258c       ??_C@_0P@MNGE@FLOAT_OVERFLOW?$AA@ 0042d58c     sp_debugger.obj
 0002:0000259c       ??_C@_0BI@KC@FLOAT_INVALID_OPERATION?$AA@ 0042d59c     sp_debugger.obj
 0002:000025b4       ??_C@_0BF@CGH@FLOAT_INEXACT_RESULT?$AA@ 0042d5b4     sp_debugger.obj
 0002:000025cc       ??_C@_0BF@MEFK@FLOAT_DIVIDE_BY_ZERO?$AA@ 0042d5cc     sp_debugger.obj
 0002:000025e4       ??_C@_0BH@HKBH@FLOAT_DENORMAL_OPERAND?$AA@ 0042d5e4     sp_debugger.obj
 0002:000025fc       ??_C@_0BG@MPHG@ARRAY_BOUNDS_EXCEEDED?$AA@ 0042d5fc     sp_debugger.obj
 0002:00002614       ??_C@_0BE@DNMD@INVALID_DISPOSITION?$AA@ 0042d614     sp_debugger.obj
 0002:00002628       ??_C@_0BJ@BKEI@NONCONTINUABLE_EXCEPTION?$AA@ 0042d628     sp_debugger.obj
 0002:00002644       ??_C@_0BE@OPNJ@ILLEGAL_INSTRUCTION?$AA@ 0042d644     sp_debugger.obj
 0002:00002658       ??_C@_09BLOO@NO_MEMORY?$AA@ 0042d658     sp_debugger.obj
 0002:00002664       ??_C@_0BC@OBGO@INVALID_PARAMETER?$AA@ 0042d664     sp_debugger.obj
 0002:00002678       ??_C@_0P@MJDA@INVALID_HANDLE?$AA@ 0042d678     sp_debugger.obj
 0002:00002688       ??_C@_0O@JOEG@IN_PAGE_ERROR?$AA@ 0042d688     sp_debugger.obj
 0002:00002698       ??_C@_0BB@EGIM@ACCESS_VIOLATION?$AA@ 0042d698     sp_debugger.obj
 0002:000026ac       ??_C@_05CDDG@?$DMCMP?$DO?$AA@ 0042d6ac     sp_debugger.obj
 0002:000026b4       ??_C@_05OKPP@?$DMRAW?$DO?$AA@ 0042d6b4     sp_debugger.obj
 0002:000026bc       ??_C@_0BI@OCFG@SPDebugger?12?414?419101?4A?$AA@ 0042d6bc     sp_debugger.obj
 0002:000026d4       ??_C@_0FM@PDMN@Uncontinuable?5Exception?5Raised?4?6@ 0042d6d4     sp_debugger.obj
 0002:00002730       ??_C@_03KFLI@SSP?$AA@      0042d730     sp_debugger.obj
 0002:00002734       ??_C@_01LLF@w?$AA@         0042d734     sp_debugger.obj
 0002:00002738       ??_C@_0N@OMCC@STACKTRC?4TXT?$AA@ 0042d738     sp_debugger.obj
 0002:00002754       ??_C@_0BI@CMDD@?6Total?5StackDepth?5?3?5?$CFu?6?$AA@ 0042d754     sp_debugger.obj
 0002:0000276c       ??_C@_0M@NOOL@?5?$CI?$CFs?9?$DO0x?$CFx?$CJ?$AA@ 0042d76c     sp_debugger.obj
 0002:00002778       ??_C@_0CN@BCFA@?$CFu?5?3?5?$CF08x?1?$CF08x?5?$CFs?5?$FL?$CF08x?0?$CF08x?0?$CF08@ 0042d778     sp_debugger.obj
 0002:000027a8       ??_C@_0BD@BGD@?6CallStack?5Trace?3?6?$AA@ 0042d7a8     sp_debugger.obj
 0002:000027bc       ??_C@_0BH@BGAC@SymFunctionTableAccess?$AA@ 0042d7bc     sp_debugger.obj
 0002:000027d4       ??_C@_0O@HGIF@SymSetOptions?$AA@ 0042d7d4     sp_debugger.obj
 0002:000027e4       ??_C@_0BB@PGCD@SymGetModuleBase?$AA@ 0042d7e4     sp_debugger.obj
 0002:000027f8       ??_C@_0BC@JLJA@SymGetSymFromAddr?$AA@ 0042d7f8     sp_debugger.obj
 0002:0000280c       ??_C@_0L@CPNA@SymCleanup?$AA@ 0042d80c     sp_debugger.obj
 0002:00002818       ??_C@_0O@FCHA@SymInitialize?$AA@ 0042d818     sp_debugger.obj
 0002:00002828       ??_C@_09CJDB@StackWalk?$AA@ 0042d828     sp_debugger.obj
 0002:00002834       ??_C@_08GDHI@imagehlp?$AA@ 0042d834     sp_debugger.obj
 0002:00002840       ??_C@_0CJ@IBOE@?$CF08x?5?$CF08x?5?$CF08x?5?$CF08x?5?$CF08x?5?$CF08x?5?$CF0@ 0042d840     sp_debugger.obj
 0002:0000286c       ??_C@_0P@GOE@?6Stack?5Dump?3?5?6?$AA@ 0042d86c     sp_debugger.obj
 0002:0000287c       ??_C@_0BC@DOLJ@EFlags?5?$CF08x?5?$CI?$CFs?$CJ?6?$AA@ 0042d87c     sp_debugger.obj
 0002:00002890       ??_C@_0CM@BNBI@SS?1ESP?1EBP?5?$CF04x?1?$CF08x?1?$CF08x?5CS?1EIP@ 0042d890     sp_debugger.obj
 0002:000028bc       ??_C@_0CD@HGPK@DS?1ESI?5?$CF04x?1?$CF08x?5ES?1EDI?5?$CF04x?1?$CF08@ 0042d8bc     sp_debugger.obj
 0002:000028e0       ??_C@_0CF@NFIJ@EAX?5?$CF08x?5EBX?5?$CF08x?5ECX?5?$CF08x?5EDX?5?$CF@ 0042d8e0     sp_debugger.obj
 0002:00002908       ??_C@_0O@CPED@?6Registers?3?5?6?$AA@ 0042d908     sp_debugger.obj
 0002:00002918       ??_C@_0BH@IHNO@?5?5?9?$DOReading?5?$CF08x?5Data?6?$AA@ 0042d918     sp_debugger.obj
 0002:00002930       ??_C@_0BH@GPBD@?5?5?9?$DOWriting?5?$CF08x?5Data?6?$AA@ 0042d930     sp_debugger.obj
 0002:00002948       ??_C@_0CN@BLIG@Exception?5Raised?5at?5?$CF08x?5because@ 0042d948     sp_debugger.obj
 0002:00002978       ??_C@_01BJG@?6?$AA@        0042d978     sp_debugger.obj
 0002:0000297c       ??_C@_0BB@MJPL@SeDebugPrivilege?$AA@ 0042d97c     sp_debugger.obj
 0002:00002990       ??_C@_0BD@GNGB@?6Loaded?5Modules?3?5?6?$AA@ 0042d990     sp_debugger.obj
 0002:000029a4       ??_C@_0BH@OABE@?6Executing?5Services?3?5?6?$AA@ 0042d9a4     sp_debugger.obj
 0002:000029bc       ??_C@_0BI@PPDH@?6Executing?5Processes?3?5?6?$AA@ 0042d9bc     sp_debugger.obj
 0002:000029d4       ??_C@_04GPCF@?5?5?5?5?$AA@ 0042d9d4     sp_debugger.obj
 0002:000029dc       ??_C@_0BD@IGMP@?6Env?4?5Variables?3?5?6?$AA@ 0042d9dc     sp_debugger.obj
 0002:000029f0       ??_C@_0BI@PKEG@?6Monitor?5Information?3?5?6?$AA@ 0042d9f0     sp_debugger.obj
 0002:00002a08       ??_C@_0BE@KPOG@EnumDisplayMonitors?$AA@ 0042da08     sp_debugger.obj
 0002:00002a1c       ??_C@_0BA@LJCP@GetMonitorInfoA?$AA@ 0042da1c     sp_debugger.obj
 0002:00002a2c       ??_C@_06IMLE@user32?$AA@   0042da2c     sp_debugger.obj
 0002:00002a34       ??_C@_08MMGE@Unknown?6?$AA@ 0042da34     sp_debugger.obj
 0002:00002a40       ??_C@_08DBCB@RAMDISK?6?$AA@ 0042da40     sp_debugger.obj
 0002:00002a4c       ??_C@_07HPHG@CD?9ROM?6?$AA@ 0042da4c     sp_debugger.obj
 0002:00002a54       ??_C@_08DKOM@Network?6?$AA@ 0042da54     sp_debugger.obj
 0002:00002a60       ??_C@_0L@CBNM@Removable?6?$AA@ 0042da60     sp_debugger.obj
 0002:00002a6c       ??_C@_0CM@HCBD@?5?5?$FL?$CF8uMB?5Free?5?$HM?$CF8uMB?5Total?5?$HM?$CF3u?$CF@ 0042da6c     sp_debugger.obj
 0002:00002a98       ??_C@_05CAKF@Fixed?$AA@    0042da98     sp_debugger.obj
 0002:00002aa0       ??_C@_09GJBB@?5?5?5?5?$CF?94s?5?$AA@ 0042daa0     sp_debugger.obj
 0002:00002aac       ??_C@_04NNOD@ZF?3?2?$AA@   0042daac     sp_debugger.obj
 0002:00002ab4       ??_C@_04CLNI@ZE?3?2?$AA@   0042dab4     sp_debugger.obj
 0002:00002abc       ??_C@_04HJMO@ZD?3?2?$AA@   0042dabc     sp_debugger.obj
 0002:00002ac4       ??_C@_04MHKP@ZC?3?2?$AA@   0042dac4     sp_debugger.obj
 0002:00002acc       ??_C@_04JFLJ@ZB?3?2?$AA@   0042dacc     sp_debugger.obj
 0002:00002ad4       ??_C@_04GDIC@ZA?3?2?$AA@   0042dad4     sp_debugger.obj
 0002:00002adc       ??_C@_03EFPG@Z?3?2?$AA@    0042dadc     sp_debugger.obj
 0002:00002ae0       ??_C@_03LDMN@Y?3?2?$AA@    0042dae0     sp_debugger.obj
 0002:00002ae4       ??_C@_03OBNL@X?3?2?$AA@    0042dae4     sp_debugger.obj
 0002:00002ae8       ??_C@_03MPAP@W?3?2?$AA@    0042dae8     sp_debugger.obj
 0002:00002aec       ??_C@_03JNBJ@V?3?2?$AA@    0042daec     sp_debugger.obj
 0002:00002af0       ??_C@_03GLCC@U?3?2?$AA@    0042daf0     sp_debugger.obj
 0002:00002af4       ??_C@_03DJDE@T?3?2?$AA@    0042daf4     sp_debugger.obj
 0002:00002af8       ??_C@_03IHFF@S?3?2?$AA@    0042daf8     sp_debugger.obj
 0002:00002afc       ??_C@_03NFED@R?3?2?$AA@    0042dafc     sp_debugger.obj
 0002:00002b00       ??_C@_03CDHI@Q?3?2?$AA@    0042db00     sp_debugger.obj
 0002:00002b04       ??_C@_03HBGO@P?3?2?$AA@    0042db04     sp_debugger.obj
 0002:00002b08       ??_C@_03HONA@O?3?2?$AA@    0042db08     sp_debugger.obj
 0002:00002b0c       ??_C@_03CMMG@N?3?2?$AA@    0042db0c     sp_debugger.obj
 0002:00002b10       ??_C@_03NKPN@M?3?2?$AA@    0042db10     sp_debugger.obj
 0002:00002b14       ??_C@_03IIOL@L?3?2?$AA@    0042db14     sp_debugger.obj
 0002:00002b18       ??_C@_03DGIK@K?3?2?$AA@    0042db18     sp_debugger.obj
 0002:00002b1c       ??_C@_03GEJM@J?3?2?$AA@    0042db1c     sp_debugger.obj
 0002:00002b20       ??_C@_03JCKH@I?3?2?$AA@    0042db20     sp_debugger.obj
 0002:00002b24       ??_C@_03MALB@H?3?2?$AA@    0042db24     sp_debugger.obj
 0002:00002b28       ??_C@_03OOGF@G?3?2?$AA@    0042db28     sp_debugger.obj
 0002:00002b2c       ??_C@_03LMHD@F?3?2?$AA@    0042db2c     sp_debugger.obj
 0002:00002b30       ??_C@_03EKEI@E?3?2?$AA@    0042db30     sp_debugger.obj
 0002:00002b34       ??_C@_03BIFO@D?3?2?$AA@    0042db34     sp_debugger.obj
 0002:00002b38       ??_C@_03KGDP@C?3?2?$AA@    0042db38     sp_debugger.obj
 0002:00002b3c       ??_C@_03PECJ@B?3?2?$AA@    0042db3c     sp_debugger.obj
 0002:00002b40       ??_C@_03CBC@A?3?2?$AA@     0042db40     sp_debugger.obj
 0002:00002b44       ??_C@_0BH@NNLG@?6Volume?5Information?3?5?6?$AA@ 0042db44     sp_debugger.obj
 0002:00002b5c       ??_C@_05MA@?5x?5?$CFu?$AA@ 0042db5c     sp_debugger.obj
 0002:00002b64       ??_C@_01KMMP@?$CJ?$AA@     0042db64     sp_debugger.obj
 0002:00002b68       ??_C@_01GFI@?$CI?$AA@      0042db68     sp_debugger.obj
 0002:00002b6c       ??_C@_09OKBO@?5Support?5?$AA@ 0042db6c     sp_debugger.obj
 0002:00002b78       ??_C@_07LBPC@?5HT?$CI?$CFu?$CJ?$AA@ 0042db78     sp_debugger.obj
 0002:00002b80       ??_C@_04KOOI@?5MMX?$AA@    0042db80     sp_debugger.obj
 0002:00002b88       ??_C@_04LIOI@with?$AA@     0042db88     sp_debugger.obj
 0002:00002b90       ??_C@_0BD@FFAP@CPU?5?3?5?$CFs?5?$CFs?5?$CFuMHz?5?$AA@ 0042db90     sp_debugger.obj
 0002:00002ba4       ??_C@_0CG@HADA@Phys?4Mem?3?5?$CFu?1?$CFuMB?5?5PageFile?3?5?$CFu?1@ 0042dba4     sp_debugger.obj
 0002:00002bcc       ??_C@_0CE@HGLP@Time?3?5?$CFu?1?$CFu?1?$CFu?5?$CF02u?3?$CF02u?3?$CF02u?4?$CF0@ 0042dbcc     sp_debugger.obj
 0002:00002bf0       ??_C@_0L@OCA@UAC?3?5?$CFs?$CFs?6?$AA@ 0042dbf0     sp_debugger.obj
 0002:00002bfc       ??_C@_08FGLH@Disabled?$AA@ 0042dbfc     sp_debugger.obj
 0002:00002c08       ??_C@_07FFME@Enabled?$AA@  0042dc08     sp_debugger.obj
 0002:00002c10       ??_C@_08PGIG@?0Limited?$AA@ 0042dc10     sp_debugger.obj
 0002:00002c1c       ??_C@_09EDHK@?0Elevated?$AA@ 0042dc1c     sp_debugger.obj
 0002:00002c28       ??_C@_0BC@KFFJ@?$CFs?$CFs?5?$CFu?4?$CFu?4?$CFu?5?$CFs?6?$AA@ 0042dc28     sp_debugger.obj
 0002:00002c3c       ??_C@_01FAFK@?$DO?$AA@     0042dc3c     sp_debugger.obj
 0002:00002c40       ??_C@_01FHE@?$DM?$AA@      0042dc40     sp_debugger.obj
 0002:00002c44       ??_C@_05LNCF@?$EAWine?$AA@ 0042dc44     sp_debugger.obj
 0002:00002c4c       ??_C@_0L@CEIK@Windows?5NT?$AA@ 0042dc4c     sp_debugger.obj
 0002:00002c58       ??_C@_0O@JFCM@Windows?59x?1Me?$AA@ 0042dc58     sp_debugger.obj
 0002:00002c68       ??_C@_06BILL@Normal?$AA@   0042dc68     sp_debugger.obj
 0002:00002c70       ??_C@_0L@GFMG@Compressed?$AA@ 0042dc70     sp_debugger.obj
 0002:00002c7c       ??_C@_0BE@ONFO@GetDiskFreeSpaceExA?$AA@ 0042dc7c     sp_debugger.obj
 0002:00002c90       ??_C@_0CN@LBHJ@?5?5?5?5?$CFd?3?5?$CFs?5?9?5Work?$DN?$CFd?0?$CFd?0?$CFd?0?$CFd?5Si@ 0042dc90     sp_debugger.obj
 0002:00002cc0       ??_C@_09EICI@?$FLPRIMARY?$FN?$AA@ 0042dcc0     sp_debugger.obj
 0002:00002ccc       ??_C@_0BH@JIPE@UNKNOWN_EXCEPTION_?$CF08x?$AA@ 0042dccc     sp_debugger.obj
 0002:00002ce4       ??_C@_0N@GIMK@?5?5?5?5?9?$CF08x?5?3?5?$AA@ 0042dce4     sp_debugger.obj
 0002:00002cf4       ??_C@_0BA@BPAP@?$FLSystem?5Device?$FN?$AA@ 0042dcf4     sp_debugger.obj
 0002:00002d04       ??_C@_0BD@GBEK@?6Loaded?5Drivers?3?5?6?$AA@ 0042dd04     sp_debugger.obj
 0002:00002d18       ??_C@_0BJ@BBGB@GetDeviceDriverBaseNameA?$AA@ 0042dd18     sp_debugger.obj
 0002:00002d34       ??_C@_0BC@IHKN@EnumDeviceDrivers?$AA@ 0042dd34     sp_debugger.obj
 0002:00002d48       ??_C@_05ECID@psapi?$AA@    0042dd48     sp_debugger.obj
 0002:00002d50       ??_C@_0EB@OIFF@?5?5?5?5?5?5?5?5?5?5?5?5?5?5?5?5?5?5?5?5?5?5?$CFu?4?$CFu?4?$CFu?4?$CF@ 0042dd50     sp_debugger.obj
 0002:00002d94       ??_C@_0BA@EJP@FileDescription?$AA@ 0042dd94     sp_debugger.obj
 0002:00002da4       ??_C@_0P@NIMM@LegalCopyright?$AA@ 0042dda4     sp_debugger.obj
 0002:00002db4       ??_C@_0P@LDLH@?9?$CF08x?5?$CFs?5?3?5?$CFs?6?$AA@ 0042ddb4     sp_debugger.obj
 0002:00002dc4       ??_C@_04KDBP@?$DN?$DN?$DO?5?$AA@ 0042ddc4     sp_debugger.obj
 0002:00002dcc       ??_C@_0BD@GIDO@?$FLWith?5ToolHelp32?$FN?6?$AA@ 0042ddcc     sp_debugger.obj
 0002:00002de0       ??_C@_0BE@PEJL@?5?5?5?5?$CFs?$CFs?5?$CI?$CFs?$CJ?5?9?5?$CFs?6?$AA@ 0042dde0     sp_debugger.obj
 0002:00002df4       ??_C@_03OCLJ@?9?9?9?$AA@   0042ddf4     sp_debugger.obj
 0002:00002df8       ??_C@_03GIGI@?$CK?$CK?$CK?$AA@ 0042ddf8     sp_debugger.obj
 0002:00002dfc       ??_C@_0P@HIPL@Stopped?1Paused?$AA@ 0042ddfc     sp_debugger.obj
 0002:00002e0c       ??_C@_07IJMD@Running?$AA@  0042de0c     sp_debugger.obj
 0002:00002e14       ??_C@_0P@JDMN@?$FLWith?5SCM?1NT?$FN?6?$AA@ 0042de14     sp_debugger.obj
 0002:00002e24       ??_C@_0BE@OFLL@EnumServicesStatusA?$AA@ 0042de24     sp_debugger.obj
 0002:00002e38       ??_C@_0BD@POGC@CloseServiceHandle?$AA@ 0042de38     sp_debugger.obj
 0002:00002e4c       ??_C@_0P@KPLF@OpenSCManagerA?$AA@ 0042de4c     sp_debugger.obj
 0002:00002e5c       ??_C@_0DF@DELJ@?5?5?5?5?5?5?5?5?5?5?5?5?5?5?5?5?$CFu?4?$CFu?4?$CFu?4?$CFu?5?9?5?$CFs@ 0042de5c     sp_debugger.obj
 0002:00002e94       ??_C@_0BA@ILM@?5?$CI?$CFd?5Threads?4?$CJ?6?$AA@ 0042de94     sp_debugger.obj
 0002:00002ea4       ??_C@_08DFCP@?9?$CF08x?5?3?5?$AA@ 0042dea4     sp_debugger.obj
 0002:00002eb0       ??_C@_08LKDA@IOPL?5HI?0?$AA@ 0042deb0     sp_debugger.obj
 0002:00002ebc       ??_C@_08IFJF@IOPL?5LO?0?$AA@ 0042debc     sp_debugger.obj
 0002:00002ec8       ??_C@_03BLAC@ID?0?$AA@     0042dec8     sp_debugger.obj
 0002:00002ecc       ??_C@_0N@GGHH@VIntPending?0?$AA@ 0042decc     sp_debugger.obj
 0002:00002edc       ??_C@_0M@ICBN@VInterrupt?0?$AA@ 0042dedc     sp_debugger.obj
 0002:00002ee8       ??_C@_0L@DABO@Alignment?0?$AA@ 0042dee8     sp_debugger.obj
 0002:00002ef4       ??_C@_06CAHH@V8086?0?$AA@  0042def4     sp_debugger.obj
 0002:00002efc       ??_C@_08DHIC@Restart?0?$AA@ 0042defc     sp_debugger.obj
 0002:00002f08       ??_C@_05HFKC@Nest?0?$AA@   0042df08     sp_debugger.obj
 0002:00002f10       ??_C@_09EKL@OverFlow?0?$AA@ 0042df10     sp_debugger.obj
 0002:00002f1c       ??_C@_0L@NPGF@Direction?0?$AA@ 0042df1c     sp_debugger.obj
 0002:00002f28       ??_C@_0L@PGDB@Interrupt?0?$AA@ 0042df28     sp_debugger.obj
 0002:00002f34       ??_C@_05EGOF@Trap?0?$AA@   0042df34     sp_debugger.obj
 0002:00002f3c       ??_C@_05HCCN@Sign?0?$AA@   0042df3c     sp_debugger.obj
 0002:00002f44       ??_C@_05EBHG@Zero?0?$AA@   0042df44     sp_debugger.obj
 0002:00002f4c       ??_C@_07KFMM@Adjust?0?$AA@ 0042df4c     sp_debugger.obj
 0002:00002f54       ??_C@_07PJA@Parity?0?$AA@  0042df54     sp_debugger.obj
 0002:00002f5c       ??_C@_06MCOM@Carry?0?$AA@  0042df5c     sp_debugger.obj
 0002:00002f64       ??_C@_0BB@IBEB@FindFirstFileExA?$AA@ 0042df64     sp_findfile.obj
 0002:00002f78       ??_C@_02OOND@?4?4?$AA@     0042df78     sp_findfile.obj
 0002:00002f7c       ??_C@_01PJCK@?4?$AA@       0042df7c     sp_findfile.obj
 0002:00002f80       ??_C@_03FANE@zip?$AA@      0042df80     sp_kei.obj
 0002:00002f84       ??_C@_03IKNC@exe?$AA@      0042df84     sp_kei.obj
 0002:00002f88       ??_C@_04OPJK@name?$AA@     0042df88     sp_kei.obj
 0002:00002f90       ??_7SPModule@@6BJLockable@@@ 0042df90     sp_module.obj
 0002:00002fa4       ??_7SPModule@@6BSPProp@@@  0042dfa4     sp_module.obj
 0002:00002fdc       ??_7JMutex@@6B@            0042dfdc     sp_module.obj
 0002:00002ff0       ??_7SPProp@@6B@            0042dff0     sp_module.obj
 0002:00003018       ??_C@_19EMCC@?$AAm?$AAa?$AAi?$AAn?$AA?$AA@ 0042e018     sp_module.obj
 0002:00003024       ??_C@_11A@?$AA?$AA@        0042e024     sp_module.obj
 0002:00003028       ??_7SPVarSystemNode@@6B@   0042e028     sp_module.obj
 0002:00003034       ??_C@_04EHIG@ansi?$AA@     0042e034     sp_module.obj
 0002:0000303c       ??_C@_08IMGJ@charmode?$AA@ 0042e03c     sp_module.obj
 0002:00003048       ??_C@_0M@OHDE@commandline?$AA@ 0042e048     sp_module.obj
 0002:00003054       ??_C@_0BA@EEEA@GetProcessHeaps?$AA@ 0042e054     sp_module.obj
 0002:00003064       ??_C@_0N@JNFD@shiolink?4dll?$AA@ 0042e064     sp_module.obj
 0002:00003074       ??_C@_04NFOM@?4exe?$AA@    0042e074     sp_module.obj
 0002:0000307c       ??_C@_0P@GBBM@?$CIfree?5library?$CJ?$AA@ 0042e07c     sp_module.obj
 0002:0000308c       ??_C@_0O@FJGM@?$CIunload?5call?$CJ?$AA@ 0042e08c     sp_module.obj
 0002:0000309c       ??_C@_1BC@EJBN@?$AA?$CF?$AAs?$AA?$CI?$AAl?$AAo?$AAa?$AAd?$AA?$CJ?$AA?$AA@ 0042e09c     sp_module.obj
 0002:000030bc       ??_C@_04JMJF@load?$AA@     0042e0bc     sp_module.obj
 0002:000030c4       ??_C@_04FGNA@?$AN?6?$AN?6?$AA@ 0042e0c4     sp_module.obj
 0002:000030cc       ??_C@_19CIAI@?$AAl?$AAo?$AAa?$AAd?$AA?$AA@ 0042e0cc     sp_module.obj
 0002:000030d8       ??_C@_1BG@ICPD@?$AA?$CF?$AAs?$AA?$CI?$AAu?$AAn?$AAl?$AAo?$AAa?$AAd?$AA?$CJ?$AA?$AA@ 0042e0d8     sp_module.obj
 0002:000030fc       ??_C@_06BFLB@unload?$AA@   0042e0fc     sp_module.obj
 0002:00003104       ??_C@_02PIMC@?$AN?6?$AA@   0042e104     sp_module.obj
 0002:00003108       ??_C@_1O@IFJN@?$AAu?$AAn?$AAl?$AAo?$AAa?$AAd?$AA?$AA@ 0042e108     sp_module.obj
 0002:00003118       ??_C@_1BI@ECIG@?$AA?$CF?$AAs?$AA?$CI?$AAr?$AAe?$AAq?$AAu?$AAe?$AAs?$AAt?$AA?$CJ?$AA?$AA@ 0042e118     sp_module.obj
 0002:0000313c       ??_C@_07GPGM@request?$AA@  0042e13c     sp_module.obj
 0002:00003144       ??_C@_1BA@BHEN@?$AAr?$AAe?$AAq?$AAu?$AAe?$AAs?$AAt?$AA?$AA@ 0042e144     sp_module.obj
 0002:00003154       ??_C@_1BA@HCKD@?$AA?$CF?$AAs?$AA?$CI?$AAg?$AAe?$AAt?$AA?$CJ?$AA?$AA@ 0042e154     sp_module.obj
 0002:00003174       ??_C@_17LBPE@?$AAa?$AAn?$AAy?$AA?$AA@ 0042e174     sp_module.obj
 0002:0000317c       ??_C@_13FCBG@?$AA?$AB?$AA?$AA@ 0042e17c     sp_module.obj
 0002:00003180       ??_C@_08FPJN@_request?$AA@ 0042e180     sp_module.obj
 0002:0000318c       ??_C@_0M@MOOM@_getversion?$AA@ 0042e18c     sp_module.obj
 0002:00003198       ??_C@_07OEMG@_unload?$AA@  0042e198     sp_module.obj
 0002:000031a0       ??_C@_07NHHK@_loadex?$AA@  0042e1a0     sp_module.obj
 0002:000031a8       ??_C@_05PGEE@_load?$AA@    0042e1a8     sp_module.obj
 0002:000031cc       ??_C@_0P@MMPA@RequestCharset?$AA@ 0042e1cc     sp_module.obj
 0002:000031dc       ??_C@_07DMJG@Charset?$AA@  0042e1dc     sp_module.obj
 0002:000031e4       ??_C@_01PKAG@?3?$AA@       0042e1e4     sp_module.obj
 0002:000031e8       ??_C@_03HHLI@?$CKS?3?$AA@  0042e1e8     sp_module.obj
 0002:000031ec       ??_C@_05FLJB@?$CKU?3?$AN?6?$AA@ 0042e1ec     sp_module.obj
 0002:000031f4       ??_C@_03MJBA@?$CKL?3?$AA@  0042e1f4     sp_module.obj
 0002:000031f8       ??_C@_07OOCC@charset?$AA@  0042e1f8     sp_param.obj
 0002:00003200       __real@8@4002a000000000000000 0042e200     sp_param.obj
 0002:00003208       ??_C@_1BO@MCG@?$AAf?$AAi?$AAr?$AAs?$AAt?$AAb?$AAo?$AAo?$AAt?$AA_?$AAt?$AAi?$AAm?$AAe?$AA?$AA@ 0042e208     sp_prop.obj
 0002:00003228       ??_C@_1BM@DNEP@?$AAl?$AAa?$AAs?$AAt?$AAb?$AAo?$AAo?$AAt?$AA_?$AAt?$AAi?$AAm?$AAe?$AA?$AA@ 0042e228     sp_prop.obj
 0002:00003244       ??_C@_1BK@DGIF@?$AAi?$AAn?$AAs?$AAt?$AAa?$AAl?$AAl?$AA_?$AAt?$AAi?$AAm?$AAe?$AA?$AA@ 0042e244     sp_prop.obj
 0002:00003260       ??_C@_1BI@LAIK@?$AA0?$AA?0?$AA0?$AA?0?$AA0?$AA?0?$AA0?$AA?0?$AA0?$AA?0?$AA0?$AA?$AA@ 0042e260     sp_prop.obj
 0002:00003278       ??_C@_1BI@FJOI@?$AAu?$AAp?$AAd?$AAa?$AAt?$AAe?$AA_?$AAt?$AAi?$AAm?$AAe?$AA?$AA@ 0042e278     sp_prop.obj
 0002:00003290       ??_C@_1BM@DMG@?$AAu?$AAp?$AAd?$AAa?$AAt?$AAe?$AA_?$AAr?$AAe?$AAs?$AAu?$AAl?$AAt?$AA?$AA@ 0042e290     sp_prop.obj
 0002:000032ac       ??_C@_1BE@NAF@?$AAt?$AAh?$AAu?$AAm?$AAb?$AAn?$AAa?$AAi?$AAl?$AA?$AA@ 0042e2ac     sp_prop.obj
 0002:000032c0       ??_C@_1M@JOGC@?$AAi?$AAn?$AAd?$AAe?$AAx?$AA?$AA@ 0042e2c0     sp_prop.obj
 0002:000032cc       ??_C@_1BA@OCB@?$AAh?$AAo?$AAm?$AAe?$AAu?$AAr?$AAl?$AA?$AA@ 0042e2cc     sp_prop.obj
 0002:000032dc       ??_C@_1BE@FCG@?$AAu?$AAp?$AAd?$AAa?$AAt?$AAe?$AAu?$AAr?$AAl?$AA?$AA@ 0042e2dc     sp_prop.obj
 0002:000032f0       ??_C@_1BI@KLFP@?$AAc?$AAr?$AAa?$AAf?$AAt?$AAm?$AAa?$AAn?$AAu?$AAr?$AAl?$AA?$AA@ 0042e2f0     sp_prop.obj
 0002:00003308       ??_C@_19HODB@?$AAp?$AAa?$AAt?$AAh?$AA?$AA@ 0042e308     sp_prop.obj
 0002:00003314       ??_C@_1BE@PDCF@?$AAc?$AAr?$AAa?$AAf?$AAt?$AAm?$AAa?$AAn?$AAw?$AA?$AA@ 0042e314     sp_prop.obj
 0002:00003328       ??_C@_1BC@BOIL@?$AAc?$AAr?$AAa?$AAf?$AAt?$AAm?$AAa?$AAn?$AA?$AA@ 0042e328     sp_prop.obj
 0002:0000333c       ??_C@_19OMOB@?$AAn?$AAa?$AAm?$AAe?$AA?$AA@ 0042e33c     sp_prop.obj
 0002:00003348       ??_C@_09DACI@updateurl?$AA@ 0042e348     sp_prop.obj
 0002:00003354       ??_C@_06KFPJ@readme?$AA@   0042e354     sp_prop.obj
 0002:0000335c       ??_C@_07DFDC@homeurl?$AA@  0042e35c     sp_prop.obj
 0002:00003364       ??_C@_0M@HMDP@craftmanurl?$AA@ 0042e364     sp_prop.obj
 0002:00003370       ??_C@_09LBGC@craftmanw?$AA@ 0042e370     sp_prop.obj
 0002:0000337c       ??_C@_08NHLK@craftman?$AA@ 0042e37c     sp_prop.obj
 0002:00003388       ??_C@_0P@IODI@cache_filetime?$AA@ 0042e388     sp_prop.obj
 0002:00003398       ??_C@_0L@LBNG@cache_desc?$AA@ 0042e398     sp_prop.obj
 0002:000033a4       ??_C@_04NCOD@path?$AA@     0042e3a4     sp_prop.obj
 0002:000033ac       ??_C@_1BA@KIJH@?$AAr?$AAe?$AAa?$AAd?$AAn?$AAe?$AA?0?$AA?$AA@ 0042e3ac     sp_prop.obj
 0002:000033bc       ??_C@_1M@OANG@?$AAn?$AAa?$AAm?$AAe?$AA?0?$AA?$AA@ 0042e3bc     sp_prop.obj
 0002:000033c8       ??_C@_1BC@DDMD@?$AAh?$AAo?$AAm?$AAe?$AAu?$AAr?$AAl?$AA?0?$AA?$AA@ 0042e3c8     sp_prop.obj
 0002:000033dc       ??_C@_1BK@JOF@?$AAc?$AAr?$AAa?$AAf?$AAt?$AAm?$AAa?$AAn?$AAu?$AAr?$AAl?$AA?0?$AA?$AA@ 0042e3dc     sp_prop.obj
 0002:000033f8       ??_C@_1BG@DCAM@?$AAc?$AAr?$AAa?$AAf?$AAt?$AAm?$AAa?$AAn?$AAw?$AA?0?$AA?$AA@ 0042e3f8     sp_prop.obj
 0002:00003410       ??_C@_1CC@LFOC@?$AA?$CK?$AAc?$AAa?$AAc?$AAh?$AAe?$AA_?$AAf?$AAi?$AAl?$AAe?$AAt?$AAi?$AAm?$AAe?$AA?0?$AA?$AA@ 0042e410     sp_prop.obj
 0002:00003434       ??_C@_1BK@EEDI@?$AA?$CK?$AAc?$AAa?$AAc?$AAh?$AAe?$AA_?$AAd?$AAe?$AAs?$AAc?$AA?0?$AA?$AA@ 0042e434     sp_prop.obj
 0002:00003450       ??_C@_15BFAC@?$AA?$AN?$AA?6?$AA?$AA@ 0042e450     sp_prop.obj
 0002:00003458       ??_C@_1O@PFIF@?$AA?$CK?$AAp?$AAa?$AAt?$AAh?$AA?0?$AA?$AA@ 0042e458     sp_prop.obj
 0002:00003468       ??_C@_0O@DJDH@ghost?2master?2?$AA@ 0042e468     sp_prop.obj
 0002:00003478       ??_C@_0M@LIC@updates?4txt?$AA@ 0042e478     sp_prop.obj
 0002:00003484       ??_C@_0N@GBMG@updates2?4dau?$AA@ 0042e484     sp_prop.obj
 0002:00003494       ??_C@_0N@LFHM@?4svn?2entries?$AA@ 0042e494     sp_prop.obj
 0002:000034a4       ??_C@_0L@EJFJ@?4svn?2wc?4db?$AA@ 0042e4a4     sp_prop.obj
 0002:000034b0       ??_C@_09FPP@?4git?2HEAD?$AA@ 0042e4b0     sp_prop.obj
 0002:000034bc       ??_C@_0BA@ENJE@?4git?2FETCH_HEAD?$AA@ 0042e4bc     sp_prop.obj
 0002:000034cc       ??_C@_07BMPC@profile?$AA@  0042e4cc     sp_prop.obj
 0002:00003534       ??_C@_13GDLP@?$AA0?$AA?$AA@ 0042e534     sp_setting.obj
 0002:00003658       ??_C@_0L@DLMJ@SHIORI?4DLL?$AA@ 0042e658     sp_shiori.obj
 0002:00003664       ??_C@_09OIOB@TOURI?4DLL?$AA@ 0042e664     sp_shiori.obj
 0002:00003670       ??_C@_09GIPI@HISUI?4DLL?$AA@ 0042e670     sp_shiori.obj
 0002:0000367c       ??_C@_09MLJF@YUHNA?4DLL?$AA@ 0042e67c     sp_shiori.obj
 0002:00003688       ??_C@_0P@JMPC@NISESHIORI?4DLL?$AA@ 0042e688     sp_shiori.obj
 0002:00003698       ??_C@_0L@PIKD@MISAKA?4DLL?$AA@ 0042e698     sp_shiori.obj
 0002:000036a4       ??_C@_0L@IJFM@KAWARI?4DLL?$AA@ 0042e6a4     sp_shiori.obj
 0002:000036b0       ??_C@_07KEJH@AYA?4DLL?$AA@ 0042e6b0     sp_shiori.obj
 0002:000036b8       ??_C@_08CNG@AYA5?4DLL?$AA@ 0042e6b8     sp_shiori.obj
 0002:000036c4       ??_C@_08CEIB@YAYA?4DLL?$AA@ 0042e6c4     sp_shiori.obj
 0002:000036d0       ??_C@_0L@EAMJ@SATORI?4DLL?$AA@ 0042e6d0     sp_shiori.obj
 0002:000036dc       ??_7SPShiori@@6BJLockable@@@ 0042e6dc     sp_shiori.obj
 0002:000036f0       ??_7SPShiori@@6BSPProp@@@  0042e6f0     sp_shiori.obj
 0002:00003728       ??_C@_17HACC@?$AAS?$AAS?$AAP?$AA?$AA@ 0042e728     sp_shiori.obj
 0002:00003730       ??_C@_1O@BPPB@?$AAS?$AAH?$AAI?$AAO?$AAR?$AAI?$AA?$AA@ 0042e730     sp_shiori.obj
 0002:00003740       ??_C@_0BD@DGFL@ssp_shiori_log?4txt?$AA@ 0042e740     sp_shiori.obj
 0002:00003754       ??_C@_1BM@DGMA@?$AAR?$AAe?$AAf?$AAe?$AAr?$AAe?$AAn?$AAc?$AAe?$AA?$CF?$AAd?$AA?3?$AA?5?$AA?$AA@ 0042e754     sp_shiori.obj
 0002:00003770       ??_C@_08DELN@BaseID?3?5?$AA@ 0042e770     sp_shiori.obj
 0002:0000377c       ??_C@_19FIHG@?$AAI?$AAD?$AA?3?$AA?5?$AA?$AA@ 0042e77c     sp_shiori.obj
 0002:00003788       ??_C@_1BG@BLOE@?$AAe?$AAx?$AAt?$AAe?$AAr?$AAn?$AAa?$AAl?$AA?$AN?$AA?6?$AA?$AA@ 0042e788     sp_shiori.obj
 0002:000037a0       ??_C@_1BA@NAMP@?$AAl?$AAo?$AAc?$AAa?$AAl?$AA?$AN?$AA?6?$AA?$AA@ 0042e7a0     sp_shiori.obj
 0002:000037b0       ??_C@_1CA@FGEC@?$AAS?$AAe?$AAc?$AAu?$AAr?$AAi?$AAt?$AAy?$AAL?$AAe?$AAv?$AAe?$AAl?$AA?3?$AA?5?$AA?$AA@ 0042e7b0     sp_shiori.obj
 0002:000037d0       ??_C@_1BC@PGED@?$AAS?$AAe?$AAn?$AAd?$AAe?$AAr?$AA?3?$AA?5?$AA?$AA@ 0042e7d0     sp_shiori.obj
 0002:000037e4       ??_C@_1BE@COB@?$AAC?$AAh?$AAa?$AAr?$AAs?$AAe?$AAt?$AA?3?$AA?5?$AA?$AA@ 0042e7e4     sp_shiori.obj
 0002:000037f8       ??_C@_1BM@GPCE@?$AA?5?$AAS?$AAH?$AAI?$AAO?$AAR?$AAI?$AA?1?$AA3?$AA?4?$AA0?$AA?$AN?$AA?6?$AA?$AA@ 0042e7f8     sp_shiori.obj
 0002:00003814       ??_C@_17KJPO@?$AAG?$AAE?$AAT?$AA?$AA@ 0042e814     sp_shiori.obj
 0002:0000381c       ??_C@_1O@LKEJ@?$AAN?$AAO?$AAT?$AAI?$AAF?$AAY?$AA?$AA@ 0042e81c     sp_shiori.obj
 0002:0000382c       ??_C@_0M@OAHE@?$CIload?5call?$CJ?$AA@ 0042e82c     sp_shiori.obj
 0002:00003838       ??_C@_0BJ@LPDP@?$CIgetversion?1loadex?5call?$CJ?$AA@ 0042e838     sp_shiori.obj
 0002:00003854       ??_C@_0BK@HEPE@?$CIfunction?5?3?5unload?5found?$CJ?$AA@ 0042e854     sp_shiori.obj
 0002:00003870       ??_C@_0BL@INP@?$CIfunction?5?3?5request?5found?$CJ?$AA@ 0042e870     sp_shiori.obj
 0002:0000388c       ??_C@_0BI@HFCJ@?$CIfunction?5?3?5load?5found?$CJ?$AA@ 0042e88c     sp_shiori.obj
 0002:000038a4       ??_C@_0BK@MFFP@?$CIfunction?5?3?5loadex?5found?$CJ?$AA@ 0042e8a4     sp_shiori.obj
 0002:000038c0       ??_C@_0P@CNOJ@_getimpression?$AA@ 0042e8c0     sp_shiori.obj
 0002:000038d0       ??_C@_0N@GHFH@_getresponse?$AA@ 0042e8d0     sp_shiori.obj
 0002:000038e0       ??_C@_0BA@NJJF@_setupnametable?$AA@ 0042e8e0     sp_shiori.obj
 0002:000038f0       ??_C@_0O@BMPA@_getmatchword?$AA@ 0042e8f0     sp_shiori.obj
 0002:00003900       ??_C@_08MDFC@_getword?$AA@ 0042e900     sp_shiori.obj
 0002:0000390c       ??_C@_07HOJF@_getdms?$AA@  0042e90c     sp_shiori.obj
 0002:00003914       ??_C@_0M@JAPC@_getaistate?$AA@ 0042e914     sp_shiori.obj
 0002:00003920       ??_C@_0BD@PGGL@_getaistringrandom?$AA@ 0042e920     sp_shiori.obj
 0002:00003934       ??_C@_0L@JDF@_construct?$AA@ 0042e934     sp_shiori.obj
 0002:00003940       ??_C@_09DMCM@_destruct?$AA@ 0042e940     sp_shiori.obj
 0002:0000394c       ??_C@_0P@GOJ@?$CIload?5library?$CJ?$AA@ 0042e94c     sp_shiori.obj
 0002:0000395c       ??_C@_09FIAF@alias?4txt?$AA@ 0042e95c     sp_shiori.obj
 0002:00003968       ??_C@_0N@KGOO@descript?4txt?$AA@ 0042e968     sp_shiori.obj
 0002:00003978       ??_C@_06BNJB@shiori?$AA@   0042e978     sp_shiori.obj
 0002:00003980       ??_C@_1CE@LONN@?$AAS?$AAH?$AAI?$AAO?$AAR?$AAI?$AA?$CI?$AAc?$AAo?$AAn?$AAs?$AAt?$AAr?$AAu?$AAc?$AAt?$AA?$CJ?$AA?$AA@ 0042e980     sp_shiori.obj
 0002:000039b4       ??_C@_05KBGO@Value?$AA@    0042e9b4     sp_shiori.obj
 0002:000039bc       ??_C@_19OFKN@?$AA?$AN?$AA?6?$AA?$AN?$AA?6?$AA?$AA@ 0042e9bc     sp_shiori.obj
 0002:000039c8       ??_7SPShioriEvent@@6B@     0042e9c8     sp_shiori.obj
 0002:000039cc       ??_7SPModuleEvent@@6B@     0042e9cc     sp_shiori.obj
 0002:000039d0       ??_C@_1BI@IFAD@?$AAB?$AAa?$AAs?$AAe?$AAE?$AAv?$AAe?$AAn?$AAt?$AA?3?$AA?5?$AA?$AA@ 0042e9d0     sp_shiori.obj
 0002:000039e8       ??_C@_1BA@DAJN@?$AAE?$AAv?$AAe?$AAn?$AAt?$AA?3?$AA?5?$AA?$AA@ 0042e9e8     sp_shiori.obj
 0002:000039f8       ??_C@_1DE@GOHI@?$AAG?$AAE?$AAT?$AA?5?$AAS?$AAe?$AAn?$AAt?$AAe?$AAn?$AAc?$AAe?$AA?5?$AAS?$AAH?$AAI?$AAO?$AAR?$AAI?$AA?1@ 0042e9f8     sp_shiori.obj
 0002:00003a2c       ??_C@_1BC@HJIP@?$AAl?$AAo?$AAg?$AA_?$AAf?$AAi?$AAl?$AAe?$AA?$AA@ 0042ea2c     sp_shiori.obj
 0002:00003a40       ??_C@_1BG@DGGL@?$AAe?$AAn?$AAa?$AAb?$AAl?$AAe?$AA_?$AAl?$AAo?$AAg?$AA?$AA@ 0042ea40     sp_shiori.obj
 0002:00003a58       ??_C@_1BK@DHHM@?$AAe?$AAn?$AAa?$AAb?$AAl?$AAe?$AA_?$AAd?$AAe?$AAb?$AAu?$AAg?$AA?$AA@ 0042ea58     sp_shiori.obj
 0002:00003a74       ??_C@_1BG@FIDH@?$AAS?$AAh?$AAi?$AAo?$AAr?$AAi?$AAE?$AAc?$AAh?$AAo?$AA?$AA@ 0042ea74     sp_shiori.obj
 0002:00003a8c       ??_C@_0O@NFPG@BalloonOffset?$AA@ 0042ea8c     sp_shiori.obj
 0002:00003a9c       ??_C@_06NDMJ@Marker?$AA@   0042ea9c     sp_shiori.obj
 0002:00003aa4       ??_C@_08HHFB@Sentence?$AA@ 0042eaa4     sp_shiori.obj
 0002:00003ab0       ??_C@_06PINC@String?$AA@   0042eab0     sp_shiori.obj
 0002:00003ab8       ??_C@_1DA@NFH@?$AAG?$AAE?$AAT?$AA?5?$AAS?$AAt?$AAr?$AAi?$AAn?$AAg?$AA?5?$AAS?$AAH?$AAI?$AAO?$AAR?$AAI?$AA?1?$AA2?$AA?4@ 0042eab8     sp_shiori.obj
 0002:00003ae8       ??_C@_1BG@PCND@?$AAe?$AAs?$AAe?$AA?9?$AAs?$AAh?$AAi?$AAo?$AAr?$AAi?$AA?$AA@ 0042eae8     sp_shiori.obj
 0002:00003b00       ??_C@_02IBHF@id?$AA@       0042eb00     sp_shiori.obj
 0002:00003b04       ??_C@_1M@DMNH@?$AAl?$AAo?$AAc?$AAa?$AAl?$AA?$AA@ 0042eb04     sp_shiori.obj
 0002:00003b10       ??_C@_0O@DKCE@SecurityLevel?$AA@ 0042eb10     sp_shiori.obj
 0002:00003b20       ??_C@_1BA@BMAP@?$AAm?$AAa?$AAt?$AAe?$AAr?$AAi?$AAa?$AA?$AA@ 0042eb20     sp_shiori.obj
 0002:00003b30       ??_C@_03NDIP@DLL?$AA@      0042eb30     sp_shiori.obj
 0002:00003b34       ??_C@_0M@KOKG@materia?4exe?$AA@ 0042eb34     sp_shiori.obj
 0002:00003b40       ??_C@_09GMDJ@first?4dll?$AA@ 0042eb40     sp_shiori.obj
 0002:00003b4c       ??_C@_1O@FPOH@?$AAe?$AAm?$AAb?$AAr?$AAy?$AAo?$AA?$AA@ 0042eb4c     sp_shiori.obj
 0002:00003b5c       ??_C@_0L@LKBG@sayuri?4dll?$AA@ 0042eb5c     sp_shiori.obj
 0002:00003b68       ??_C@_0L@PKJP@futaba?4dll?$AA@ 0042eb68     sp_shiori.obj
 0002:00003b74       ??_C@_07DLDI@mai?4dll?$AA@ 0042eb74     sp_shiori.obj
 0002:00003b7c       ??_C@_0L@OANM@embryo?4exe?$AA@ 0042eb7c     sp_shiori.obj
 0002:00003b88       ??_C@_0P@LHBH@Toyoaki?5Sagawa?$AA@ 0042eb88     sp_shiori.obj
 0002:00003b98       ??_C@_0L@KJII@sakura?4dll?$AA@ 0042eb98     sp_shiori.obj
 0002:00003ba4       ??_C@_0BE@KBCC@UnhookWindowsHookEx?$AA@ 0042eba4     sp_shiori.obj
 0002:00003bb8       ??_C@_0BC@OAPA@SetWindowsHookExW?$AA@ 0042ebb8     sp_shiori.obj
 0002:00003bcc       ??_C@_0BC@LGPC@SetWindowsHookExA?$AA@ 0042ebcc     sp_shiori.obj
 0002:00003be0       ??_C@_0BD@PPDH@GetModuleFileNameA?$AA@ 0042ebe0     sp_shiori.obj
 0002:00003bf4       ??_C@_0P@DGOG@GetProcAddress?$AA@ 0042ebf4     sp_shiori.obj
 0002:00003c04       ??_C@_0P@NML@LoadLibraryExW?$AA@ 0042ec04     sp_shiori.obj
 0002:00003c14       ??_C@_0P@FLMJ@LoadLibraryExA?$AA@ 0042ec14     sp_shiori.obj
 0002:00003c24       ??_C@_0N@ENMI@LoadLibraryW?$AA@ 0042ec24     sp_shiori.obj
 0002:00003c34       ??_C@_0N@BLMK@LoadLibraryA?$AA@ 0042ec34     sp_shiori.obj
 0002:00003c44       ??_C@_0M@KMCI@MessageBoxW?$AA@ 0042ec44     sp_shiori.obj
 0002:00003c50       ??_C@_0M@PKCK@MessageBoxA?$AA@ 0042ec50     sp_shiori.obj
 0002:00003c5c       ??_C@_0BA@HBIG@PdhVbAddCounter?$AA@ 0042ec5c     sp_shiori.obj
 0002:00003c6c       ??_C@_0BL@ENCP@PdhVbGetDoubleCounterValue?$AA@ 0042ec6c     sp_shiori.obj
 0002:00003c88       ??_C@_08OHBC@?2ssp?4exe?$AA@ 0042ec88     sp_shiori.obj
 0002:00003c94       ??_C@_0BK@NBFM@ImageDirectoryEntryToData?$AA@ 0042ec94     sp_shiori.obj
 0002:00003cb0       ??_C@_07DGOH@?5Test?$CFu?$AA@ 0042ecb0     sp_sysinfo.obj
 0002:00003cb8       ??_C@_03POF@?9?$CFu?$AA@   0042ecb8     sp_sysinfo.obj
 0002:00003cbc       ??_C@_05PLPC@?5RC?$CFu?$AA@ 0042ecbc     sp_sysinfo.obj
 0002:00003cc4       ??_C@_06EELN@?5Pre?$CFu?$AA@ 0042ecc4     sp_sysinfo.obj
 0002:00003ccc       ??_C@_05CED@?5DR?$CFu?$AA@ 0042eccc     sp_sysinfo.obj
 0002:00003cd4       ??_C@_0BP@LGAF@?$FLH?$CFu?4?$CFu?9?$CFu?4?$CFu?1S?$CFu?4?$CFu?4?$CFu?9?$CFu?9?$CFu?$FN?$AA@ 0042ecd4     sp_sysinfo.obj
 0002:00003cf4       ??_C@_0N@GKFE@GenuineTMx86?$AA@ 0042ecf4     sp_sysinfo.obj
 0002:00003d04       ??_C@_0M@EGHG@?$CFu?4?$CFu?4?$CFu?4?$CFu?$AA@ 0042ed04     sp_sysinfo.obj
 0002:00003d10       ??_C@_07IJDM@0?40?40?40?$AA@ 0042ed10     sp_sysinfo.obj
 0002:00003d18       ??_C@_07PCHH@Unknown?$AA@  0042ed18     sp_sysinfo.obj
 0002:00003d20       ??_C@_0O@JDAJ@IsThemeActive?$AA@ 0042ed20     sp_sysinfo.obj
 0002:00003d30       ??_C@_07NGFJ@uxtheme?$AA@  0042ed30     sp_sysinfo.obj
 0002:00003d38       ??_C@_01FCOA@?5?$AA@       0042ed38     sp_sysinfo.obj
 0002:00003d3c       ??_C@_0BG@HBBP@wine_get_host_version?$AA@ 0042ed3c     sp_sysinfo.obj
 0002:00003d54       ??_C@_0BB@OJOH@wine_get_version?$AA@ 0042ed54     sp_sysinfo.obj
 0002:00003d68       ??_C@_0BI@PFKN@wine_get_unix_file_name?$AA@ 0042ed68     sp_sysinfo.obj
 0002:00003d80       ??_C@_08EIKE@comctl32?$AA@ 0042ed80     sp_sysinfo.obj
 0002:00003d8c       ??_C@_07MFEP@shell32?$AA@  0042ed8c     sp_sysinfo.obj
 0002:00003d94       ??_C@_0O@GDAK@RtlGetVersion?$AA@ 0042ed94     sp_sysinfo.obj
 0002:00003da4       ??_C@_05OEEN@ntdll?$AA@    0042eda4     sp_sysinfo.obj
 0002:00003dac       ??_C@_06KFAF@Compaq?$AA@   0042edac     sp_sysinfo.obj
 0002:00003db4       ??_C@_0N@JJGH@Compaq?5FX32?$CB?$AA@ 0042edb4     sp_sysinfo.obj
 0002:00003dc4       ??_C@_03FIOC@NSC?$AA@      0042edc4     sp_sysinfo.obj
 0002:00003dc8       ??_C@_0N@GJDM@Geode?5By?5NSC?$AA@ 0042edc8     sp_sysinfo.obj
 0002:00003dd8       ??_C@_03LHAE@UMC?$AA@      0042edd8     sp_sysinfo.obj
 0002:00003ddc       ??_C@_0N@OLGO@UMC?5UMC?5UMC?5?$AA@ 0042eddc     sp_sysinfo.obj
 0002:00003dec       ??_C@_06EACG@NexGen?$AA@   0042edec     sp_sysinfo.obj
 0002:00003df4       ??_C@_0N@PLND@NexGenDriven?$AA@ 0042edf4     sp_sysinfo.obj
 0002:00003e04       ??_C@_04JHJG@Rise?$AA@     0042ee04     sp_sysinfo.obj
 0002:00003e0c       ??_C@_0N@PBDK@RiseRiseRise?$AA@ 0042ee0c     sp_sysinfo.obj
 0002:00003e1c       ??_C@_03BBOK@IDT?$AA@      0042ee1c     sp_sysinfo.obj
 0002:00003e20       ??_C@_0N@CBMN@CentaurHauls?$AA@ 0042ee20     sp_sysinfo.obj
 0002:00003e30       ??_C@_05NJMG@Cyrix?$AA@    0042ee30     sp_sysinfo.obj
 0002:00003e38       ??_C@_0N@MOOL@CyrixInstead?$AA@ 0042ee38     sp_sysinfo.obj
 0002:00003e48       ??_C@_09LCBG@Transmeta?$AA@ 0042ee48     sp_sysinfo.obj
 0002:00003e54       ??_C@_03ILNB@AMD?$AA@      0042ee54     sp_sysinfo.obj
 0002:00003e58       ??_C@_0N@OLMF@AuthenticAMD?$AA@ 0042ee58     sp_sysinfo.obj
 0002:00003e68       ??_C@_05DHJM@Intel?$AA@    0042ee68     sp_sysinfo.obj
 0002:00003e70       ??_C@_0N@GALO@GenuineIntel?$AA@ 0042ee70     sp_sysinfo.obj
 0002:00003e8c       ??_C@_19KFLE@?$AAP?$AAE?$AAR?$AAF?$AA?$AA@ 0042ee8c     sp_sysinfo.obj
 0002:00003e98       ??_C@_01KOLO@2?$AA@        0042ee98     sp_sysinfo.obj
 0002:00003e9c       ??_C@_0O@CDEE@DllGetVersion?$AA@ 0042ee9c     sp_sysinfo.obj
 0002:00003eac       ??_C@_04BBPO@?$HOMHz?$AA@  0042eeac     sp_sysinfo.obj
 0002:00003eb4       ??_C@_0CP@HBON@HARDWARE?2DESCRIPTION?2System?2Cent@ 0042eeb4     sp_sysinfo.obj
 0002:00003ee4       ??_C@_0BF@BEPG@GlobalMemoryStatusEx?$AA@ 0042eee4     sp_sysinfo.obj
 0002:00003efc       ??_C@_0BA@DLLO@SSP?1?$CFs?5?$CI?$CFs?$DL?5?$CFs?$CJ?$AA@ 0042eefc     sp_sysinfo.obj
 0002:00003f0c       ??_C@_1BK@DGEA@?$AA?$CF?$AAu?$AA?4?$AA?$CF?$AAu?$AA?4?$AA?$CF?$AA0?$AA2?$AAu?$AA?$CF?$AAs?$AA?$AA@ 0042ef0c     sp_sysinfo.obj
 0002:00003f28       ??_C@_0N@PMHO@?$CFu?4?$CFu?4?$CF02u?$CFs?$AA@ 0042ef28     sp_sysinfo.obj
 0002:00003f38       ??_C@_0L@EOHC@Windows?5Me?$AA@ 0042ef38     sp_sysinfo.obj
 0002:00003f44       ??_C@_02FOPI@SE?$AA@       0042ef44     sp_sysinfo.obj
 0002:00003f48       ??_C@_0L@FJEF@Windows?598?$AA@ 0042ef48     sp_sysinfo.obj
 0002:00003f54       ??_C@_04JFLH@OSR2?$AA@     0042ef54     sp_sysinfo.obj
 0002:00003f5c       ??_C@_0L@NDG@Windows?595?$AA@ 0042ef5c     sp_sysinfo.obj
 0002:00003f68       ??_C@_09LHJE@Wow64?$EAx64?$AA@ 0042ef68     sp_sysinfo.obj
 0002:00003f74       ??_C@_0L@JOIA@?1Wow64?$EAx64?$AA@ 0042ef74     sp_sysinfo.obj
 0002:00003f80       ??_C@_08PJNC@?$EAUnknown?$AA@ 0042ef80     sp_sysinfo.obj
 0002:00003f8c       ??_C@_05BMGH@?$EAIA64?$AA@ 0042ef8c     sp_sysinfo.obj
 0002:00003f94       ??_C@_06BMOD@?$EAARM64?$AA@ 0042ef94     sp_sysinfo.obj
 0002:00003f9c       ??_C@_04JPND@?$EAARM?$AA@  0042ef9c     sp_sysinfo.obj
 0002:00003fa4       ??_C@_04LLON@?$EAx64?$AA@  0042efa4     sp_sysinfo.obj
 0002:00003fac       ??_C@_05IEKO@Wow64?$AA@    0042efac     sp_sysinfo.obj
 0002:00003fb4       ??_C@_06HFML@?1Wow64?$AA@  0042efb4     sp_sysinfo.obj
 0002:00003fbc       ??_C@_0BA@LJFP@IsWow64Process2?$AA@ 0042efbc     sp_sysinfo.obj
 0002:00003fcc       ??_C@_0P@OBHG@IsWow64Process?$AA@ 0042efcc     sp_sysinfo.obj
 0002:00003fdc       ??_C@_07PJED@?$CLRollup?$AA@ 0042efdc     sp_sysinfo.obj
 0002:00003fe4       ??_C@_02PHED@SP?$AA@       0042efe4     sp_sysinfo.obj
 0002:00003fe8       ??_C@_0O@DAEN@Service?5Pack?5?$AA@ 0042efe8     sp_sysinfo.obj
 0002:00003ff8       ??_C@_06HDNO@?5?$CIVer?4?$AA@ 0042eff8     sp_sysinfo.obj
 0002:00004000       ??_C@_09BCCP@ReleaseId?$AA@ 0042f000     sp_sysinfo.obj
 0002:0000400c       ??_C@_03PJNO@?4?$CFu?$AA@  0042f00c     sp_sysinfo.obj
 0002:00004010       ??_C@_03GAOC@UBR?$AA@      0042f010     sp_sysinfo.obj
 0002:00004014       ??_C@_0CN@OICJ@Software?2Microsoft?2Windows?5NT?2Cu@ 0042f014     sp_sysinfo.obj
 0002:00004044       ??_C@_0P@IJJG@Windows?510?5RSx?$AA@ 0042f044     sp_sysinfo.obj
 0002:00004054       ??_C@_0BE@HBGA@Windows?510?5RS5?1WIPB?$AA@ 0042f054     sp_sysinfo.obj
 0002:00004068       ??_C@_0BC@LJPM@Windows?510?5RS4?1CB?$AA@ 0042f068     sp_sysinfo.obj
 0002:0000407c       ??_C@_0BE@OEMA@Windows?510?5RS4?1WIPB?$AA@ 0042f07c     sp_sysinfo.obj
 0002:00004090       ??_C@_0BC@EDEC@Windows?510?5RS3?1CB?$AA@ 0042f090     sp_sysinfo.obj
 0002:000040a4       ??_C@_0BE@MKA@Windows?510?5RS3?1WIPB?$AA@ 0042f0a4     sp_sysinfo.obj
 0002:000040b8       ??_C@_0BC@GGBA@Windows?510?5RS2?1CB?$AA@ 0042f0b8     sp_sysinfo.obj
 0002:000040cc       ??_C@_0BE@JJAA@Windows?510?5RS2?1WIPB?$AA@ 0042f0cc     sp_sysinfo.obj
 0002:000040e0       ??_C@_0BC@JOG@Windows?510?5RS1?1CB?$AA@ 0042f0e0     sp_sysinfo.obj
 0002:000040f4       ??_C@_0BE@CHOA@Windows?510?5RS1?1WIPB?$AA@ 0042f0f4     sp_sysinfo.obj
 0002:00004108       ??_C@_0BC@PIMA@Windows?510?5TH2?1CB?$AA@ 0042f108     sp_sysinfo.obj
 0002:0000411c       ??_C@_0BE@MHKO@Windows?510?5TH2?1WIPB?$AA@ 0042f11c     sp_sysinfo.obj
 0002:00004130       ??_C@_0BC@JHDG@Windows?510?5TH1?1CB?$AA@ 0042f130     sp_sysinfo.obj
 0002:00004144       ??_C@_0BE@HJEO@Windows?510?5TH1?1WIPB?$AA@ 0042f144     sp_sysinfo.obj
 0002:00004158       ??_C@_0BE@DHGL@Windows?5Server?52016?$AA@ 0042f158     sp_sysinfo.obj
 0002:0000416c       ??_C@_0M@FJBO@Windows?58?41?$AA@ 0042f16c     sp_sysinfo.obj
 0002:00004178       ??_C@_0BH@OHBP@Windows?5Server?52012?5R2?$AA@ 0042f178     sp_sysinfo.obj
 0002:00004190       ??_C@_09MHPP@Windows?58?$AA@ 0042f190     sp_sysinfo.obj
 0002:0000419c       ??_C@_0BE@JNDH@Windows?5Server?52012?$AA@ 0042f19c     sp_sysinfo.obj
 0002:000041b0       ??_C@_09MGKC@Windows?57?$AA@ 0042f1b0     sp_sysinfo.obj
 0002:000041bc       ??_C@_0BH@CHAO@Windows?5Server?52008?5R2?$AA@ 0042f1bc     sp_sysinfo.obj
 0002:000041d4       ??_C@_0O@EDAH@Windows?5Vista?$AA@ 0042f1d4     sp_sysinfo.obj
 0002:000041e4       ??_C@_0BE@IKAL@Windows?5Server?52008?$AA@ 0042f1e4     sp_sysinfo.obj
 0002:000041f8       ??_C@_0BE@CBAK@Windows?5Server?52003?$AA@ 0042f1f8     sp_sysinfo.obj
 0002:0000420c       ??_C@_0BH@GCGI@Windows?5Server?52003?5R2?$AA@ 0042f20c     sp_sysinfo.obj
 0002:00004224       ??_C@_0L@JDIA@Windows?5XP?$AA@ 0042f224     sp_sysinfo.obj
 0002:00004230       ??_C@_0BD@ECDE@HeapSetInformation?$AA@ 0042f230     sp_sysinfo.obj
 0002:00004244       ??_C@_0N@CDPP@Windows?52000?$AA@ 0042f244     sp_sysinfo.obj
 0002:00004254       ??_C@_0BE@EOAC@Windows?5NT?5?$CFd?4?$CFd?4?$CFd?$AA@ 0042f254     sp_sysinfo.obj
 0002:00004268       ??_C@_0BB@KDH@Windows?5NT?5?$CFd?4?$CFd?$AA@ 0042f268     sp_sysinfo.obj
 0002:0000427c       ??_C@_0BL@BOMG@ABCDEFGHIJKLMNOPQRSTUVWXYZ?$AA@ 0042f27c     sp_sysinfo.obj
 0002:00004298       ??_C@_1BI@KPON@?$AA?$CF?$AAu?$AA?4?$AA?$CF?$AAu?$AA?4?$AA?$CF?$AAu?$AA?4?$AA?$CF?$AAu?$AA?$AA@ 0042f298     sp_sysinfo.obj
 0002:00004538       ??_C@_03PGJO@Dec?$AA@      0042f538     sp_utils.obj
 0002:0000453c       ??_C@_03PDLM@Nov?$AA@      0042f53c     sp_utils.obj
 0002:00004540       ??_C@_03BLHK@Oct?$AA@      0042f540     sp_utils.obj
 0002:00004544       ??_C@_03DPFM@Sep?$AA@      0042f544     sp_utils.obj
 0002:00004548       ??_C@_03CMCH@Aug?$AA@      0042f548     sp_utils.obj
 0002:0000454c       ??_C@_03OBKI@Jul?$AA@      0042f54c     sp_utils.obj
 0002:00004550       ??_C@_03LEIG@Jun?$AA@      0042f550     sp_utils.obj
 0002:00004554       ??_C@_03MGHB@May?$AA@      0042f554     sp_utils.obj
 0002:00004558       ??_C@_03MJJM@Apr?$AA@      0042f558     sp_utils.obj
 0002:0000455c       ??_C@_03GNHA@Mar?$AA@      0042f55c     sp_utils.obj
 0002:00004560       ??_C@_03PICE@Feb?$AA@      0042f560     sp_utils.obj
 0002:00004564       ??_C@_03IEIF@Jan?$AA@      0042f564     sp_utils.obj
 0002:00004568       ??_C@_03MPKK@Sat?$AA@      0042f568     sp_utils.obj
 0002:0000456c       ??_C@_03FINJ@Fri?$AA@      0042f56c     sp_utils.obj
 0002:00004570       ??_C@_03HIKC@Thu?$AA@      0042f570     sp_utils.obj
 0002:00004574       ??_C@_03HECK@Wed?$AA@      0042f574     sp_utils.obj
 0002:00004578       ??_C@_03ECCP@Tue?$AA@      0042f578     sp_utils.obj
 0002:0000457c       ??_C@_03PIEP@Mon?$AA@      0042f57c     sp_utils.obj
 0002:00004580       ??_C@_03FHEP@Sun?$AA@      0042f580     sp_utils.obj
 0002:00004584       ??_C@_19HAML@?$AAl?$AAp?$AAt?$AA9?$AA?$AA@ 0042f584     sp_utils.obj
 0002:00004590       ??_C@_19CCNN@?$AAl?$AAp?$AAt?$AA8?$AA?$AA@ 0042f590     sp_utils.obj
 0002:0000459c       ??_C@_19MAJ@?$AAl?$AAp?$AAt?$AA7?$AA?$AA@ 0042f59c     sp_utils.obj
 0002:000045a8       ??_C@_19FOBP@?$AAl?$AAp?$AAt?$AA6?$AA?$AA@ 0042f5a8     sp_utils.obj
 0002:000045b4       ??_C@_19KICE@?$AAl?$AAp?$AAt?$AA5?$AA?$AA@ 0042f5b4     sp_utils.obj
 0002:000045c0       ??_C@_19PKDC@?$AAl?$AAp?$AAt?$AA4?$AA?$AA@ 0042f5c0     sp_utils.obj
 0002:000045cc       ??_C@_19EEFD@?$AAl?$AAp?$AAt?$AA3?$AA?$AA@ 0042f5cc     sp_utils.obj
 0002:000045d8       ??_C@_19BGEF@?$AAl?$AAp?$AAt?$AA2?$AA?$AA@ 0042f5d8     sp_utils.obj
 0002:000045e4       ??_C@_19OAHO@?$AAl?$AAp?$AAt?$AA1?$AA?$AA@ 0042f5e4     sp_utils.obj
 0002:000045f0       ??_C@_19NKDH@?$AAc?$AAo?$AAm?$AA9?$AA?$AA@ 0042f5f0     sp_utils.obj
 0002:000045fc       ??_C@_19IICB@?$AAc?$AAo?$AAm?$AA8?$AA?$AA@ 0042f5fc     sp_utils.obj
 0002:00004608       ??_C@_19KGPF@?$AAc?$AAo?$AAm?$AA7?$AA?$AA@ 0042f608     sp_utils.obj
 0002:00004614       ??_C@_19PEOD@?$AAc?$AAo?$AAm?$AA6?$AA?$AA@ 0042f614     sp_utils.obj
 0002:00004620       ??_C@_19CNI@?$AAc?$AAo?$AAm?$AA5?$AA?$AA@ 0042f620     sp_utils.obj
 0002:0000462c       ??_C@_19FAMO@?$AAc?$AAo?$AAm?$AA4?$AA?$AA@ 0042f62c     sp_utils.obj
 0002:00004638       ??_C@_19OOKP@?$AAc?$AAo?$AAm?$AA3?$AA?$AA@ 0042f638     sp_utils.obj
 0002:00004644       ??_C@_19LMLJ@?$AAc?$AAo?$AAm?$AA2?$AA?$AA@ 0042f644     sp_utils.obj
 0002:00004650       ??_C@_19EKIC@?$AAc?$AAo?$AAm?$AA1?$AA?$AA@ 0042f650     sp_utils.obj
 0002:0000465c       ??_C@_17NEIH@?$AAn?$AAu?$AAl?$AA?$AA@ 0042f65c     sp_utils.obj
 0002:00004664       ??_C@_17GKNK@?$AAp?$AAr?$AAn?$AA?$AA@ 0042f664     sp_utils.obj
 0002:0000466c       ??_C@_17PC@?$AAa?$AAu?$AAx?$AA?$AA@ 0042f66c     sp_utils.obj
 0002:00004674       ??_C@_17NDPB@?$AAc?$AAo?$AAn?$AA?$AA@ 0042f674     sp_utils.obj
 0002:0000467c       ??_C@_04ONEB@lpt9?$AA@     0042f67c     sp_utils.obj
 0002:00004684       ??_C@_04EHNG@lpt8?$AA@     0042f684     sp_utils.obj
 0002:0000468c       ??_C@_04EGIL@lpt7?$AA@     0042f68c     sp_utils.obj
 0002:00004694       ??_C@_04OMBM@lpt6?$AA@     0042f694     sp_utils.obj
 0002:0000469c       ??_C@_04BDKF@lpt5?$AA@     0042f69c     sp_utils.obj
 0002:000046a4       ??_C@_04LJDC@lpt4?$AA@     0042f6a4     sp_utils.obj
 0002:000046ac       ??_C@_04OMNH@lpt3?$AA@     0042f6ac     sp_utils.obj
 0002:000046b4       ??_C@_04EGEA@lpt2?$AA@     0042f6b4     sp_utils.obj
 0002:000046bc       ??_C@_04LJPJ@lpt1?$AA@     0042f6bc     sp_utils.obj
 0002:000046c4       ??_C@_04PLIG@com9?$AA@     0042f6c4     sp_utils.obj
 0002:000046cc       ??_C@_04FBBB@com8?$AA@     0042f6cc     sp_utils.obj
 0002:000046d4       ??_C@_04FAEM@com7?$AA@     0042f6d4     sp_utils.obj
 0002:000046dc       ??_C@_04PKNL@com6?$AA@     0042f6dc     sp_utils.obj
 0002:000046e4       ??_C@_04FGC@com5?$AA@      0042f6e4     sp_utils.obj
 0002:000046ec       ??_C@_04KPPF@com4?$AA@     0042f6ec     sp_utils.obj
 0002:000046f4       ??_C@_04PKBA@com3?$AA@     0042f6f4     sp_utils.obj
 0002:000046fc       ??_C@_04FAIH@com2?$AA@     0042f6fc     sp_utils.obj
 0002:00004704       ??_C@_04KPDO@com1?$AA@     0042f704     sp_utils.obj
 0002:0000470c       ??_C@_03OLCH@nul?$AA@      0042f70c     sp_utils.obj
 0002:00004710       ??_C@_03ICPE@prn?$AA@      0042f710     sp_utils.obj
 0002:00004714       ??_C@_03MGNP@aux?$AA@      0042f714     sp_utils.obj
 0002:00004718       ??_C@_03MGFI@con?$AA@      0042f718     sp_utils.obj
 0002:0000471c       ??_C@_0N@EHDE@XtraStuf?4mac?$AA@ 0042f71c     sp_utils.obj
 0002:0000472c       ??_C@_08FNCJ@__MACOSX?$AA@ 0042f72c     sp_utils.obj
 0002:00004738       ??_C@_03GIEB@var?$AA@      0042f738     sp_utils.obj
 0002:0000473c       ??_C@_0BE@PLPH@satori_savedata?4sat?$AA@ 0042f73c     sp_utils.obj
 0002:00004750       ??_C@_0BE@IMMB@satori_savedata?4txt?$AA@ 0042f750     sp_utils.obj
 0002:00004764       ??_C@_0BC@LLN@yaya_variable?4ays?$AA@ 0042f764     sp_utils.obj
 0002:00004778       ??_C@_0BC@BCBE@yaya_variable?4cfg?$AA@ 0042f778     sp_utils.obj
 0002:0000478c       ??_C@_0BC@EMDG@aya5_variable?4cfg?$AA@ 0042f78c     sp_utils.obj
 0002:000047a0       ??_C@_0N@LMFH@_CATALOG?4VIX?$AA@ 0042f7a0     sp_utils.obj
 0002:000047b0       ??_C@_0N@DBAE@mscreate?4dir?$AA@ 0042f7b0     sp_utils.obj
 0002:000047c0       ??_C@_0M@JCKF@desktop?4ini?$AA@ 0042f7c0     sp_utils.obj
 0002:000047cc       ??_C@_0L@OPBC@folder?4htt?$AA@ 0042f7cc     sp_utils.obj
 0002:000047d8       ??_C@_09EGIG@?4DS_Store?$AA@ 0042f7d8     sp_utils.obj
 0002:000047e4       ??_C@_09DBCG@thumbs?4db?$AA@ 0042f7e4     sp_utils.obj
 0002:000047f0       ??_C@_07LBEP@ngm?4dat?$AA@ 0042f7f0     sp_utils.obj
 0002:000047f8       ??_C@_06JJKD@Local?2?$AA@  0042f7f8     sp_utils.obj
 0002:00004800       ??_C@_02HEEH@?3?1?$AA@     0042f800     sp_utils.obj
 0002:00004804       ??_C@_02NNKG@?2?2?$AA@     0042f804     sp_utils.obj
 0002:00004808       ??_C@_02NFKO@?3?2?$AA@     0042f808     sp_utils.obj
 0002:0000480c       ??_C@_17BLBD@?$AA?3?$AA?1?$AA?1?$AA?$AA@ 0042f80c     sp_utils.obj
 0002:00004814       ??_C@_03FMJ@?3?1?1?$AA@    0042f814     sp_utils.obj
 0002:00004818       ??_C@_17PIBE@?$AA?4?$AA?4?$AA?2?$AA?$AA@ 0042f818     sp_utils.obj
 0002:00004820       ??_C@_15LJHA@?$AA?4?$AA?2?$AA?$AA@ 0042f820     sp_utils.obj
 0002:00004828       ??_C@_17OIDK@?$AA?4?$AA?4?$AA?1?$AA?$AA@ 0042f828     sp_utils.obj
 0002:00004830       ??_C@_15KJFO@?$AA?4?$AA?1?$AA?$AA@ 0042f830     sp_utils.obj
 0002:00004838       ??_C@_04KHOB@open?$AA@     0042f838     sp_utils.obj
 0002:00004840       ??_C@_07PCOP@http?3?1?1?$AA@ 0042f840     sp_utils.obj
 0002:00004848       ??_C@_01HMO@?$CC?$AA@      0042f848     sp_utils.obj
 0002:0000484c       ??_C@_0BC@NDDB@?$CFd?0?$CFd?0?$CFd?0?$CFd?0?$CFd?0?$CFd?$AA@ 0042f84c     sp_utils.obj
 0002:00004860       ??_C@_0DB@KMGG@?$CF08x?9?$CF04x?9?$CF04x?9?$CF02x?$CF02x?9?$CF02x?$CF02x@ 0042f860     sp_utils.obj
 0002:00004894       ??_C@_01FDHG@?$CK?$AA@     0042f894     sp_utils.obj
 0002:00004898       ??_C@_08HGPB@?$CF04x?$CF04x?$AA@ 0042f898     sp_versioninfo.obj
 0002:000048a4       ??_C@_0BJ@KCFH@?2VarFileInfo?2Translation?$AA@ 0042f8a4     sp_versioninfo.obj
 0002:000048c0       ??_C@_0BB@KMND@?2StringFileInfo?2?$AA@ 0042f8c0     sp_versioninfo.obj
 0002:000048d4       ??_C@_06KBFD@?$CD32770?$AA@ 0042f8d4     ssph.obj
 0002:000048dc       ??_C@_0L@JHDA@?4?4?2ssp?4exe?$AA@ 0042f8dc     ssph.obj
 0002:000048e8       ??_C@_03NLLK@?4?4?2?$AA@   0042f8e8     ssph.obj
 0002:000048ec       ??_C@_19CKBP@?$AAt?$AAi?$AAm?$AAe?$AA?$AA@ 0042f8ec     ssph.obj
 0002:000048f8       ??_C@_1BI@IOPF@?$AAu?$AAp?$AAd?$AAa?$AAt?$AAe?$AA_?$AAs?$AAe?$AAl?$AAf?$AA?$AA@ 0042f8f8     ssph.obj
 0002:00004910       ??_C@_1BG@FJDC@?$AAs?$AAh?$AAi?$AAo?$AAr?$AAi?$AA_?$AAu?$AAr?$AAl?$AA?$AA@ 0042f910     ssph.obj
 0002:00004928       ??_C@_04CGA@?1u?51?$AA@    0042f928     ssph.obj
 0002:00004930       ??_C@_07PJA@ssp?4exe?$AA@  0042f930     ssph.obj
 0002:00004938       ??_C@_0BG@DLDP@SeSystemtimePrivilege?$AA@ 0042f938     ssph.obj
 0002:00004950       ??_C@_0BA@BOLL@X_SSPH_FMO_NAME?$AA@ 0042f950     ssph.obj
 0002:00004960       ??_C@_1BE@ECEM@?$AAO?$AAn?$AAD?$AAe?$AAs?$AAt?$AAr?$AAo?$AAy?$AA?$AA@ 0042f960     ssph.obj
 0002:00004974       ??_C@_1BG@NPFA@?$AAc?$AAo?$AAu?$AAn?$AAt?$AAe?$AAr?$AAu?$AAr?$AAl?$AA?$AA@ 0042f974     ssph.obj
 0002:0000498c       ??_C@_1BK@GMFB@?$AAO?$AAn?$AAI?$AAn?$AAi?$AAt?$AAi?$AAa?$AAl?$AAi?$AAz?$AAe?$AA?$AA@ 0042f98c     ssph.obj
 0002:000049e8       ??_C@_09HFOF@_template?$AA@ 0042f9e8     ssph_url.obj
 0002:000049f4       ??_C@_08JIDH@_network?$AA@ 0042f9f4     ssph_url.obj
 0002:00004a00       ??_C@_07LNKB@_string?$AA@  0042fa00     ssph_url.obj
 0002:00004a08       ??_C@_07KBML@_config?$AA@  0042fa08     ssph_url.obj
 0002:00004a10       ??_C@_06BBMH@?9keeps?$AA@  0042fa10     ssph_url.obj
 0002:00004a18       ??_C@_05MPGP@_link?$AA@    0042fa18     ssph_url.obj
 0002:00004a20       ??_C@_04BMBM@_url?$AA@     0042fa20     ssph_url.obj
 0002:00004a28       ??_C@_03LGB@_id?$AA@       0042fa28     ssph_url.obj
 0002:00004a2c       ??_C@_0L@DIMP@format?91st?$AA@ 0042fa2c     ssph_url.obj
 0002:00004a38       ??_C@_08EBDK@resource?$AA@ 0042fa38     ssph_url.obj
 0002:00004a44       ??_C@_02GAFC@ai?$AA@       0042fa44     ssph_url.obj
 0002:00004a48       ??_C@_03PNFK@?2id?$AA@     0042fa48     ssph_url.obj
 0002:00004a4c       ??_C@_0M@PLBB@?2id?$FLhomeurl?$AA@ 0042fa4c     ssph_url.obj
 0002:00004a58       ??_C@_0BB@JGCP@resource?4homeurl?$AA@ 0042fa58     ssph_url.obj
 0002:00004a6c       ??_C@_08BAFK@$homeurl?$AA@ 0042fa6c     ssph_url.obj
 0002:00004a78       ??_C@_0L@GAPD@On_homeurl?$AA@ 0042fa78     ssph_url.obj
 0002:00004a84       ??_C@_09LOAH@?$IB?$JHhomeurl?$AA@ 0042fa84     ssph_url.obj
 0002:00004a90       ??_C@_02NGAF@wb?$AA@       0042fa90     ioapi.obj
 0002:00004a94       ??_C@_03LLMP@r?$CLb?$AA@   0042fa94     ioapi.obj
 0002:00004a98       ??_C@_02JKAF@rb?$AA@       0042fa98     ioapi.obj
 0002:00004ab4       ??_C@_03DCMC@?$CK?4?$CK?$AA@ 0042fab4     kei.obj
 0002:00004ab8       ??_C@_03PKEJ@txt?$AA@      0042fab8     kei.obj
 0002:00004abc       ??_C@_03PKBH@cab?$AA@      0042fabc     kei.obj
 0002:00004ac0       ??_C@_03DBFH@lzh?$AA@      0042fac0     kei.obj
 0002:00004ac4       ??_C@_01A@?$AA?$AA@        0042fac4     kei.obj
 0002:00004ac8       ??_C@_03JLAJ@kei?$AA@      0042fac8     kei.obj
 0002:00004acc       ??_C@_0DA@FFNC@e?5?9n1?5?9s1?5?9y1?5?9gm1?5?9jc1?5?9jr1?5?9x1@ 0042facc     kei.obj
 0002:00004afc       ??_C@_0BK@DBOF@UnlhaClearEnumMembersProc?$AA@ 0042fafc     kei.obj
 0002:00004b18       ??_C@_0BI@KJJN@UnlhaSetEnumMembersProc?$AA@ 0042fb18     kei.obj
 0002:00004b30       ??_C@_0BC@PKFJ@UnlhaGetFileCount?$AA@ 0042fb30     kei.obj
 0002:00004b44       ??_C@_0BD@DGAL@UnlhaSetCursorMode?$AA@ 0042fb44     kei.obj
 0002:00004b58       ??_C@_05KIIO@Unlha?$AA@    0042fb58     kei.obj
 0002:00004b60       ??_C@_0M@MFKA@unlha32?4dll?$AA@ 0042fb60     kei.obj
 0002:00004b6c       ??_C@_03IIIE@lha?$AA@      0042fb6c     kei.obj
 0002:00004b70       ??_C@_02CFMC@?9l?$AA@      0042fb70     kei.obj
 0002:00004b74       ??_C@_04HDCD@PK?$AD?$AE?$AA@ 0042fb74     kei.obj
 0002:00004b7c       ??_C@_04FHBM@MSCF?$AA@     0042fb7c     kei.obj
 0002:00004b84       _unz_copyright             0042fb84     unzip.obj
 0002:00004bd8       ??_C@_06MNHP@1?42?411?$AA@ 0042fbd8     unzip.obj
 0002:00004be0       ??_7CUnzipper@@6B@         0042fbe0     Unzipper.obj
 0002:00004be4       ??_C@_02OFKN@?4?2?$AA@     0042fbe4     Unzipper.obj
 0002:00004be8       _zip_copyright             0042fbe8     zip.obj
 0002:000074e0       _deflate_copyright         004324e0     zlib:deflate.obj
 0002:000075a8       _z_errmsg                  004325a8     zlib:zutil.obj
 0002:000075d0       _inflate_copyright         004325d0     zlib:inftrees.obj
 0002:00007d44       __dist_code                00432d44     zlib:trees.obj
 0002:00007f44       __length_code              00432f44     zlib:trees.obj
 0002:000081c0       __tls_used                 004331c0     LIBCMT:tlssup.obj
 0002:000082c0       ??_C@_0BH@PHHF@__GLOBAL_HEAP_SELECTED?$AA@ 004332c0     LIBCMT:heapinit.obj
 0002:000082d8       ??_C@_0BF@BBGL@__MSVCRT_HEAP_SELECT?$AA@ 004332d8     LIBCMT:heapinit.obj
 0002:000082f0       __real@8@3fff8000000000000000 004332f0     LIBCMT:testfdiv.obj
 0002:000082f8       __real@8@4015800bf60000000000 004332f8     LIBCMT:testfdiv.obj
 0002:00008300       __real@8@4014bffffc0000000000 00433300     LIBCMT:testfdiv.obj
 0002:00008308       ??_C@_0BK@JEGK@IsProcessorFeaturePresent?$AA@ 00433308     LIBCMT:testfdiv.obj
 0002:00008324       ??_C@_08OBID@KERNEL32?$AA@ 00433324     LIBCMT:testfdiv.obj
 0002:00008330       ??_C@_05OFLO@e?$CL000?$AA@ 00433330     LIBCMT:cvt.obj
 0002:00008338       ??_C@_13A@?$AA?$AA?$AA?$AA@ 00433338     LIBCMT:a_map.obj
 0002:00008364       ___lookuptable             00433364     LIBCMT:output.obj
 0002:000083c0       ??_C@_1O@POHA@?$AA?$CI?$AAn?$AAu?$AAl?$AAl?$AA?$CJ?$AA?$AA@ 004333c0     LIBCMT:output.obj
 0002:000083d0       ??_C@_06ONKE@?$CInull?$CJ?$AA@ 004333d0     LIBCMT:output.obj
 0002:000083e4       ??_C@_0P@GGKG@runtime?5error?5?$AA@ 004333e4     LIBCMT:crt0msg.obj
 0002:000083f4       ??_C@_0O@DELO@TLOSS?5error?$AN?6?$AA@ 004333f4     LIBCMT:crt0msg.obj
 0002:00008404       ??_C@_0N@OMLL@SING?5error?$AN?6?$AA@ 00433404     LIBCMT:crt0msg.obj
 0002:00008414       ??_C@_0P@OJAK@DOMAIN?5error?$AN?6?$AA@ 00433414     LIBCMT:crt0msg.obj
 0002:00008424       ??_C@_0CF@EANP@R6028?$AN?6?9?5unable?5to?5initialize?5he@ 00433424     LIBCMT:crt0msg.obj
 0002:0000844c       ??_C@_0DF@ECGN@R6027?$AN?6?9?5not?5enough?5space?5for?5lo@ 0043344c     LIBCMT:crt0msg.obj
 0002:00008484       ??_C@_0DF@FKAC@R6026?$AN?6?9?5not?5enough?5space?5for?5st@ 00433484     LIBCMT:crt0msg.obj
 0002:000084bc       ??_C@_0CG@DPMN@R6025?$AN?6?9?5pure?5virtual?5function?5c@ 004334bc     LIBCMT:crt0msg.obj
 0002:000084e4       ??_C@_0DF@CKIP@R6024?$AN?6?9?5not?5enough?5space?5for?5_o@ 004334e4     LIBCMT:crt0msg.obj
 0002:0000851c       ??_C@_0CJ@GGOE@R6019?$AN?6?9?5unable?5to?5open?5console?5@ 0043351c     LIBCMT:crt0msg.obj
 0002:00008548       ??_C@_0CB@LBOB@R6018?$AN?6?9?5unexpected?5heap?5error?$AN?6@ 00433548     LIBCMT:crt0msg.obj
 0002:0000856c       ??_C@_0CN@FPEG@R6017?$AN?6?9?5unexpected?5multithread?5@ 0043356c     LIBCMT:crt0msg.obj
 0002:0000859c       ??_C@_0CM@OBIC@R6016?$AN?6?9?5not?5enough?5space?5for?5th@ 0043359c     LIBCMT:crt0msg.obj
 0002:000085c8       ??_C@_0CB@HPAL@?$AN?6abnormal?5program?5termination?$AN?6@ 004335c8     LIBCMT:crt0msg.obj
 0002:000085ec       ??_C@_0CM@JOOB@R6009?$AN?6?9?5not?5enough?5space?5for?5en@ 004335ec     LIBCMT:crt0msg.obj
 0002:00008618       ??_C@_0CK@OIBL@R6008?$AN?6?9?5not?5enough?5space?5for?5ar@ 00433618     LIBCMT:crt0msg.obj
 0002:00008644       ??_C@_0CF@LKPB@R6002?$AN?6?9?5floating?5point?5not?5load@ 00433644     LIBCMT:crt0msg.obj
 0002:0000866c       ??_C@_0CF@JPDF@Microsoft?5Visual?5C?$CL?$CL?5Runtime?5Lib@ 0043366c     LIBCMT:crt0msg.obj
 0002:00008694       ??_C@_02JJJH@?6?6?$AA@     00433694     LIBCMT:crt0msg.obj
 0002:00008698       ??_C@_0BK@DEOK@Runtime?5Error?$CB?6?6Program?3?5?$AA@ 00433698     LIBCMT:crt0msg.obj
 0002:000086b4       ??_C@_03NAME@?4?4?4?$AA@   004336b4     LIBCMT:crt0msg.obj
 0002:000086b8       ??_C@_0BH@NNCD@?$DMprogram?5name?5unknown?$DO?$AA@ 004336b8     LIBCMT:crt0msg.obj
 0002:000086d0       ??_C@_07CJME@H?3mm?3ss?$AA@ 004336d0     LIBCMT:strftime.obj
 0002:000086d8       ??_C@_0BE@MHI@dddd?0?5MMMM?5dd?0?5yyyy?$AA@ 004336d8     LIBCMT:strftime.obj
 0002:000086ec       ??_C@_06HCAD@M?1d?1yy?$AA@ 004336ec     LIBCMT:strftime.obj
 0002:000086f4       ??_C@_02DBLP@PM?$AA@       004336f4     LIBCMT:strftime.obj
 0002:000086f8       ??_C@_02ENLM@AM?$AA@       004336f8     LIBCMT:strftime.obj
 0002:000086fc       ??_C@_08LIDF@December?$AA@ 004336fc     LIBCMT:strftime.obj
 0002:00008708       ??_C@_08NJLI@November?$AA@ 00433708     LIBCMT:strftime.obj
 0002:00008714       ??_C@_07IAMM@October?$AA@  00433714     LIBCMT:strftime.obj
 0002:0000871c       ??_C@_09MKGD@September?$AA@ 0043371c     LIBCMT:strftime.obj
 0002:00008728       ??_C@_06PADP@August?$AA@   00433728     LIBCMT:strftime.obj
 0002:00008730       ??_C@_04PIJO@July?$AA@     00433730     LIBCMT:strftime.obj
 0002:00008738       ??_C@_04ICFP@June?$AA@     00433738     LIBCMT:strftime.obj
 0002:00008740       ??_C@_05JFGC@April?$AA@    00433740     LIBCMT:strftime.obj
 0002:00008748       ??_C@_05FGPD@March?$AA@    00433748     LIBCMT:strftime.obj
 0002:00008750       ??_C@_08PGBA@February?$AA@ 00433750     LIBCMT:strftime.obj
 0002:0000875c       ??_C@_07BPKJ@January?$AA@  0043375c     LIBCMT:strftime.obj
 0002:00008764       ??_C@_08FAKH@Saturday?$AA@ 00433764     LIBCMT:strftime.obj
 0002:00008770       ??_C@_06ONCK@Friday?$AA@   00433770     LIBCMT:strftime.obj
 0002:00008778       ??_C@_08CCFO@Thursday?$AA@ 00433778     LIBCMT:strftime.obj
 0002:00008784       ??_C@_09PBIN@Wednesday?$AA@ 00433784     LIBCMT:strftime.obj
 0002:00008790       ??_C@_07BMBC@Tuesday?$AA@  00433790     LIBCMT:strftime.obj
 0002:00008798       ??_C@_06CHLK@Monday?$AA@   00433798     LIBCMT:strftime.obj
 0002:000087a0       ??_C@_06OOEM@Sunday?$AA@   004337a0     LIBCMT:strftime.obj
 0002:000087d8       ___dnames                  004337d8     LIBCMT:timeset.obj
 0002:000087f0       ___mnames                  004337f0     LIBCMT:timeset.obj
 0002:00008818       ??_C@_0BD@NJFP@GetLastActivePopup?$AA@ 00433818     LIBCMT:crtmbox.obj
 0002:0000882c       ??_C@_0BA@GILI@GetActiveWindow?$AA@ 0043382c     LIBCMT:crtmbox.obj
 0002:0000883c       ??_C@_0L@HKL@user32?4dll?$AA@ 0043383c     LIBCMT:crtmbox.obj
 0002:00008848       ??_C@_06PAPI@1?$CDQNAN?$AA@ 00433848     LIBCMT:x10fout.obj
 0002:00008850       ??_C@_05BGNL@1?$CDINF?$AA@ 00433850     LIBCMT:x10fout.obj
 0002:00008858       ??_C@_05EDPF@1?$CDIND?$AA@ 00433858     LIBCMT:x10fout.obj
 0002:00008860       ??_C@_06LKFM@1?$CDSNAN?$AA@ 00433860     LIBCMT:x10fout.obj
 0002:00009f18       __IMPORT_DESCRIPTOR_KERNEL32 00434f18     kernel32:KERNEL32.dll
 0002:00009f2c       __IMPORT_DESCRIPTOR_USER32 00434f2c     user32:USER32.dll
 0002:00009f40       __IMPORT_DESCRIPTOR_ADVAPI32 00434f40     advapi32:ADVAPI32.dll
 0002:00009f54       __IMPORT_DESCRIPTOR_SHELL32 00434f54     shell32:SHELL32.dll
 0002:00009f68       __IMPORT_DESCRIPTOR_WINMM  00434f68     winmm:WINMM.dll
 0002:00009f7c       __IMPORT_DESCRIPTOR_VERSION 00434f7c     Version:VERSION.dll
 0002:00009f90       __IMPORT_DESCRIPTOR_SETUPAPI 00434f90     setupapi:SETUPAPI.dll
 0002:00009fa4       __IMPORT_DESCRIPTOR_ole32  00434fa4     ole32:ole32.dll
 0002:00009fb8       __NULL_IMPORT_DESCRIPTOR   00434fb8     kernel32:KERNEL32.dll
 0003:00000000       ___xc_a                    00436000     LIBCMT:crt0init.obj
 0003:00000028       ___xc_z                    00436028     LIBCMT:crt0init.obj
 0003:0000002c       ___xi_a                    0043602c     LIBCMT:crt0init.obj
 0003:00000040       ___xi_z                    00436040     LIBCMT:crt0init.obj
 0003:00000044       ___xl_a                    00436044     LIBCMT:tlssup.obj
 0003:00000048       ___xl_z                    00436048     LIBCMT:tlssup.obj
 0003:0000004c       ___xp_a                    0043604c     LIBCMT:crt0init.obj
 0003:00000054       ___xp_z                    00436054     LIBCMT:crt0init.obj
 0003:00000058       ___xt_a                    00436058     LIBCMT:crt0init.obj
 0003:00000060       ___xt_z                    00436060     LIBCMT:crt0init.obj
 0003:00000070       ?jgxUseDibSection@@3HA     00436070     j_dibsurf.obj
 0003:00000074       ?JMeshTable@@3PAY03GA      00436074     j_objman.obj
 0003:00000094       ?JMeshTable8x8@@3PAY07GA   00436094     j_objman.obj
 0003:00000138       ?spBuildDateString@@3PBDB  00436138     BuildDate.obj
 0003:0000013c       ??_C@_0L@CBED@20180912?98?$AA@ 0043613c     BuildDate.obj
 0003:00000148       ??_C@_0BH@PBLF@incorrect?5length?5check?$AA@ 00436148     zlib:inflate.obj
 0003:00000160       ??_C@_0BF@OBFI@incorrect?5data?5check?$AA@ 00436160     zlib:inflate.obj
 0003:00000178       ??_C@_0BO@EEIF@invalid?5distance?5too?5far?5back?$AA@ 00436178     zlib:inflate.obj
 0003:00000198       ??_C@_0BG@EGK@invalid?5distance?5code?$AA@ 00436198     zlib:inflate.obj
 0003:000001b0       ??_C@_0BM@CHJP@invalid?5literal?1length?5code?$AA@ 004361b0     zlib:inflate.obj
 0003:000001cc       ??_C@_0BG@DILP@invalid?5distances?5set?$AA@ 004361cc     zlib:inflate.obj
 0003:000001e4       ??_C@_0BM@BLEK@invalid?5literal?1lengths?5set?$AA@ 004361e4     zlib:inflate.obj
 0003:00000200       ??_C@_0CF@OIBI@invalid?5code?5?9?9?5missing?5end?9of?9b@ 00436200     zlib:inflate.obj
 0003:00000228       ??_C@_0BK@BNJN@invalid?5bit?5length?5repeat?$AA@ 00436228     zlib:inflate.obj
 0003:00000244       ??_C@_0CE@LAKP@too?5many?5length?5or?5distance?5symb@ 00436244     zlib:inflate.obj
 0003:00000268       ??_C@_0BJ@PEEP@invalid?5code?5lengths?5set?$AA@ 00436268     zlib:inflate.obj
 0003:00000284       ??_C@_0BN@DBOJ@invalid?5stored?5block?5lengths?$AA@ 00436284     zlib:inflate.obj
 0003:000002a4       ??_C@_0BD@IFBC@invalid?5block?5type?$AA@ 004362a4     zlib:inflate.obj
 0003:000002b8       ??_C@_0BE@GABH@header?5crc?5mismatch?$AA@ 004362b8     zlib:inflate.obj
 0003:000002cc       ??_C@_0BJ@LBGI@unknown?5header?5flags?5set?$AA@ 004362cc     zlib:inflate.obj
 0003:000002e8       ??_C@_0BH@NLIB@incorrect?5header?5check?$AA@ 004362e8     zlib:inflate.obj
 0003:00000300       ??_C@_0BE@FAJE@invalid?5window?5size?$AA@ 00436300     zlib:inflate.obj
 0003:00000314       ??_C@_0BL@KPEJ@unknown?5compression?5method?$AA@ 00436314     zlib:inflate.obj
 0003:00000330       ??_C@_0BF@HPBB@incompatible?5version?$AA@ 00436330     zlib:zutil.obj
 0003:00000348       ??_C@_0N@EHHN@buffer?5error?$AA@ 00436348     zlib:zutil.obj
 0003:00000358       ??_C@_0BE@EMHE@insufficient?5memory?$AA@ 00436358     zlib:zutil.obj
 0003:0000036c       ??_C@_0L@EBEB@data?5error?$AA@ 0043636c     zlib:zutil.obj
 0003:00000378       ??_C@_0N@OPOA@stream?5error?$AA@ 00436378     zlib:zutil.obj
 0003:00000388       ??_C@_0L@DFEP@file?5error?$AA@ 00436388     zlib:zutil.obj
 0003:00000394       ??_C@_0L@JPFB@stream?5end?$AA@ 00436394     zlib:zutil.obj
 0003:000003a0       ??_C@_0BA@FKCH@need?5dictionary?$AA@ 004363a0     zlib:zutil.obj
 0003:000003b0       __NLG_Destination          004363b0     LIBCMT:exsup.obj
 0003:000003c0       __fltused                  004363c0     LIBCMT:fpinit.obj
 0003:000003c4       __ldused                   004363c4     LIBCMT:fpinit.obj
 0003:000003c8       __FPinit                   004363c8     LIBCMT:fpinit.obj
 0003:000003cc       __FPmtinit                 004363cc     LIBCMT:fpinit.obj
 0003:000003d0       __FPmtterm                 004363d0     LIBCMT:fpinit.obj
 0003:000005f0       __aexit_rtn                004365f0     LIBCMT:wincrt0.obj
 0003:000005f4       ___app_type                004365f4     LIBCMT:wincrt0.obj
 0003:00000610       ___tlsindex                00436610     LIBCMT:tidtable.obj
 0003:00000614       ?__pInconsistency@@3P6AXXZA 00436614     LIBCMT:hooks.obj
 0003:00000618       __amblksiz                 00436618     LIBCMT:heapinit.obj
 0003:00000620       ___old_small_block_heap    00436620     LIBCMT:sbheap.obj
 0003:00002644       ___old_sbh_threshold       00438644     LIBCMT:sbheap.obj
 0003:00002648       __locktable                00438648     LIBCMT:mlock.obj
 0003:00002708       __cfltcvt_tab              00438708     LIBCMT:cmiscdat.obj
 0003:00002888       __XcptActTab               00438888     LIBCMT:winxfltr.obj
 0003:00002900       __First_FPE_Indx           00438900     LIBCMT:winxfltr.obj
 0003:00002904       __Num_FPE                  00438904     LIBCMT:winxfltr.obj
 0003:00002908       __XcptActTabSize           00438908     LIBCMT:winxfltr.obj
 0003:0000290c       __XcptActTabCount          0043890c     LIBCMT:winxfltr.obj
 0003:00002910       __pctype                   00438910     LIBCMT:ctype.obj
 0003:00002914       __pwctype                  00438914     LIBCMT:ctype.obj
 0003:00002918       __ctype                    00438918     LIBCMT:ctype.obj
 0003:00002b1c       ___mb_cur_max              00438b1c     LIBCMT:nlsdata1.obj
 0003:00002b20       ___decimal_point           00438b20     LIBCMT:nlsdata1.obj
 0003:00002b24       ___decimal_point_length    00438b24     LIBCMT:nlsdata1.obj
 0003:00002b28       ___nullstring              00438b28     LIBCMT:output.obj
 0003:00002b2c       ___wnullstring             00438b2c     LIBCMT:output.obj
 0003:00002b30       __iob                      00438b30     LIBCMT:_file.obj
 0003:00002dc0       ___badioinfo               00438dc0     LIBCMT:ioinit.obj
 0003:00002ea8       ___lc_time_curr            00438ea8     LIBCMT:strftime.obj
 0003:00002eb0       ___lc_time_c               00438eb0     LIBCMT:strftime.obj
 0003:00002f60       ___lconv_static_decimal    00438f60     LIBCMT:lconv.obj
 0003:00002f68       ___lconv_c                 00438f68     LIBCMT:lconv.obj
 0003:00002f98       ___lconv                   00438f98     LIBCMT:lconv.obj
 0003:00002fa0       __timezone                 00438fa0     LIBCMT:timeset.obj
 0003:00002fa4       __daylight                 00438fa4     LIBCMT:timeset.obj
 0003:00002fa8       __dstbias                  00438fa8     LIBCMT:timeset.obj
 0003:0000302c       __tzname                   0043902c     LIBCMT:timeset.obj
 0003:00003054       __lpdays                   00439054     LIBCMT:days.obj
 0003:00003088       __days                     00439088     LIBCMT:days.obj
 0003:000030c0       __pow10pos                 004390c0     LIBCMT:constpow.obj
 0003:00003220       __pow10neg                 00439220     LIBCMT:constpow.obj
 0003:000033d4       ?jgxSurfaceType@@3HA       004393d4     j_objman.obj
 0003:000033d8       ?nullString@@3VJString@@A  004393d8     j_str.obj
 0003:00003490       ?nullString@@3VJWString@@A 00439490     j_wstr.obj
 0003:00003b18       ?g_ExceptionRecord@@3U_EXCEPTION_RECORD@@A 00439b18     sp_se.obj
 0003:00003b68       ?g_TranslateProc@@3P6AXKPAU_EXCEPTION_RECORD@@PAG@ZA 00439b68     sp_se.obj
 0003:00004f78       ?app@@3VCSSPHApp@@A        0043af78     ssph.obj
 0003:00004ff0       _g_pfnGetSystemMetrics     0043aff0     ssph.obj
 0003:00004ff4       _g_pfnMonitorFromWindow    0043aff4     ssph.obj
 0003:00004ff8       _g_pfnMonitorFromRect      0043aff8     ssph.obj
 0003:00004ffc       _g_pfnMonitorFromPoint     0043affc     ssph.obj
 0003:00005000       _g_pfnGetMonitorInfo       0043b000     ssph.obj
 0003:00005004       _g_pfnEnumDisplayMonitors  0043b004     ssph.obj
 0003:00005008       _g_pfnEnumDisplayDevices   0043b008     ssph.obj
 0003:0000500c       _g_fMultiMonInitDone       0043b00c     ssph.obj
 0003:00005010       _g_fMultimonPlatformNT     0043b010     ssph.obj
 0003:00005014       ?g_hook@@3PAUHHOOK__@@A    0043b014     ssph.obj
 0003:00005018       ?g_hLha@@3PAUHINSTANCE__@@A 0043b018     kei.obj
 0003:0000501c       ?g_pCallback@@3P6AHIIPAX@ZA 0043b01c     kei.obj
 0003:00005020       ?g_pCallbackFilter@@3P6AHPBDHPAX@ZA 0043b020     kei.obj
 0003:00005024       ?g_pCallbackUserPointer@@3PAXA 0043b024     kei.obj
 0003:00005028       ?g_pCallbackFilterUserPointer@@3PAXA 0043b028     kei.obj
 0003:0000502c       ?g_procArc@@3P6GHQAUHWND__@@PBDPADK@ZA 0043b02c     kei.obj
 0003:00005030       ?g_procSetCursorMode@@3P6GHH@ZA 0043b030     kei.obj
 0003:00005034       ?g_procGetFileCount@@3P6GHPBD@ZA 0043b034     kei.obj
 0003:00005038       ?g_procSetEnumMembersProc@@3P6GHP6GHPAX@Z@ZA 0043b038     kei.obj
 0003:0000503c       ?g_procClearEnumMembersProc@@3P6GHXZA 0043b03c     kei.obj
 0003:00005040       ?g_maxCount@@3IA           0043b040     kei.obj
 0003:00005044       ?g_curCount@@3IA           0043b044     kei.obj
 0003:00005048       ?g_isCancel@@3_NA          0043b048     kei.obj
 0003:00005050       ___fastflag                0043b050     LIBCMT:fpinit.obj
 0003:00005054       __adjust_fdiv              0043b054     LIBCMT:fpinit.obj
 0003:00005068       __tls_index                0043b068     LIBCMT:tlssup.obj
 0003:00005098       __aenvptr                  0043b098     LIBCMT:wincrt0.obj
 0003:0000509c       __wenvptr                  0043b09c     LIBCMT:wincrt0.obj
 0003:000050a0       ___error_mode              0043b0a0     LIBCMT:wincrt0.obj
 0003:000050a4       __umaskval                 0043b0a4     LIBCMT:crt0dat.obj
 0003:000050a8       __osver                    0043b0a8     LIBCMT:crt0dat.obj
 0003:000050ac       __winver                   0043b0ac     LIBCMT:crt0dat.obj
 0003:000050b0       __winmajor                 0043b0b0     LIBCMT:crt0dat.obj
 0003:000050b4       __winminor                 0043b0b4     LIBCMT:crt0dat.obj
 0003:000050b8       ___argc                    0043b0b8     LIBCMT:crt0dat.obj
 0003:000050bc       ___argv                    0043b0bc     LIBCMT:crt0dat.obj
 0003:000050c0       ___wargv                   0043b0c0     LIBCMT:crt0dat.obj
 0003:000050c4       __environ                  0043b0c4     LIBCMT:crt0dat.obj
 0003:000050c8       ___initenv                 0043b0c8     LIBCMT:crt0dat.obj
 0003:000050cc       __wenviron                 0043b0cc     LIBCMT:crt0dat.obj
 0003:000050d0       ___winitenv                0043b0d0     LIBCMT:crt0dat.obj
 0003:000050d4       __pgmptr                   0043b0d4     LIBCMT:crt0dat.obj
 0003:000050d8       __wpgmptr                  0043b0d8     LIBCMT:crt0dat.obj
 0003:000050dc       __exitflag                 0043b0dc     LIBCMT:crt0dat.obj
 0003:000050e0       __C_Termination_Done       0043b0e0     LIBCMT:crt0dat.obj
 0003:000050e4       __C_Exit_Done              0043b0e4     LIBCMT:crt0dat.obj
 0003:000050e8       __newmode                  0043b0e8     LIBCMT:_newmode.obj
 0003:000050ec       ?_pnhHeap@@3P6AHI@ZA       0043b0ec     LIBCMT:handler.obj
 0003:0000515c       ___lc_handle               0043b15c     LIBCMT:nlsdata2.obj
 0003:00005174       ___lc_codepage             0043b174     LIBCMT:nlsdata2.obj
 0003:00005178       ___lc_collate_cp           0043b178     LIBCMT:nlsdata2.obj
 0003:00005180       ___lc_time_intl            0043b180     LIBCMT:inittime.obj
 0003:0000519c       ___lc_id                   0043b19c     LIBCMT:nlsdata3.obj
 0003:000051e4       __cflush                   0043b1e4     LIBCMT:_file.obj
 0003:000051e8       __stdbuf                   0043b1e8     LIBCMT:_sftbuf.obj
 0003:000052f8       __adbgmsg                  0043b2f8     LIBCMT:crt0msg.obj
 0003:00005308       ___lconv_static_null       0043b308     LIBCMT:lconv.obj
 0003:00005314       __commode                  0043b314     LIBCMT:ncommode.obj
 0003:000053e8       __fmode                    0043b3e8     LIBCMT:txtmode.obj
 0003:000053f0       ??_B?1???id@?$ctype@G@std@@$D@@9@51 0043b3f0     <common>
 0003:00005400       ___pioinfo                 0043b400     <common>
 0003:00005500       __nhandle                  0043b500     <common>
 0003:00005504       ___piob                    0043b504     <common>
 0003:00005520       __bufin                    0043b520     <common>
 0003:00006520       __nstream                  0043c520     <common>
 0003:00006524       ___sbh_sizeHeaderList      0043c524     <common>
 0003:00006528       ___sbh_indGroupDefer       0043c528     <common>
 0003:0000652c       ___sbh_pHeaderScan         0043c52c     <common>
 0003:00006530       ___sbh_pHeaderDefer        0043c530     <common>
 0003:00006534       ___sbh_cntHeaderList       0043c534     <common>
 0003:00006538       ___sbh_pHeaderList         0043c538     <common>
 0003:0000653c       ___sbh_threshold           0043c53c     <common>
 0003:00006540       __crtheap                  0043c540     <common>
 0003:00006544       ___active_heap             0043c544     <common>
 0003:00006548       ___env_initialized         0043c548     <common>
 0003:0000654c       ___mbctype_initialized     0043c54c     <common>
 0003:00006550       ___onexitend               0043c550     <common>
 0003:00006554       ___onexitbegin             0043c554     <common>
 0003:00006558       __acmdln                   0043c558     <common>
 0003:0000655c       ___setlc_active            0043c55c     <common>
 0003:00006560       ___unguarded_readlc_active 0043c560     <common>
 0003:00006564       ___mbcodepage              0043c564     <common>
 0003:00006570       ___mbulinfo                0043c570     <common>
 0003:0000657c       ___ismbcodepage            0043c57c     <common>
 0003:00006580       __mbcasemap                0043c580     <common>
 0003:00006680       __mbctype                  0043c680     <common>
 0003:00006784       ___mblcid                  0043c784     <common>
 0004:00000000       __tls_start                0043d000     LIBCMT:tlssup.obj
 0004:00001ce0       __tls_end                  0043ece0     LIBCMT:tlssup.obj

 entry point at        0001:00020331

 Static symbols

 0001:000153a0       _unzOpenInternal           004163a0 f   unzip.obj
 0001:00015870       _unz64local_getShort       00416870 f   unzip.obj
 0001:000158d0       _unz64local_getByte        004168d0 f   unzip.obj
 0001:00015920       _unz64local_getLong        00416920 f   unzip.obj
 0001:000159c0       _unz64local_getLong64      004169c0 f   unzip.obj
 0001:00015b30       _unz64local_SearchCentralDir 00416b30 f   unzip.obj
 0001:00015ce0       _unz64local_SearchCentralDir64 00416ce0 f   unzip.obj
 0001:00016040       _unz64local_GetCurrentFileInfoInternal 00417040 f   unzip.obj
 0001:00016500       _unz64local_DosDateToTmuDate 00417500 f   unzip.obj
 0001:000169d0       _unz64local_CheckCurrentFileCoherencyHeader 004179d0 f   unzip.obj
 0001:00015360       _$E19                      00416360 f   kei.obj
 0001:00015380       _$E18                      00416380 f   kei.obj
 0001:00013f50       _fread_file_func           00414f50 f   ioapi.obj
 0001:00013f70       _fwrite_file_func          00414f70 f   ioapi.obj
 0001:00013f90       _fclose_file_func          00414f90 f   ioapi.obj
 0001:00013fb0       _ferror_file_func          00414fb0 f   ioapi.obj
 0001:00014000       _fopen64_file_func         00415000 f   ioapi.obj
 0001:00014050       _ftell64_file_func         00415050 f   ioapi.obj
 0001:00014070       _fseek64_file_func         00415070 f   ioapi.obj
 0001:000139e0       ?SSPH_ScanURL_FindURL@@YIHPADAAVJString@@@Z 004149e0 f   ssph_url.obj
 0001:00013c80       ?SSPH_ScanURL_FindURLSub@@YIHAAVJTokenStream@@JAAVJString@@@Z 00414c80 f   ssph_url.obj
 0001:00013ce0       ?SSPH_ScanURL_FindURL_ExtractURL@@YIHPADAAVJString@@@Z 00414ce0 f   ssph_url.obj
 0001:00012b30       _$E4                       00413b30 f   ssph.obj
 0001:00012b40       _$E1                       00413b40 f   ssph.obj
 0001:00012b50       _$E3                       00413b50 f   ssph.obj
 0001:00012b60       _$E2                       00413b60 f   ssph.obj
 0001:00012f10       ?SSPH_UnhandledExceptionFilter@@YGJPAU_EXCEPTION_POINTERS@@@Z 00413f10 f   ssph.obj
 0001:00011da0       _$E2                       00412da0 f   sp_utils.obj
 0001:000123a0       ?split_charscan@@YAPAGPAGPBG_N@Z 004133a0 f   sp_utils.obj
 0001:00012490       ?CreateProcessWrapperEvent@@YAAAVSPEventObject@@XZ 00413490 f   sp_utils.obj
 0001:000124e0       _$E8                       004134e0 f   sp_utils.obj
 0001:000126d0       _$E10                      004136d0 f   sp_utils.obj
 0001:000126e0       _$E9                       004136e0 f   sp_utils.obj
 0001:00011af0       _$E2                       00412af0 f   sp_urltranslate.obj
 0001:0000fea0       _$E2                       00410ea0 f   sp_sysinfo.obj
 0001:000107d0       ?SPSystemInfo_GetCPUName@@YIPADPAD@Z 004117d0 f   sp_sysinfo.obj
 0001:000108e0       ?SPSystemInfo_GetCpuid@@YAHKPAK000@Z 004118e0 f   sp_sysinfo.obj
 0001:000109c0       ?SPSystemInfo_GetUpTime@@YAHAA_K@Z 004119c0 f   sp_sysinfo.obj
 0001:00010b10       ?SPSystemInfo_GetDllVersion@@YIKPBD@Z 00411b10 f   sp_sysinfo.obj
 0001:00010cd0       ?SPSystemInfo_GetCpuClockFromPerfCounter@@YIKXZ 00411cd0 f   sp_sysinfo.obj
 0001:0000c790       ?SPShiori_CheckAliasFileName@@YIHPBD0AAVJString@@@Z 0040d790 f   sp_shiori.obj
 0001:0000c940       ?SPShiori_CompleteCommonName@@YIHPBDAAVJString@@@Z 0040d940 f   sp_shiori.obj
 0001:0000caa0       ?SPShiori_CallConstructSEH@@YIHP6AHXZ@Z 0040daa0 f   sp_shiori.obj
 0001:0000e9f0       ?SPShiori_HookAPICallReal@@YAXPAXW4SPSHIORI_HOOKTYPE@@@Z 0040f9f0 f   sp_shiori.obj
 0001:0000ee30       ?SPShiori_MessageBoxA@@YGHPAUHWND__@@PAD1I@Z 0040fe30 f   sp_shiori.obj
 0001:0000ee60       ?SPShiori_MessageBoxW@@YGHPAUHWND__@@PAG1I@Z 0040fe60 f   sp_shiori.obj
 0001:0000ee90       ?SPShiori_SetWindowsHookExA@@YGPAUHHOOK__@@HP6GJHIJ@ZPAUHINSTANCE__@@K@Z 0040fe90 f   sp_shiori.obj
 0001:0000ee90       ?SPShiori_SetWindowsHookExW@@YGPAUHHOOK__@@HP6GJHIJ@ZPAUHINSTANCE__@@K@Z 0040fe90 f   sp_shiori.obj
 0001:0000eea0       ?SPShiori_UnhookWindowsHookEx@@YGHPAUHHOOK__@@@Z 0040fea0 f   sp_shiori.obj
 0001:0000eeb0       ?SPShiori_GetProcAddress@@YGP6GHXZPAUHINSTANCE__@@PAD@Z 0040feb0 f   sp_shiori.obj
 0001:0000ef00       ?SPShiori_PdhVbGetDoubleCounterValue@@YGNPAXPAJ@Z 0040ff00 f   sp_shiori.obj
 0001:0000ef10       ?SPShiori_PdhVbAddCounter@@YGJPAXPBDPAPAX@Z 0040ff10 f   sp_shiori.obj
 0001:0000ef30       ?SPShiori_LoadLibraryA@@YGPAUHINSTANCE__@@PAD@Z 0040ff30 f   sp_shiori.obj
 0001:0000ef80       ?SPShiori_IsSystemModule@@YA_NPAUHINSTANCE__@@@Z 0040ff80 f   sp_shiori.obj
 0001:0000efe0       ?SPShiori_LoadCompatModuleA@@YAPAUHINSTANCE__@@PAD@Z 0040ffe0 f   sp_shiori.obj
 0001:0000eff0       ?SPShiori_LoadLibraryW@@YGPAUHINSTANCE__@@PAG@Z 0040fff0 f   sp_shiori.obj
 0001:0000f040       ?SPShiori_LoadCompatModuleW@@YAPAUHINSTANCE__@@PAG@Z 00410040 f   sp_shiori.obj
 0001:0000f120       ?SPShiori_LoadLibraryExA@@YGPAUHINSTANCE__@@PADPAXK@Z 00410120 f   sp_shiori.obj
 0001:0000f180       ?SPShiori_LoadLibraryExW@@YGPAUHINSTANCE__@@PAGPAXK@Z 00410180 f   sp_shiori.obj
 0001:0000f1e0       ?SPShiori_GetModuleFileNameA_FIRST@@YGKPAUHINSTANCE__@@PADK@Z 004101e0 f   sp_shiori.obj
 0001:0000f250       ?SPShiori_GetModuleFileNameA_FUTABA@@YGKPAUHINSTANCE__@@PADK@Z 00410250 f   sp_shiori.obj
 0001:0000f2c0       ?SPShiori_ReplaceUPXEntry@@YAXPAXKPAPAX1PA_N@Z 004102c0 f   sp_shiori.obj
 0001:0000f380       ?sp_memsearch@@YAPAXPAXK0K@Z 00410380 f   sp_shiori.obj
 0001:0000f3e0       ?SPShiori_ReplaceIATEntry@@YAXPAXKPAPAX1PA_N@Z 004103e0 f   sp_shiori.obj
 0001:0000f500       _$E2                       00410500 f   sp_shiori.obj
 0001:0000abc0       ?SPParamManager_ScanToNextReturn@@YIPADPAD@Z 0040bbc0 f   sp_param.obj
 0001:0000a130       ?SPModule_Write@@YAXPAXAAVJString@@@Z 0040b130 f   sp_module.obj
 0001:0000a160       ?SPModule_ReadLine@@YAXPAXAAVJString@@@Z 0040b160 f   sp_module.obj
 0001:000073e0       _$E4                       004083e0 f   sp_findfile.obj
 0001:000073f0       _$E1                       004083f0 f   sp_findfile.obj
 0001:00007400       _$E3                       00408400 f   sp_findfile.obj
 0001:00007410       _$E2                       00408410 f   sp_findfile.obj
 0001:00005710       _$E4                       00406710 f   sp_debugger.obj
 0001:00005720       _$E1                       00406720 f   sp_debugger.obj
 0001:00005750       _$E3                       00406750 f   sp_debugger.obj
 0001:00005760       _$E2                       00406760 f   sp_debugger.obj
 0001:000058b0       ?SPSEDefaultFilterMain@@YIJPAU_EXCEPTION_POINTERS@@PAU_iobuf@@@Z 004068b0 f   sp_debugger.obj
 0001:00005da0       ?SPDebugMakeSystemPath@@YAPBDPBD@Z 00406da0 f   sp_debugger.obj
 0001:00005ea0       ?WriteEnvironmentMain@@YAXPAU_iobuf@@PAX@Z 00406ea0 f   sp_debugger.obj
 0001:00006600       ?SPGetDriveInfoStrFromFlag@@YAPADK@Z 00407600 f   sp_debugger.obj
 0001:00006620       ?SPGetDiskFreeSpace@@YAXPBDAAK1@Z 00407620 f   sp_debugger.obj
 0001:00006700       ?MonitorEnumProc@@YGHPAUHMONITOR__@@PAUHDC__@@PAUtagRECT@@J@Z 00407700 f   sp_debugger.obj
 0001:000067d0       ?DumpDrivers@@YAXPAU_iobuf@@@Z 004077d0 f   sp_debugger.obj
 0001:000068f0       ?CompareAddr@@YAHPBX0@Z    004078f0 f   sp_debugger.obj
 0001:00006910       ?DumpModules@@YAXPAX0PAU_iobuf@@@Z 00407910 f   sp_debugger.obj
 0001:00006b50       ?DumpServices@@YAXPAU_iobuf@@@Z 00407b50 f   sp_debugger.obj
 0001:00006ca0       ?DumpProcesses@@YAXPAU_iobuf@@@Z 00407ca0 f   sp_debugger.obj
 0001:00006f20       ?GetFlagRegState@@YAPADK@Z 00407f20 f   sp_debugger.obj
 0001:000072f0       ?ExtractFileName@@YAXPAD@Z 004082f0 f   sp_debugger.obj
 0001:00005420       _$E2                       00406420 f   sp_adjustpriv.obj
 0001:000030a0       _$E4                       004040a0 f   j_wstr.obj
 0001:000030b0       _$E1                       004040b0 f   j_wstr.obj
 0001:00003180       _$E3                       00404180 f   j_wstr.obj
 0001:00003190       _$E2                       00404190 f   j_wstr.obj
 0001:00003d10       ?JWString_CodePage_Compare@@YIHPBD0@Z 00404d10 f   j_wstr.obj
 0001:00003020       _$E4                       00404020 f   j_wintrd.obj
 0001:00003030       _$E1                       00404030 f   j_wintrd.obj
 0001:00003040       _$E3                       00404040 f   j_wintrd.obj
 0001:00003050       _$E2                       00404050 f   j_wintrd.obj
 0001:00003060       _$E9                       00404060 f   j_wintrd.obj
 0001:00003070       _$E6                       00404070 f   j_wintrd.obj
 0001:00003080       _$E8                       00404080 f   j_wintrd.obj
 0001:00003090       _$E7                       00404090 f   j_wintrd.obj
 0001:000009a0       _$E4                       004019a0 f   j_str.obj
 0001:000009b0       _$E1                       004019b0 f   j_str.obj
 0001:00000a70       _$E3                       00401a70 f   j_str.obj
 0001:00000a80       _$E2                       00401a80 f   j_str.obj
 0001:000018d0       ?sp_mbcjistojms@@YIII@Z    004028d0 f   j_str.obj
 0001:00001bd0       ?sp_mbcjmstojis@@YIII@Z    00402bd0 f   j_str.obj
 0001:0001b5a0       _init_block                0041c5a0 f   zlib:trees.obj
 0001:0001b960       _build_tree                0041c960 f   zlib:trees.obj
 0001:0001bb90       _pqdownheap                0041cb90 f   zlib:trees.obj
 0001:0001bc70       _gen_bitlen                0041cc70 f   zlib:trees.obj
 0001:0001be80       _gen_codes                 0041ce80 f   zlib:trees.obj
 0001:0001bf00       _build_bl_tree             0041cf00 f   zlib:trees.obj
 0001:0001bf80       _scan_tree                 0041cf80 f   zlib:trees.obj
 0001:0001c080       _send_all_trees            0041d080 f   zlib:trees.obj
 0001:0001c2f0       _send_tree                 0041d2f0 f   zlib:trees.obj
 0001:0001c880       _compress_block            0041d880 f   zlib:trees.obj
 0001:0001ccd0       _detect_data_type          0041dcd0 f   zlib:trees.obj
 0001:0001cd50       _bi_reverse                0041dd50 f   zlib:trees.obj
 0001:0001cd80       _bi_flush                  0041dd80 f   zlib:trees.obj
 0001:0001ce10       _bi_windup                 0041de10 f   zlib:trees.obj
 0001:000199b0       _slide_hash                0041a9b0 f   zlib:deflate.obj
 0001:00019a00       _flush_pending             0041aa00 f   zlib:deflate.obj
 0001:00019a80       _fill_window               0041aa80 f   zlib:deflate.obj
 0001:00019c70       _read_buf                  0041ac70 f   zlib:deflate.obj
 0001:00019d00       _deflate_stored            0041ad00 f   zlib:deflate.obj
 0001:0001a110       _deflate_fast              0041b110 f   zlib:deflate.obj
 0001:0001a490       _longest_match             0041b490 f   zlib:deflate.obj
 0001:0001a600       _deflate_slow              0041b600 f   zlib:deflate.obj
 0001:00019700       _crc32_little              0041a700 f   zlib:crc32.obj
 0001:00017b60       _inflateStateCheck         00418b60 f   zlib:inflate.obj
 0001:00019530       _fixedtables               0041a530 f   zlib:inflate.obj
 0001:00019560       _updatewindow              0041a560 f   zlib:inflate.obj
 0001:00027cc7       _x_ismbbtype               00428cc7 f   LIBCMT:ismbbyte.obj
 0001:00026db9       _wcsncnt                   00427db9 f   LIBCMT:w_map.obj
 0001:00026275       __abstract_cw              00427275 f   LIBCMT:ieee87.obj
 0001:00026307       __hw_cw                    00427307 f   LIBCMT:ieee87.obj
 0001:00025ced       _parse_cmdline             00426ced f   LIBCMT:stdargv.obj
 0001:000249f9       _write_char                004259f9 f   LIBCMT:woutput.obj
 0001:00024a19       _write_multi_char          00425a19 f   LIBCMT:woutput.obj
 0001:00024a4a       _write_string              00425a4a f   LIBCMT:woutput.obj
 0001:00024249       _get_int_arg               00425249 f   LIBCMT:output.obj
 0001:00024a83       _get_int64_arg             00425a83 f   LIBCMT:woutput.obj
 0001:000241ab       _write_char                004251ab f   LIBCMT:output.obj
 0001:000241e0       _write_multi_char          004251e0 f   LIBCMT:output.obj
 0001:00024211       _write_string              00425211 f   LIBCMT:output.obj
 0001:00024249       _get_int_arg               00425249 f   LIBCMT:output.obj
 0001:00024a83       _get_int64_arg             00425a83 f   LIBCMT:woutput.obj
 0001:00024256       _get_short_arg             00425256 f   LIBCMT:output.obj
 0001:00023276       _xcptlookup                00424276 f   LIBCMT:winxfltr.obj
 0001:00023088       _strncnt                   00424088 f   LIBCMT:a_map.obj
 0001:00022b10       LeadUp1                    00423b10 f   LIBCMT:memcpy.obj
 0001:00022b3c       LeadUp2                    00423b3c f   LIBCMT:memcpy.obj
 0001:00022b60       LeadUp3                    00423b60 f   LIBCMT:memcpy.obj
 0001:00022bdf       UnwindUp0                  00423bdf f   LIBCMT:memcpy.obj
 0001:00022bcc       UnwindUp1                  00423bcc f   LIBCMT:memcpy.obj
 0001:00022bc4       UnwindUp2                  00423bc4 f   LIBCMT:memcpy.obj
 0001:00022bbc       UnwindUp3                  00423bbc f   LIBCMT:memcpy.obj
 0001:00022bb4       UnwindUp4                  00423bb4 f   LIBCMT:memcpy.obj
 0001:00022bac       UnwindUp5                  00423bac f   LIBCMT:memcpy.obj
 0001:00022ba4       UnwindUp6                  00423ba4 f   LIBCMT:memcpy.obj
 0001:00022b9c       UnwindUp7                  00423b9c f   LIBCMT:memcpy.obj
 0001:00022bf8       TrailUp0                   00423bf8 f   LIBCMT:memcpy.obj
 0001:00022c00       TrailUp1                   00423c00 f   LIBCMT:memcpy.obj
 0001:00022c0c       TrailUp2                   00423c0c f   LIBCMT:memcpy.obj
 0001:00022c20       TrailUp3                   00423c20 f   LIBCMT:memcpy.obj
 0001:00022c98       LeadDown1                  00423c98 f   LIBCMT:memcpy.obj
 0001:00022cb8       LeadDown2                  00423cb8 f   LIBCMT:memcpy.obj
 0001:00022ce0       LeadDown3                  00423ce0 f   LIBCMT:memcpy.obj
 0001:00022d34       UnwindDown7                00423d34 f   LIBCMT:memcpy.obj
 0001:00022d3c       UnwindDown6                00423d3c f   LIBCMT:memcpy.obj
 0001:00022d44       UnwindDown5                00423d44 f   LIBCMT:memcpy.obj
 0001:00022d4c       UnwindDown4                00423d4c f   LIBCMT:memcpy.obj
 0001:00022d54       UnwindDown3                00423d54 f   LIBCMT:memcpy.obj
 0001:00022d5c       UnwindDown2                00423d5c f   LIBCMT:memcpy.obj
 0001:00022d64       UnwindDown1                00423d64 f   LIBCMT:memcpy.obj
 0001:00022d77       UnwindDown0                00423d77 f   LIBCMT:memcpy.obj
 0001:00022d90       TrailDown0                 00423d90 f   LIBCMT:memcpy.obj
 0001:00022d98       TrailDown1                 00423d98 f   LIBCMT:memcpy.obj
 0001:00022da8       TrailDown2                 00423da8 f   LIBCMT:memcpy.obj
 0001:00022dbc       TrailDown3                 00423dbc f   LIBCMT:memcpy.obj
 0001:000227d7       __cftoe2                   004237d7 f   LIBCMT:cvt.obj
 0001:000228ee       __cftof2                   004238ee f   LIBCMT:cvt.obj
 0001:00022a79       __shift                    00423a79 f   LIBCMT:cvt.obj
 0001:00020fa0       _doexit                    00421fa0 f   LIBCMT:crt0dat.obj
 0001:00021057       __initterm                 00422057 f   LIBCMT:crt0dat.obj
 0001:0002060d       ?FindHandler@@YAXPAUEHExceptionRecord@@PAUEHRegistrationNode@@PAU_CONTEXT@@PAXPBU_s_FuncInfo@@EH1@Z 0042160d f   LIBCMT:frame.obj
 0001:000207c0       ?FindHandlerForForeignException@@YAXPAUEHExceptionRecord@@PAUEHRegistrationNode@@PAU_CONTEXT@@PAXPBU_s_FuncInfo@@HH1@Z 004217c0 f   LIBCMT:frame.obj
 0001:0002086a       ?TypeMatch@@YAHPBU_s_HandlerType@@PBU_s_CatchableType@@PBU_s_ThrowInfo@@@Z 0042186a f   LIBCMT:frame.obj
 0001:0001f260       ?FrameUnwindFilter@@YAHPAU_EXCEPTION_POINTERS@@@Z 00420260 f   LIBCMT:ehvecdtr.obj
 0001:00020965       ?CatchIt@@YAXPAUEHExceptionRecord@@PAUEHRegistrationNode@@PAU_CONTEXT@@PAXPBU_s_FuncInfo@@PBU_s_HandlerType@@PBU_s_CatchableType@@PBU_s_TryBlockMapEntry@@H1E@Z 00421965 f   LIBCMT:frame.obj
 0001:000209e0       ?CallCatchBlock@@YAPAXPAUEHExceptionRecord@@PAUEHRegistrationNode@@PAU_CONTEXT@@PBU_s_FuncInfo@@PAXHK@Z 004219e0 f   LIBCMT:frame.obj
 0001:00020afb       ?ExFilterRethrow@@YAHPAU_EXCEPTION_POINTERS@@@Z 00421afb f   LIBCMT:frame.obj
 0001:00020b25       ?BuildCatchObject@@YAXPAUEHExceptionRecord@@PAUEHRegistrationNode@@PBU_s_HandlerType@@PBU_s_CatchableType@@@Z 00421b25 f   LIBCMT:frame.obj
 0001:00020d50       ?AdjustPointer@@YAPAXPAXABUPMD@@@Z 00421d50 f   LIBCMT:frame.obj
 0001:0002045e       _fast_error_exit           0042145e f   LIBCMT:wincrt0.obj
 0001:0001f260       ?ArrayUnwindFilter@@YAHPAU_EXCEPTION_POINTERS@@@Z 00420260 f   LIBCMT:ehvecdtr.obj
 0001:0001f108       _shortsort                 00420108 f   LIBCMT:qsort.obj
 0001:0001f156       _swap                      00420156 f   LIBCMT:qsort.obj
 0001:0001ecd8       _flsall                    0041fcd8 f   LIBCMT:fflush.obj
 0001:0001e946       _ctrlevent_capture@4       0041f946 f   LIBCMT:winsig.obj
 0001:0001eb2a       _siglookup                 0041fb2a f   LIBCMT:winsig.obj
 0001:0001e4aa       _wcstoxl                   0041f4aa f   LIBCMT:wcstol.obj
 0001:0001e277       _strtoxl                   0041f277 f   LIBCMT:strtol.obj
 0001:0001df4a       _getSystemCP               0041ef4a f   LIBCMT:mbctype.obj
 0001:0001df94       _CPtoLCID                  0041ef94 f   LIBCMT:mbctype.obj
 0001:0001dfc7       _setSBCS                   0041efc7 f   LIBCMT:mbctype.obj
 0001:0001dff0       _setSBUpLow                0041eff0 f   LIBCMT:mbctype.obj
 0001:0001d700       LeadUp1                    0041e700 f   LIBCMT:memmove.obj
 0001:0001d72c       LeadUp2                    0041e72c f   LIBCMT:memmove.obj
 0001:0001d750       LeadUp3                    0041e750 f   LIBCMT:memmove.obj
 0001:0001d7cf       UnwindUp0                  0041e7cf f   LIBCMT:memmove.obj
 0001:0001d7bc       UnwindUp1                  0041e7bc f   LIBCMT:memmove.obj
 0001:0001d7b4       UnwindUp2                  0041e7b4 f   LIBCMT:memmove.obj
 0001:0001d7ac       UnwindUp3                  0041e7ac f   LIBCMT:memmove.obj
 0001:0001d7a4       UnwindUp4                  0041e7a4 f   LIBCMT:memmove.obj
 0001:0001d79c       UnwindUp5                  0041e79c f   LIBCMT:memmove.obj
 0001:0001d794       UnwindUp6                  0041e794 f   LIBCMT:memmove.obj
 0001:0001d78c       UnwindUp7                  0041e78c f   LIBCMT:memmove.obj
 0001:0001d7e8       TrailUp0                   0041e7e8 f   LIBCMT:memmove.obj
 0001:0001d7f0       TrailUp1                   0041e7f0 f   LIBCMT:memmove.obj
 0001:0001d7fc       TrailUp2                   0041e7fc f   LIBCMT:memmove.obj
 0001:0001d810       TrailUp3                   0041e810 f   LIBCMT:memmove.obj
 0001:0001d888       LeadDown1                  0041e888 f   LIBCMT:memmove.obj
 0001:0001d8a8       LeadDown2                  0041e8a8 f   LIBCMT:memmove.obj
 0001:0001d8d0       LeadDown3                  0041e8d0 f   LIBCMT:memmove.obj
 0001:0001d924       UnwindDown7                0041e924 f   LIBCMT:memmove.obj
 0001:0001d92c       UnwindDown6                0041e92c f   LIBCMT:memmove.obj
 0001:0001d934       UnwindDown5                0041e934 f   LIBCMT:memmove.obj
 0001:0001d93c       UnwindDown4                0041e93c f   LIBCMT:memmove.obj
 0001:0001d944       UnwindDown3                0041e944 f   LIBCMT:memmove.obj
 0001:0001d94c       UnwindDown2                0041e94c f   LIBCMT:memmove.obj
 0001:0001d954       UnwindDown1                0041e954 f   LIBCMT:memmove.obj
 0001:0001d967       UnwindDown0                0041e967 f   LIBCMT:memmove.obj
 0001:0001d980       TrailDown0                 0041e980 f   LIBCMT:memmove.obj
 0001:0001d988       TrailDown1                 0041e988 f   LIBCMT:memmove.obj
 0001:0001d998       TrailDown2                 0041e998 f   LIBCMT:memmove.obj
 0001:0001d9ac       TrailDown3                 0041e9ac f   LIBCMT:memmove.obj
 0001:0001d19c       _gu_return                 0041e19c f   LIBCMT:exsup.obj
 0001:0001d1a4       __unwind_handler           0041e1a4 f   LIBCMT:exsup.obj
 0001:0001cfb6       ?CatchGuardHandler@@YA?AW4_EXCEPTION_DISPOSITION@@PAUEHExceptionRecord@@PAUCatchGuardRN@@PAX2@Z 0041dfb6 f   LIBCMT:trnsctrl.obj
 0001:0001d091       ?TranslatorGuardHandler@@YA?AW4_EXCEPTION_DISPOSITION@@PAUEHExceptionRecord@@PAUTranslatorGuardRN@@PAX2@Z 0041e091 f   LIBCMT:trnsctrl.obj

 1015 bytes saved through ICF

